:1000000000800020BD010000F5C30000ADC300006A
:10001000ADC30000ADC30000ADC30000ADC3000020
:10002000ADC30000ADC30000ADC30000F5C30000C8
:10003000F5C30000ADC3000075BA000079BB000035
:10004000F5C30000F5C30000F5C30000F5C30000D0
:10005000F5C30000F5C30000F5C30000F5C30000C0
:10006000F5C30000F5C30000F5C30000F5C30000B0
:10007000F5C30000F5C30000F5C30000F5C30000A0
:10008000F5C30000F5C30000F5C30000F5C3000090
:10009000F5C30000F5C30000F5C30000F5C3000080
:1000A000B19F0000BD9F0000F5C30000F5C3000034
:1000B000F5C30000F5C30000F5C30000F5C3000060
:1000C000F5C30000F5C30000F5C30000F5C3000050
:1000D000F5C30000F5C30000F5C30000F5C3000040
:1000E000F5C30000F5C30000F5C30000F5C3000030
:1000F000F5C3000061E40000F5C300008DE50000D9
:10010000F5C30000CDCD0000F5C30000F5C300002D
:10011000F5C30000F5C30000F5C30000F5C30000FF
:10012000F5C30000F5C30000F5C30000F5C30000EF
:10013000F5C30000F5C30000F5C30000F5C30000DF
:10014000F5C30000F5C30000F5C30000F5C30000CF
:1001500065BC000079BC00008DBC0000A1BC0000A3
:10016000F5C30000E9D00000F5C30000F5C30000AE
:10017000F5C30000F5C30000F5C30000F5C300009F
:10018000F5C30000F5C30000F5C30000F5C300008F
:10019000F5C30000F5C30000F5C30000F5C300007F
:1001A000F5C30000F5C30000F5C30000F5C300006F
:1001B000F5C30000F5C30000F5C30000564B4CF238
:1001C000205210B51A804DF628121A8000BF00BFC9
:1001D0000CF014F9514B4FF010621A60504A9A60BB
:1001E000504ADA60504A136813F4807304D14F49BF
:1001F0000B604FF4A85313604D4B1A78110703D5C9
:100200001A7842F008021A704A4B4B492A221A7097
:100210004A4A4B4B8B4204D252F8040F43F8040B6A
:10022000F8E7484B484900228B4202D243F8042B9E
:10023000FAE74649464A002352F8230041F82300D2
:1002400001336F2BF8D1434B434A802103F8011B44
:100250009342FBD1414B3D4A1A60414B8A221A70AE
:10026000A3F5805324225A70A0221A709A7992071B
:10027000FCD59A79D406FCD43A4A937903F00C035E
:10028000082B384BF9D103221A7140225A719A79FE
:100290009006FCD5334A9179324B4906FBD5324A58
:1002A000324911600221516020221A709A7902F0BD
:1002B0000C020C2AFAD12E4B2E4A1A602E4B2F4AD2
:1002C0001A6000225A60072243F8042C2C4AC3F813
:1002D0000C2D62B60CF042FC144B1B68DA0705D5F6
:1002E00028480CF00FFA284B284A1A60284B1B7834
:1002F0005B0609D5244C254B22689A4204D121483B
:100300000CF000FA002323600FF0FAFB0CF07CF8ED
:100310000BF0AAFFFEE700BF0E200540308004402E
:10032000823F04000100002B10D0034014D0034092
:1003300002D0074000E00740049BFF1FC4320100C9
:100340004088FF1F049BFF1FF0A2FF1F0082FF1FBA
:100350000000000000E400E05FE400E008ED00E0E1
:100360000050064000400640448004400000030165
:1003700004800440C010050014E000E0FF76010096
:1003800000002020D035135F1CE00340A5C3945A21
:1003900000F00740FFFFFFFFFFFFFFFFFFFFFFFF32
:1003A000FFFFFFFFFFFFFFFFFFFFFFFFFFFFFFFF5D
:1003B000FFFFFFFFFFFFFFFFFFFFFFFFFFFFFFFF4D
:1003C000FFFFFFFFFFFFFFFFFFFFFFFFFFFFFFFF3D
:1003D000FFFFFFFFFFFFFFFFFFFFFFFFFFFFFFFF2D
:1003E000FFFFFFFFFFFFFFFFFFFFFFFFFFFFFFFF1D
:1003F000FFFFFFFFFFFFFFFFFFFFFFFFFFFFFFFF0D
:10040000FFFFFFFFFFFFFFFFFFFFFFFFDEF9FFFF23
:1004100010B5054C237833B9044B13B10448AFF33E
:1004200000800123237010BD049BFF1F000000000B
:10043000C8320100084B10B51BB108490848AFF39A
:1004400000800848036803B910BD074B002BFBD0A0
:10045000BDE81040184700BF00000000089BFF1FC8
:10046000C8320100049BFF1F0000000038B504469D
:10047000104621700A491D460FF024F901464FF03D
:100480007E500FF0D3F907490FF01CF9E56060606A
:10049000256165610CF0F2FAE061204638BD00BFCD
:1004A000DB0FC9400024744938B50446104621705A
:1004B00009491D460FF006F901464FF07E500FF036
:1004C000B5F906490FF0FEF8E560606025616561E9
:1004D0000CF0D4FAE06138BDDB0FC9400024744948
:1004E00038B503780446032B20D8DFE803F01A1848
:1004F0001002C16840690EF0DBFF0D4905466068D7
:100500000FF094F9014628460FF090F938BD0849DC
:1005100040680FF08BF9E1680FF0D4F838BDC0687F
:1005200038BDC16840690EF0C3FF38BD002038BD3A
:100530000024744970B504460E460CF09FFA054637
:10054000E069281A0FF06AF8E3682361E5616661E3
:10055000A061014660680FF069F90146A06010488B
:100560000FF064F90EF03AFC0EF0DAF80EF04CFFE2
:10057000054601464FF07E500EF09AFF61690FF07C
:10058000A1F82169064628460FF09CF8014630463E
:100590000EF090FFE0602046BDE87040FFF7A0BF7E
:1005A000000080BF08B50E200BF038FD114B1B88F2
:1005B000012B19D0104B1B88984213DB40F6FF71BA
:1005C0008842D4BFC3EB0001C3EB0101C1EB013191
:1005D000C3F57F630F33282091FBF3F1BDE808409A
:1005E0000CF0A2B80021F3E70146BDE80840142052
:1005F0000CF09AB8309DFF1FE09BFF1F10B504461A
:100600000BF00EFB204610BD70B44C88A04220D9E0
:1006100001230133DBB21CB2660031F8144084427E
:100620001D46F6D3A04211D005F10045013D965B71
:1006300031F8151032F81530401AF21A00FB02F0AA
:10064000641A90FBF4F4E01870BC7047905B70BCC7
:10065000704702260125E5E700280CDA064A4342E6
:1006600082FB0320DA17C2EB600000EB4000A3EB33
:100670008000C0F10C007047ABAAAA2A2DE9F04710
:100680000C200BF097FC0C200CF04CF99C4914202A
:100690000CF058F99B499C4809F090F9022103207D
:1006A0000CF0E6F9022104200CF0E2F90221052009
:1006B0000CF0DEF9022106200CF0DAF901210A2003
:1006C0000CF0D6F9012109200CF0D2F901210D20FE
:1006D0000CF0CEF9012128200CF0CAF901211420D8
:1006E0000CF0C6F902210B200CF0C2F901210C20FC
:1006F0000CF0BEF90C2000210CF0A6F904200CF03F
:10070000A9F970B305200CF0A5F9044680B30024C4
:1007100020467E4D287006F0ABFB2B78EBB92046C7
:1007200007F0C8FF7A4B7B491B887B4C09887B4AC2
:100730002170A3F5AF7140F23A7303FB01F382FB22
:100740000312DB17764D7748A3EB621332335A213D
:100750002B6009F0DDFC90B9FEE7BDE8F04709F039
:100760003DB806200CF076F90028CBD10124D0E763
:1007700003200CF06FF9B0FA80F04009C9E76A4A2B
:100780006A481268DFF8F8A100230121FFF78CFE08
:100790000B200CF05FF9011E0CBF012300238AF827
:1007A000003002D111200CF063F9DFF89081604E27
:1007B000604F614D0023C8F8003033603B604FF05C
:1007C000040914E00BF02AFC33681844306009F087
:1007D000010080F0010005F0A1F82B88002B14BF68
:1007E0004B20DC200CF06CF9B9F1010919D00F2075
:1007F0000CF058FB3B6803440E203B600BF00EFCF2
:10080000D8F800309AF800200344C8F800301520CA
:10081000002AD7D111200CF045FB33681844306012
:10082000D5E73B68D8F8002044493068DFF854E148
:100830002D88002BB8BF0333002AB8BF03329210B3
:100840000A603F493F4A0988128800284FEAA303FB
:10085000B8BF03303B6080103B4F30605E1A1944D4
:100860003E60CEF80010394F394E3A49C2EB000EC7
:100870000244C7F800E032600B605DB94FF4FA70D3
:1008800005F05CF805F046F806F0F2FD4FF4AF60B5
:100890000CF016F9304B012504201D600CF0DAF83D
:1008A00010B92E4B20701D702D4B1B881C2B1CD09B
:1008B0002C4C04F1C80523200BF0B0FB44F8040FC6
:1008C00001200CF0FDF8A542F5D1274A274B1078FE
:1008D000187007F0F9FD05F019F845F6BF522449E4
:1008E0002448BDE8F0470BF051B9234B1888002885
:1008F000DED0224BC0B2197807F02EFDD8E700BF3A
:10090000001B3746801A06000C90FF1F649BFF1FD8
:10091000849DFF1F649DFF1FB49BFF1FB5814E1B6D
:100920009089FF1FD49BFF1F2489FF1FF89CFF1F86
:10093000209BFF1F509DFF1F269DFF1F389BFF1F01
:10094000A289FF1F2C89FF1F549DFF1FAC9DFF1F15
:10095000B89BFF1FA09DFF1F5C9DFF1F529BFF1FA9
:10096000629DFF1FEC9BFF1FE49CFF1FCA9CFF1FA3
:10097000A5050000789DFF1FBC9BFF1F809BFF1FEC
:10098000409DFF1FCC9CFF1FF0B40E8886420DD205
:1009900003F10043013B31F81350854202D9F0BC0A
:1009A000FFF732BE32F81300F0BC70471088F0BC7D
:1009B000704700BF094B1B880C2B09D8084A80B22E
:1009C00052F8232028B143F6FE73984203D9108CC5
:1009D0007047108870470349FFF716BE609BFF1FE2
:1009E000200E010024100100374A38491088384A87
:1009F000F8B5384B12881B68834248DB9342A8BF86
:100A0000134698420B60C8BF002342DD101AB0F5B0
:100A1000804FAABF9B03C3EB8333013093FBF0F0FD
:100A2000FFF7C8FF2C4B2D4F1C883B68C0F3C61541
:100A300005FB04F47F2CA8BF7F249D42064608D006
:100A4000274B1B88002B38D1264B1B88002B30D11D
:100A50003D60254D2B689E4205D0214B1B885A1FB7
:100A6000032A1DD92E60214D2B689C420ED0204BAD
:100A7000188848B11A4B1F4A1B88D35C834203D0A5
:100A8000C0B2E1B207F068FC2C60F8BDF8BD0346C7
:100A900008609A42D4BFC0EB0203C0EB0303B5E782
:100AA000144AD05C2030C0B206F07F0107F054FC3D
:100AB000D8E7284607F0C4FCCAE70E4A2946D05CAE
:100AC00007F04AFCC0E700BFE09BFF1F289BFF1F09
:100AD0008C9DFF1F2C9DFF1F709BFF1F949BFF1F72
:100AE0001A9DFF1FD69BFF1F989DFF1FD89BFF1FBE
:100AF000669DFF1F9489FF1F2DE9F04F172089B0D5
:100B00000CF0D0F9AF4B186016200CF0CBF9AE4BBF
:100B1000AE4A1B8810600C2B00F03B81AC4BAD4AF9
:100B200019880093AC4B52F8214000221A70AB4B4D
:100B3000AB4D1B88AB4A2E88013B32F91370002E57
:100B40005CD0A94BA94A1B88A9491278013B31F90D
:100B50001380002A40F0DF8011200CF0A3F9A54B90
:100B60000193D3F800A00646B24540F3DF80A24BC4
:100B7000DFF8A4921B88A14A012BD9F80030B2F803
:100B800000B09F4A02922046C8EB030800F09A8208
:100B90000EF044FD029A52F82B100EF093FD014620
:100BA00000200EF085FC0EF053FFCAEB0802B045A2
:100BB000B8BFB0469042CAEB080880F2968200FBAC
:100BC0000888013298FBF2F08E4BDFF850820293D6
:100BD000D8F80030034403EBD3735B10C8F800303F
:100BE0002B88012B12D1884BDFF834B20393874B4B
:100BF000DBF8005004934FF0000A47E07D4B01936F
:100C0000DFF814927F4BDFF8148202937E4B03933C
:100C10001D460F200CF046F92B689842824641DAB7
:100C2000754A1288012A00F01D82744A05931288C1
:100C3000734D049220460EF0F1FC049ADFF8E0B107
:100C400055F82210DBF800500EF03CFD0146002064
:100C50000EF02EFC0EF0FCFEEF1B059B5745A7EB9C
:100C60000302B8BF5746FF1A9042BABF013200FBD9
:100C70000777474397FBF2F7D8F80020634B0493BC
:100C8000BB1803EBD3735B10C8F80030604B1B88B4
:100C9000013B032B00F2B082DFE813F06301A901EE
:100CA000C4008601594B04931B68984240F3C281EB
:100CB000514A1288012A00F0A682504A07931188EF
:100CC0004F4A0691204605920EF0A8FC059A069917
:100CD000DFF84CB152F82110DBF800500EF0F2FCB6
:100CE0000EF0B6FE079B2F445745A7EB0302A8BFA3
:100CF0005746FF1AD8F800309042BABF00FB07777A
:100D00000132474397FBF2F73B4403EBD3735B108D
:100D1000C8F80030BAE715200BF080F9354B019385
:100D2000D3F800A00646B2453FF721AF354B0293FA
:100D3000D3F800A0B24580F289812F4BDFF8D8901C
:100D40001B882E4A012BD9F80030B2F800B02C4A8B
:100D500003922046984400F070820EF05FFC039AE4
:100D600052F82B100EF0AEFC0EF072FEB045CAEB3E
:100D70000802A8BFB046CAEB08089042B6BF00FB05
:100D8000088800FB08F8013298FBF2F0DFF88C804D
:100D90001EE7204B1B78002B3FF4C0AE0C4B0D4AD6
:100DA000198800930C4B52F8210001221A700EF0A2
:100DB00035FC4FF07C510EF085FC0EF049FE0446E8
:100DC000B5E600BF8C9BFF1F629DFF1FA89DFF1F04
:100DD000909BFF1F5889FF1F329BFF1FA089FF1F99
:100DE000D49CFF1F0C120100A689FF1F409DFF1F0E
:100DF00000100100AC9DFF1FC49BFF1F5C9BFF1FE9
:100E000024120100B89BFF1F549DFF1FCC9CFF1FA5
:100E10002E89FF1F189DFF1F209BFF1F6C9DFF1F2A
:100E2000509DFF1F28460EF0F9FBB2490EF04AFC18
:100E3000054650460EF0F2FBAF490EF043FC01466A
:100E400028460EF037FB0EF003FE0546CBF80050A7
:100E5000D9F800000EF0E2FBA6490EF033FC07467D
:100E600030460EF0DBFBA4490EF02CFC0146384660
:100E70000EF020FB0EF0ECFDC9F800009F4AA04BDD
:100E8000168819889F4AA04B12681B889F4FC6EB93
:100E9000050E3544039EC6F800E0461A084404993E
:100EA0000D6001990E6002993E8808609A4280F2B6
:100EB00089810025C3EB060E954974450F6880F2C1
:100EC0007681611C9F4205FB01F50EF1010E95FB39
:100ED000FEF5C0F2BE81BE42A8BF3E46F61A01FB37
:100EE00006F494FBFEF49A4200F33681BB42C0F252
:100EF0003381884C20680EF091FB87490EF0E2FBAD
:100F000086490EF0D7FA0EF0A3FDA0F5FF531C3B67
:100F1000082B98BF4FF40050D8F800301844002830
:100F20002060C0F24281B0F5804F80F252817C4B4C
:100F30001B781BB1B0F5005F40F05381794D2B78E1
:100F4000002B40F05481784D20682B68714C9842FA
:100F500004D080B207F0DEFA23682B6009B0BDE848
:100F6000F08F28460EF05AFB70490EF0ABFB054699
:100F700050460EF053FB6E490EF0A4FB0146284686
:100F80000EF098FA0EF064FD0546CBF80050D9F843
:100F900000000EF043FB65490EF094FB0746304617
:100FA0000EF03CFB62495FE728460EF037FB5A49DA
:100FB0000EF088FB054650460EF030FB5D490EF002
:100FC00081FB014628460EF075FA0EF041FD0546FC
:100FD000CBF80050D9F800000EF020FB4E490EF07F
:100FE00071FB074630460EF019FB52493CE7284694
:100FF0000EF014FB50490EF065FB054650460EF00E
:101000000DFB4E490EF05EFB014628460EF052FAEB
:101010000EF01EFD0546CBF80050D9F800000EF08A
:10102000FDFA45490EF04EFB074630460EF0F6FA43
:10103000424919E7D8F80030DFF810B103EBD37359
:101040005B10DBF80050C8F800301FE6DFF80081C5
:10105000DFF80091D8F8003003EBD3735B10C8F8C9
:101060000030BDE5364A06931188364A0591204680
:101070000492DFF8D8B00EF0D1FA049A0599DBF8A3
:10108000005052F821100EF01DFB0EF0E1FCEF1B9A
:10109000069B5745A7EB0302B8BF5746FF1AD8F87F
:1010A00000309042BABF013200FB0777474397FBFD
:1010B000F2F73B4403EBD373234A04925B10C8F866
:1010C0000030E3E50EF0AAFA029A52F82B100EF067
:1010D000F9FA0EF0BDFCCAEB0802B045B8BFB04645
:1010E0008242CAEB08083FF76AAD00FB08F898FB9C
:1010F000F2F069E5CDCC4C3FCDCC4C3EA289FF1F30
:101100002C89FF1F8C9BFF1F2A9DFF1F729BFF1FB7
:10111000A89DFF1F8C89FF1F9A99193FCDCC4C4584
:101120005E9EFF1FD59BFF1F2089FF1F3333733F38
:10113000CDCC4C3DCDCCCC3E6666663FCDCCCC3DD7
:101140005C9BFF1F24120100CC9CFF1F509DFF1FC2
:101150006C9DFF1F209BFF1F009B1B88002B3FF4F3
:10116000C8AE2B1B002BB8BF5B42092B47DD05F532
:1011700000500130001B0EF051FA3B493B4C0EF081
:10118000A1FA054620680EF049FA39490EF09AFA9C
:10119000014628460EF08EF90EF05AFCD8F80030C1
:1011A000184400282060BFF6BEAE002213E09F4224
:1011B00005FB04F5B8BF002195FBFEF54BDA91FB6A
:1011C000FEF490E6B242D4BFC3EB0205C3EB0605C2
:1011D00070E643F6FF72274B22601B78002B3FF42A
:1011E000ADAE04F097FB244B01221A70ABE604F07D
:1011F0008DFB00232B70A6E6D9F800003EE64FF4E5
:1012000000501A4C88E61D491D4A069320460D8859
:1012100005920EF003FA059ADFF868B052F825102F
:10122000DBF800500EF04EFA014600200EF040F9B7
:101230000EF00EFC2F44069B56E50EF0EFF9039AD4
:1012400052F82B100EF03EFA014600200EF030F955
:101250008AE51E4642E6B742D4BFC3EB0701C3EBA3
:10126000060104FB01F1AAE7CDCCCC3E8C89FF1F1F
:101270009A99193F5E9EFF1FD59BFF1F5C9BFF1F26
:1012800024120100509DFF1F08B5244B1B88FBB1A1
:10129000234B1B78FBB1234B1B78E3B1224B1B780C
:1012A000CBB1224B1B78B3B1214B22481A78C2B97B
:1012B000214A22490088128809680244B1EB620F72
:1012C00009DD01221A706420BDE8084004F036BB35
:1012D000174A117801B908BD1370BDE8084007F03E
:1012E000E3B8154A16490088128809680244B1EB30
:1012F000620FF0DD00221A7007F0D6F8642004F0C7
:101300001DFB642004F01AFB642004F017FB4FF46B
:101310001670BDE808400BF0D3BB00BFD69CFF1F82
:10132000B39DFF1F869DFF1F879DFF1F889DFF1F89
:101330005E9BFF1F729BFF1F2A9DFF1F8C9BFF1F41
:10134000A89DFF1F38B5114C232025780AF066FEB2
:101350000F4A42F82500131F02F1C400002253F87F
:10136000041F83420A44FAD123780A4907480A4CE9
:101370000133DBB2322B81FB025108BF0023D217AD
:10138000C2EB21120370226038BD00BF4A9BFF1FD1
:10139000F09BFF1F1F85EB514C9DFF1F2DE9F04F68
:1013A000B84CB94D2068B94F83B00EF037F9B84941
:1013B0000EF088F9064610200BF074FD0EF02EF9A1
:1013C000B4490EF07FF931460EF074F80EF040FB90
:1013D0002988206088423B8843DA9E465B1A7F2B2F
:1013E0004FF0000247DDD2015E1C92FBF6F2AA4EDE
:1013F000DFF8C882B6F800C0C8F80020BCF1190FA9
:1014000000F0DF80BCF11A0F00F01781BCF11E0F55
:1014100000F020810126B146A04A1288002A00F07F
:101420009D808842C0F207817045D4BFC1EB0000A7
:10143000C1EB0E009A42BABF02FB000001335043D9
:1014400090FBF3F3964A1360964B1888C0B9964AFE
:101450001288AAB9954B197801B11A7003B0BDE88A
:10146000F08F9842D4BFC1EB0002C1EB03029E464D
:101470005B1A7F2BB7DCC2EBC21292FBF3F2B6E72A
:101480002988D4F800E0DFF80082DFF8F8A1714580
:101490006CDCDFF818C29CF80020002A2ED14FF037
:1014A000010B04288CF800B028D1002E40F0948164
:1014B0007D4B18880028D1D0B9F1000FCED0236819
:1014C0002C883A88A34280F265810023141B7E2C6D
:1014D000774DD5BFC3EB8313C3EBC3135B0001345C
:1014E00093FBF4F42B680134A34203D0C0B2E1B201
:1014F00006F032FF2C6003B0BDE8F08F012800F049
:10150000F680022800F0EB800328D1D1694B1B88BC
:10151000092BCDD0002ECBD023682E883A88B34239
:1015200080F27B810023961B7E2EDFF88CA1D5BF35
:10153000C3EB8313C3EBC3135B00013693FBF6F6D7
:10154000DAF800300136B34203D0F1B24A2006F097
:1015500003FFCAF80060ABE716469146BCF11E0FC8
:101560007FF472AF0022DFF858817EE04F4B1A788B
:10157000002A3FF473AF002401281C7000F0A480FF
:10158000022840F00E81002E00F0A3804A4D2B6807
:10159000002B00F09E800420214606F0DDFE424B29
:1015A0002C60188800283FF459AFB9F1000F3FF4C0
:1015B00055AFC0B2002106F0CFFE3D4B00221A60AD
:1015C0004CE7DFF8FC8098F80020C2B1DFF8D89033
:1015D000B9F800A0BAF1000F11D0DFF8E89099F83F
:1015E00000B0934578D05FFA8AF07F2106F0B4FE10
:1015F00098F80030B6F800C089F8003010E0DFF845
:10160000C49099F800A0924566D0274B0021187825
:1016100006F0A2FE98F80030B6F800C089F8003055
:101620001E4B1A88002A97D0BCF11E0F40F006818D
:101630000026B14619E00020FCE6DFF8848098F827
:101640000020002A0BBF012600264FF000094FF0B2
:101650000109E1E6DFF86880104B98F800601A880D
:10166000B6FA86F676094FF0000998F80030002B9C
:101670003FF4E8AE2988B7F800E02068C1EB0E031C
:10168000CFE600BF849BFF1FDC9CFF1FD89CFF1F81
:101690009A99193FCDCCCC3E629DFF1F949DFF1FB0
:1016A000E89BFF1F8A9BFF1F729DFF1F699DFF1F05
:1016B000689BFF1F1A9DFF1FEC9BFF1F449DFF1F90
:1016C000189DFF1F4E9BFF1F1EB1614D2B68002B05
:1016D0007BD1604B188865E70026B1469CE6002E5A
:1016E0003FF4E6AEDFF868A1DAF800202EE0002E25
:1016F0003FF4DEAEB7F80080F045D4BFC1EB08027E
:10170000C1EB0E02C1EB0808B8F17E0FDFF840A173
:10171000D5BFC2EB8212C2EBC212520008F101081F
:1017200092FBF8F8DAF8002008F10108424506D0EB
:101730005FFA88F10120009306F00EFE009B1888E6
:10174000CAF8008002287FF4DFAE42462168B5F86F
:1017500000803888414559DA0021C8EB0008B8F10B
:101760007E0FD3BFC1EB8111C1EBC11108F101089C
:10177000490091FBF8F808F10108904506D05FFA9E
:1017800088F10420009306F0E7FD009B1888CAF852
:101790000080B9E69342D4BFC4EB0303C4EB020359
:1017A00094E6032827D12C4B1B88092B91D0002EBF
:1017B0008FD0274D2B68002B8BD04A20214606F076
:1017C000CBFD244B2C601888ECE6214606F0C4FDC6
:1017D000204B2C601888E5E640207F218DE80C0026
:1017E00006F0BAFD019B009A188858451CD00228C3
:1017F0007FF48AAE76E704287FF46BAF002E3FF4C7
:1018000068AF2146402006F0A7FD62E78142D4BFC1
:10181000C8EB0101C8EB00019FE79342D4BFC6EBC0
:101820000303C6EB02037EE6B8F80010DAF800E026
:10183000B7F800808E45FFF665AF5DE72988B7F8F9
:1018400000E020680026C1EB0E03B146E9E500BFC9
:10185000EC9BFF1F729DFF1F1A9DFF1F08B50F4BCA
:101860001B88022B0FD0032B12D0042B03D00C4B60
:1018700001221A7008BD7F21092006F06DFD084B7A
:1018800001221A7008BD7F21412006F065FDEEE7B8
:101890004021092006F060FDE9E700BFE49BFF1F3F
:1018A000A49BFF1F38B51C4B1B881D2B26D01B4B40
:1018B0001B88012B25D01A4A1A4B14881B681A4A18
:1018C000A342128818DB9342D4BFC4EB0303C4EBDA
:1018D0000203141B7F2CC6BFDB010134C3EBC3130F
:1018E00093FBF4F4114D2B689C4203D0E1B2052028
:1018F00006F032FD2C6038BD0023EAE70C4B1C8853
:10190000F0E70C4B0C4A0D491B6812680C689B1AD7
:101910001C1B84F30704E5E7629DFF1FD49CFF1F97
:10192000489DFF1F349BFF1F609DFF1F2C9BFF1FC7
:10193000809BFF1FA09DFF1F2889FF1FE09CFF1FAA
:1019400010B50F4C23685BB90E4B1B88022B11D0CE
:10195000033B012B09D90C4A00231370236010BDEF
:101960000021052006F0F8FCEEE70021092006F032
:10197000F3FCF0E70021412006F0EEFCEBE700BFAE
:101980002C9BFF1FE49BFF1FA49BFF1F08B5274B49
:101990001B78ABB115200AF041FB254A254B128874
:1019A00018601D2A15D0244A1288EAB1012A25D0D0
:1019B000224B1B78002B34D0BDE80840FFF7C0BF96
:1019C00011200BF06FFA1A4A1A4B128818601D2A60
:1019D000E9D11B4B1B78002BEAD0184B1B780BB3BB
:1019E000BDE80840FFF75EBF164A1288002ADFD024
:1019F000154A1B6812889A42DADCEEE70F200BF0DA
:101A000051FA104B114A1B88106033B1104B114A28
:101A10001B6812689B1A9842DFDD084B1B78002B6D
:101A2000CAD108BDFFF71AFFDAE700BF409DFF1FCC
:101A3000629DFF1F349BFF1FD49CFF1FA49BFF1FB1
:101A4000189DFF1FE49BFF1F489DFF1FE09CFF1F89
:101A5000A09DFF1F2889FF1F2DE9F04F8BB007AD18
:101A6000B54F2C460AAE611BC9B2B44808F014FB4E
:101A70003B88834294BF0020012004F8010BA6425A
:101A8000F1D1AF48AF4A9DF81C50AF4905709DF8A1
:101A90001E00AE4E10709DF820209DF82430AC4FF3
:101AA000AC4C0A709DF82210317000263B702670F5
:101AB00063B9002940F00581002A40F0C581A64A9B
:101AC000002800F0C9810223237005E0002A40F0BD
:101AD000A9800523A04A2370DFF8D4B2DFF8D4929E
:101AE0009DF81DE09DF81F00DFF8CC82DFF8CCA246
:101AF0009A4D9B4F9B4E9DF8211013708BF800E080
:101B00009DF826209DF823309DF825E089F80000F7
:101B10009DF827C088F8001001208AF800202B705B
:101B200087F800E086F800C00BF0BCF98E4A8F4BB6
:101B300011688842CCBF012200221A7076DD8C4BDE
:101B40001B88182B72D88B4AB2F800E00C3B00932C
:101B5000BEF1000F72D1884A9BF800C092F800B025
:101B600098F8008099F800209AF8009094F800A066
:101B70002C78ABEB4C0BC2EB0B0BA8EB880EDE44C6
:101B8000C9EB897BC9EB8B09DFF8F4B1F14497F815
:101B900000E0BBF800B009EB44093478CE4404FB04
:101BA0000BEE4FF00C09754C19FB0AEEC4F800E07F
:101BB000B8F1000F0BD036784EB1714E3688042E36
:101BC0000CBF0EF1020E0EF1040EC4F800E06D4CD5
:101BD000DFF8EC912488B9F800A06B4EDFF8E491AF
:101BE0003688D9F80090009B033C04EB4404CAEB10
:101BF000CA0A0EEB84043444D144644E0C3C56F8BB
:101C000029601C44A319BCF1000F28D02C7834B3F0
:101C1000002A5AD1B8FA88F85D4C4FEA581884F86F
:101C2000008023E0062323704B4A55E7514AB2F85F
:101C300000E000230093BEF1000F8CD0BEF1010F35
:101C400047D0BEF1020F00F0C1804C4C9BF800C0A1
:101C500099F8002098F80080D4F800E0A8E74C4CF0
:101C6000002525700AB13A781ABB0022494C8842F7
:101C700022704949C4BF494AC2F800E00A68934249
:101C800013D0474A474C10680590059820601268A9
:101C90000692454C069A24880B60121AA24284BF11
:101CA000424A13600BB0BDE8F08F3E483C4A0068E2
:101CB000EDE7BCF1000FD8D1B8F1000FD5D101226A
:101CC000D4E704232370244A06E7314A0024147021
:101CD000CBE7294A9BF800C092F800E098F8008012
:101CE00099F8002094F800B09AF800902C780194AC
:101CF000AEEB4C0EC2EB0E0EA8EB88047444C9EB9D
:101D0000C909D944A31EDFF878A0DFF8BCE0019C24
:101D100097F800B05EF829E0BAF800A096F80090B5
:101D200003EB44045C4409FB0A4909F11809134C0C
:101D3000CE44C4F800E03BE7849DFF1FD49BFF1F07
:101D4000869DFF1F879DFF1F889DFF1F899DFF1F89
:101D50008A9DFF1FD19CFF1FDA9CFF1FB49DFF1FB0
:101D6000B59DFF1F689DFF1F9089FF1F189DFF1FD6
:101D7000629DFF1F309BFF1FA489FF1F209DFF1F37
:101D8000929BFF1F349DFF1F4C9BFF1F540E0100B1
:101D90009C9DFF1F9D9DFF1F9C9BFF1F7C9BFF1F0A
:101DA0009C9EFF1FC09BFF1F709DFF1FA49DFF1FD8
:101DB000B09DFF1FB19DFF1FB29DFF1FB39DFF1F71
:101DC000589DFF1FE89BFF1FD4110100274A9BF875
:101DD00000C092F800B0247899F8002098F80080AC
:101DE0000394ABEB4C049AF80090214B95F800A0BB
:101DF000CDF804A0A8EB880BA41A5C444FF0050BA7
:101E00001BFB094B039C97F800A0CDF808A0C9EB79
:101E1000C909B3F800A009EB0403BDF80490029CC3
:101E20000BF1050B1EFB09BE96F800B0DFF84C90D5
:101E3000A6440BFB0AEE59F823900E4C0EF10C0E43
:101E4000CE44C4F800E0B3E60B4A1378002B3FF40D
:101E500037AE032323703FE615B1012323703BE621
:101E60001378012B8CBF23702B4635E6A489FF1F06
:101E7000929BFF1F209DFF1FDA9CFF1FFC13010098
:101E80002DE9F04F3B4B1B788BB0002B6DD10E2012
:101E90000AF0C4F80DF0C2FB01463748374E384D02
:101EA000FEF748FB3448FEF71BFB0DF0D1FD80F335
:101EB0000C003060FFF7D0FD2C68012C7CD0022C88
:101EC00000F0AA82032C00F0B9832E4E33682E4A0C
:101ED0002E4E0993099B177830682D4C072101225B
:101EE000181A11FB07229042236000F29082294EBB
:101EF00032689A1A0D2A00F28382274E32689A1AA3
:101F0000132A00F27882254E32689A1A252A1AD9A5
:101F1000234B1B88002B40F06781224B1B78002B42
:101F200040F06281FFF70EFA1F4B1B881B3B9BB2F0
:101F3000022B04D81D4B1B78002B40F0588103F076
:101F40000FFD236833601A4D2A689B1A502B00F24C
:101F50001182184B1B88012B00F0298206F090FAA1
:101F600006F0BEF80BB0BDE8F08F07F0BFFA0BB07B
:101F7000BDE8F08F649BFF1FF89CFF1F2C9DFF1F87
:101F80005C9DFF1F9C9EFF1FCB9CFF1FDC9BFF1FC8
:101F9000F49CFF1FCC9BFF1FAC9BFF1FB09BFF1F40
:101FA000D69CFF1F5E9BFF1F629DFF1F189DFF1F9A
:101FB000E89CFF1F309DFF1FDFF82893A34AB9F864
:101FC00000001378834204D0C3B21846137006F0A1
:101FD00093F9DFF80C839E4AB8F8003011789942E3
:101FE00004D09C4F3978002940F0D3869A4A336850
:101FF00012889A4E9A42C0F2FF80994A1278002ABB
:1020000040F0FA80DFF8E0A2BAF8003023B9954B2F
:102010001B88002B00F00685934A944B11881B887F
:10202000934A0B4412685B109342924A126880F202
:102030007B8400219342B4BF01230B46049100939B
:10204000ACBF4FF0010B8B4605910E2009F0E6FF67
:10205000894B8A4A1B68176803930133A7F25232EF
:10206000002B8446029240F3A586802BA8BF8023D4
:10207000834A844912780191002A00F0C7800978C8
:10208000914200F0C380B8F80010DFF854E29942A2
:1020900001F078806F49AEF800307B4B4FF0010EB5
:1020A00081F800E01978DFF844E2019B8EF8001017
:1020B0001A70009B002B00F01B81BAF80030002B37
:1020C00000F01681714B1B685A1C002A40F376867B
:1020D000802A00F372866E4C6E496F482488098806
:1020E00000682144B0EB610FC1F2B982A3F148024C
:1020F0000F2A02D8473BA9F800300E2009F08EFFC6
:102100006FF454731F44874202DC644B00221A7040
:1021100000200AF0C7FE624A624B1168624C1B88BD
:102120008842D4BF002201222270002B00F0F383EA
:102130005E4B1C78944240D088423EDD5C490C786E
:10214000002C00F0ED865B4991F800C0BCF1000F57
:1021500040F0E486584F0097584F59480297564F21
:10216000007887F800C0554F4FF0010E87F800C087
:1021700081F800E0002841F07B805249097800296D
:1021800000F0A987504903910C460978002940F0D6
:102190009F874E48494F007839700121029721707E
:1021A00058B1454843490090002008700099029FAB
:1021B0000870039901243C7008701A70444B1B8806
:1021C000A3F11B02012A40F2BF851D2B7FF47EAED6
:1021D0003E4F3B78002B41F012803E4C2378002B81
:1021E00040F05084237071E6FFF74EF89AE62B68B2
:1021F000012B7FF4A4AEA4E63168374A0691069815
:102200003649106002220B602A60FBE61E49DFF8A7
:10221000DCE0097800293FF448AF9EF800008142D5
:102220003FF443AF03984B2840F373871833802B58
:10223000B8F80000A8BF802398423FF436AF284882
:1022400003800448012303702FE700BFCA9CFF1FCF
:10225000B49BFF1F529BFF1FE09BFF1F9C9EFF1F15
:102260005E9BFF1FD29BFF1F729BFF1F2A9DFF1FBC
:102270008C9BFF1FA89DFF1F7C9BFF1F389BFF1F90
:102280009C9DFF1F989BFF1F9D9DFF1F209DFF1F73
:10229000DC9CFF1FD89CFF1F849BFF1FD09CFF1F4F
:1022A0009089FF1FE69CFF1F789BFF1F249BFF1F49
:1022B000B39DFF1F289DFF1F749DFF1FE29BFF1F03
:1022C000B49DFF1FB09DFF1F259BFF1F189DFF1F83
:1022D000629DFF1F4E9BFF1FA89BFF1FF09CFF1FCF
:1022E000649DFF1FE49CFF1FA09BFF1F999BFF1F86
:1022F000029B9C45BFF601AFAC4B1B88002B3FF403
:10230000FCAEBBF1000F7FF4DDAEA94B1B881BB107
:10231000059B002B7FF4D6AE049B002B3FF4EDAE63
:10232000A44B1A78002A7FF4E8AEDFF8049399F8FA
:10233000004001221A70002C40F041839E4B1B7814
:10234000002B01F0F6879D4B1B78002B02F0D48206
:102350009B4B1B78002B7FF4D0AE9A4B1B78002B45
:102360003FF4CBAEB8F8003097490A3BA8F80030EC
:102370000A70C2E604F0C4FD944B1B7873B9944B09
:102380001B785BB9934B1B7843B9934B1B782BB9E4
:10239000924B1B7813B903F0B9FA01E003F0C2FACB
:1023A00023682B608E4B1B88012B7FF4D7AD8D4AA1
:1023B0008D4B11688D481A78A1F118032A2101FB71
:1023C00003F10160002A00F09082894A1368994263
:1023D00000F32C8380F2368386480068D0F17F00BA
:1023E00048BF0330801001301B1A994200F32A8342
:1023F000136019467BE2FFF7C9FA2368336082E570
:10240000FEF77AFBFEF7CAFF2368336075E5FEF737
:10241000EBFA236833606AE5774A34681288A2428F
:1024200004DB6E4B1B78002B00F02783734E74483F
:1024300033680793734B079900681B88091A994200
:1024400063D8002B61D0704B198800293FF43EAD52
:102450006E4B6F481B680088A342B8BF23469A4260
:1024600041F3F3806B4B1A60DFF8C88188F80010E5
:102470005C4FFEF7B9FA38687F2840F34B85664B0E
:102480007F3883FB0032C317C3EB620303EB4303C4
:10249000A0EB83007330614B01931B883860002BE5
:1024A00040F05E864B4B00931B78002B00F0998325
:1024B0005B4C2378002B00F09483DFF87C91DFF8ED
:1024C00058A14FF0000B0CE003F17300C0B298F874
:1024D000001005F069FF23780BF1010B5B4540F319
:1024E00080833B6859F8040F1844A0F17F038AFBEE
:1024F0000321DA17C2EB610202EB42027F28A3EB51
:102500008203E1DCFEF7A8F8E0E7404B40491B6896
:1025100008883D49A342B8BF23469A4200F39482FB
:102520003C4C09888342A8BF0346236000299BD105
:102530009A42C8BF0B4640F38E82801AB0F5804F96
:10254000AABF9B03C3EB8333013093FBF0F0FEF78C
:1025500031FAC0F3C6100DF061F8324B044618880A
:102560000DF05CF83049074620460DF0ABF8014607
:1025700038460DF0A7F821460CF09CFF4FF07E5135
:1025800004460DF03DFA002841F0548027492046CA
:102590000DF054FA002840F0658620460DF07EFAD2
:1025A000C0B2DFF8908088F8000061E7D29BFF1F7F
:1025B000EC9CFF1FD09CFF1FB09DFF1FB19DFF1F14
:1025C000B29DFF1FB39DFF1F529BFF1FE29BFF1F8A
:1025D000289DFF1F749DFF1F259BFF1F5E9BFF1FF4
:1025E000309DFF1FA49DFF1FA49BFF1F909DFF1FF9
:1025F000589BFF1F2C9BFF1FE09BFF1F9C9EFF1FF4
:10260000A89BFF1FD09BFF1F509BFF1FF09CFF1F2D
:102610008C9DFF1F289BFF1FABAAAA2A889BFF1F28
:102620005489FF1F9E9DFF1FCDCCCC3D0000FE4274
:10263000D19CFF1FC69BFF1F2C89FF1FC14B346815
:102640001988A14253DDC04B1B78002B4FD1DFF816
:10265000449399F800007F2840F3CD85A3F15533CA
:102660007F3803F1004383FB0032C317C3EB6203DF
:1026700003EB4303A0EB83007330B44B01931B883F
:10268000C0B289F80000002B40F0BF87B04B009328
:102690001B78002B00F07184AE4C2378002B00F0E7
:1026A0006C84AD4FDFF8B8824FF0000A0AE003F106
:1026B0007300C0B205F0A0FE23780AF1010A534569
:1026C00040F35B8457F8043F99F800001844A0F1E8
:1026D0007F0388FB0321DA17C2EB610202EB42029F
:1026E0007F28A3EB8203E2DCFDF7B6FFE1E79B4F17
:1026F00038687F2840F3B681994B7F3883FB0032DE
:10270000C317C3EB620303EB4303A0EB83007330F7
:10271000DFF8809299F800A0824500F00982914B81
:102720001B88002B43D1904A904812680088914240
:1027300005DC8242D4BFC1EB0203C1EB0003411AA6
:10274000B1F5804FA6BF9B030131C3EB833393FBED
:10275000F1F0FEF72FF9C0F3C6100CF05FFF844BC9
:10276000044618880CF05AFF8249804620460CF037
:10277000A9FF014640460CF0A5FF21460CF09AFE49
:102780004FF07E5104460DF03BF9002840F0AD8635
:10279000794920460DF052F9002840F06085204626
:1027A0000DF07CF9C0B2DFF8F08188F80000BAF1D2
:1027B0007F0F40F3AB836A48AAF17F0A80FB0A309F
:1027C0004FEAEA73C3EB600000EB4000AAEB800025
:1027D00073305F4B00931B78C0B289F80000002B68
:1027E00040F00B83654B03931B78002B40F0F7847C
:1027F000634B02931B78002B40F01F87534B0193D0
:10280000029B1B78FBB15F4B1B88012B00F0EB8513
:10281000022B00F04187032B01F0D280042B01F042
:10282000F482052B01F07083062B01F04285072B03
:1028300001F05986082B02F00D80092B02F0D88098
:102840000A2B02F01283009B1B78002B00F05384AC
:10285000019B3E4C1988002900F0A98438687F2824
:1028600040F3C8823E4B7F3883FB0032C317C3EB73
:10287000620303EB4303A0EB83007330386000294D
:1028800040F05884009B1B78002B00F05C81314C99
:102890002378002B00F05781DFF8BCA0DFF8F88028
:1028A0004FF0000B0CE003F17300C0B298F8001079
:1028B00005F07AFD23780BF1010B5B4540F3438172
:1028C0003B685AF8040F264A1844A0F17F0382FBA4
:1028D0000321DA17C2EB610202EB42027F28A3EB6D
:1028E0008203E0DCFDF7B8FEDFE7274B1960274BDA
:1028F0001B68A92202FB03F3002BBCBF03F57F5327
:102900003F339B13543B194481F30C01282009F0F9
:102910000BFFFFF723BB1A4C1D480D49174A2370C4
:1029200003700B70137049E493424FF0000B80F278
:102930009C800123CDF800B0CDF814B00493FFF7CC
:1029400084BB00BFE09BFF1F5E9BFF1F889BFF1F98
:10295000749DFF1F5489FF1F2C89FF1FA49DFF1F1B
:10296000ABAAAA2A509BFF1F289BFF1F8C9DFF1F0D
:102970009E9DFF1FCDCCCC3D0000FE42259BFF1F3E
:10298000E29BFF1FE69CFF1F589BFF1F8C89FF1FC8
:10299000289DFF1F1C9DFF1FC69BFF1FA94B1B7877
:1029A000002B7FF4AAAB039BA74A243B83F3470386
:1029B000D9B25B20136005F0CFFC99F80040032CDE
:1029C00030D1DFF8D88298F80030002B42F08E81A9
:1029D0009E4F3B78002B42F07C819A4C2378002B51
:1029E00042F06A819A4B1B78002B42F03D81994A54
:1029F0001380994B1B78002B42F08481974B7F22E8
:102A00001A8098F800306BB93B785BB923784BB9E2
:102A1000934A7F210720138005F09EFC7F210B2025
:102A200005F09AFC8F4B1F68FFF767BB8E48006864
:102A3000D0F17F0048BF033003EBA003013399427C
:102A4000BFF6D6AC116052E7884B09881A6000299E
:102A50007FF40AAD13469842D4BFC2EB0003C2EB29
:102A600003036AE5FDF7F8FD52E60123CDF810B047
:102A7000CDF800B00593FFF7E8BA01232B607C4E38
:102A8000FFF724BA7B4B6A20198805F0E9FD3B78F3
:102A90002370FFF71BBA029B1B78FBB1764B1B8898
:102AA000012B00F01984022B00F07486032B00F038
:102AB000FD87042B01F08581052B01F09B82062BFD
:102AC00001F00C84072B01F0B985082B01F0768604
:102AD000092B01F0AE870A2B02F08C81019B1B8829
:102AE000002B00F03083009B1B783BB9039B1B78C5
:102AF00023B9029B1B78002B00F052875F4B1B7899
:102B0000002B00F044815E490B78082B00F23F81D6
:102B10005C483A6800685C4C0133DBB25F1E101AF7
:102B200044F827000B70594B3468198889F8002045
:102B30008C424F4E7FF7CAA93268554B0892089ACB
:102B40001A60FFF7C3B9039B1B78002BA3D03B6827
:102B5000A3F10C007F2840F331834E488B3B80FB70
:102B60000320DA17C2EB600000EB4000A3EB800308
:102B700003F17300DFF82881C0B298F8001005F067
:102B800013FC009B1B78002B85D03D4C2378002B39
:102B900081D0DFF810A14FF0000B0CE003F17300BF
:102BA000C0B298F8001005F0FFFB23780BF1010B81
:102BB0005B457FF770AF3B685AF8040F354A1844FD
:102BC000A0F18B0382FB0321DA17C2EB61020C3800
:102BD00002EB42027F28A3EB8203DFDCFDF73CFD22
:102BE000DEE7264B1B78002B40F0C1823B682A4A67
:102BF0001278002A7AD0A3F10C007F2840F3F882E3
:102C0000244A8B3B82FB0321DA17C2EB610202EB01
:102C10004202A3EB820303F17300C0B298F80010E4
:102C200005F0C2FB009B1B78002B5ED0144C237870
:102C3000002B5AD0DFF86C90DFF858A04FF0000B53
:102C40003EE000BFB39DFF1F809DFF1FB29DFF1F91
:102C5000B19DFF1FD69BFF1FB49DFF1F509BFF1F01
:102C60001A9DFF1F389BFF1F2C9BFF1F289BFF1FD8
:102C70009C9EFF1F809BFF1FE69CFF1F289DFF1F40
:102C80005489FF1F549BFF1F3089FF1FE09BFF1FCC
:102C9000449EFF1FABAAAA2A259BFF1FB09DFF1FC2
:102CA000C69BFF1F2C89FF1F03F17300C0B298F869
:102CB000001005F079FB23780BF1010B5B4514DD67
:102CC0003B6859F8040F1844A0F18B038AFB0321D9
:102CD000DA17C2EB61020C3802EB42027F28A3EB49
:102CE0008203E1DCFDF7B8FCE0E73B68B74A127805
:102CF000FAB1B74A1288012A00F0FA83022A00F0DA
:102D0000CA85032A00F05287042A01F0A380052A0D
:102D100001F0DD81062A01F0FC82072A01F03E83E2
:102D2000082A01F01B86092A01F0BA860A2A02F055
:102D30002A80019A1288002A00F00B82A5490322FA
:102D40000B702A60FFF7C2B8A34F3B78002B3FF40B
:102D500044AAA24C207802F053FEA14B1B78002B12
:102D600000F0658223887E2B00F261829D4A013348
:102D7000108899B22180002800F06982C9B2C0B2DF
:102D8000994C05F0E9FA3B782370FFF79FB83A6851
:102D9000C9E6DBB21846137005F0BCFA934B9449B0
:102DA0001A46944B184600230B703B701370037047
:102DB000FFF71CB90123FFF75BB980248E498F4BC5
:102DC0008F4A09881B8812680B44B2EB630FBFF669
:102DD00094A9814B1B78002B40F0DA81B8F80030C1
:102DE000884AA3423FF489A9874B148001221A70B4
:102DF000FFF783B9FDF730FC40E5844B01931B8856
:102E0000002B42F0E2807B4B0393704B0293804C8B
:102E100023786BB3DFF80882DFF8F8A14FF0000BDE
:102E200009E003F17300C0B205F0E6FA23780BF174
:102E3000010B5B451CDD58F8043F99F8000018446D
:102E4000A0F17F038AFB0321DA17C2EB610202EBD8
:102E500042027F28A3EB8203E3DCFDF7FDFBE2E700
:102E60005A4B029305F0C8FA009B1B78002BCED179
:102E7000039B1B78002B3FF4C3AC99F80030A3F1FF
:102E80000C007F2840F3A88162488B3B80FB032025
:102E9000DA17C2EB600000EB4000A3EB800303F104
:102EA0007300C0B205F0A8FA009B1B78002B00F05D
:102EB0008881574C2378002B01F01882DFF860815D
:102EC000DFF850A14FF0000B0AE003F17300C0B22D
:102ED00005F092FA23780BF1010B5B457FF790AC7C
:102EE00058F8043F99F800001844A0F18B038AFBBE
:102EF0000321DA17C2EB61020C3802EB42027F2891
:102F0000A3EB8203E1DCFDF7A7FBE0E75046FDF70A
:102F1000A3FB5EE4FDF7A0FBFFF7BDBA002008703D
:102F20003D49087840B1314900910978002900F005
:102F30009C81009F002139703849097800297FF46D
:102F400021A9002C40F0C780002840F0C480224C0A
:102F5000264F94F800E0274C03941C4C0294254C17
:102F600023492070194C0097087038702070BEF10A
:102F7000000F7FF419A9FFF720B91E4B1B78002B17
:102F800070D099F80030A3F10C007F2840F36A83D9
:102F9000204A8B3B82FB0321DA17C2EB610202EB72
:102FA0004202A3EB820303F17300C0B205F024FADE
:102FB000009B1B78002B55D0154C2378002B51D04B
:102FC000174FDFF850804FF0000A35E0E29BFF1FFB
:102FD000E69CFF1F1C9DFF1F189DFF1F809BFF1F6E
:102FE000B59DFF1FBC9BFF1F4E9BFF1F749DFF1FC6
:102FF000289DFF1F259BFF1FD89CFF1FDC9CFF1FE8
:10300000849BFF1F649DFF1F529BFF1F889BFF1F18
:103010005489FF1FABAAAA2AB49DFF1FB09DFF1FB2
:103020002C89FF1F03F17300C0B205F0E5F9237886
:103030000AF1010A534515DD57F8043F99F80000DD
:103040001844A0F18B0388FB0321DA17C2EB61025D
:103050000C3802EB42027F28A3EB8203E2DCFDF78F
:10306000FBFAE1E7894B1B78FBB1894B1B88012BED
:1030700000F02086022B00F01A87032B01F09480C9
:10308000042B01F04D81052B01F07D83062B01F00F
:103090001584072B01F04E85082B01F04386092B80
:1030A00001F03C870A2B01F01987019B1B88002B3C
:1030B00000F0A682774B1B78002B40F09C82764B69
:1030C000764A198834680020012310602B602FE5B0
:1030D0000398002101707249097800293FF46DA816
:1030E0006A4902910978002900F0078702980021B7
:1030F0000170FFF762B8039B1B78002B7FF4A8AB2D
:10310000029B1B78002B7FF4A3AB019B1988FFF770
:10311000A5BB243B002BB8F8000040F33B84984249
:103120003EF4C3AF9BB25F48A8F8003001230370A0
:10313000FEF7BBBFDFF87081C0B298F8001005F051
:1031400033F9FFF79FBB584B3878197805F02CF905
:10315000C9E4D8B298F8001005F026F93B68EDE50F
:10316000C0B298F8001005F01FF9FFF79BB97F2156
:10317000402005F0F1F84D494D4A3B680B600021B5
:10318000117034E54B4BDFF84CE11978FEF78DBF39
:103190004B2C40F33E821834802CB8F80030464A5D
:1031A000A8BF8024A3427FF41FAEFEF7A6BF99F804
:1031B000000005F021F92188FFF750BBFDF74CFA1C
:1031C000D8E4029B1B78002B7FF41DAB039B1B787C
:1031D000002B7FF43DAB98E7FDF73EFA61E6374BF5
:1031E00001931B88002B7FF43BAE284B029344E6EF
:1031F000FDF732FA11E5FDF72FFAFFF73EBA304C32
:10320000207802F0FDFB2F4B1B781BB123887E2B0F
:1032100041F230802C4B1B7823B12388284A002BA5
:1032200041F05080294C3B782370FEF74FBE264B6F
:103230001B78002BF6D02388214A002BF2D024499A
:10324000013B088899B2118000287FF497ADC8B27D
:103250001E4C05F0F5F83B782370FEF737BE7F2053
:10326000FFF7A1BA7F20FFF79CB9084F09490297E1
:103270004FF0000C81F800C0009F02994FF0010E42
:1032800087F800E081F800C056E600BFE29BFF1F10
:10329000E69CFF1F289DFF1FE09BFF1F289BFF1F31
:1032A000189DFF1F529BFF1FC69BFF1F549BFF1FB4
:1032B0005489FF1F9D9DFF1F649DFF1F889BFF1F5B
:1032C000809BFF1FB59DFF1FB49DFF1F4E9BFF1FDF
:1032D000BC9BFF1F999BFF1FDFF8B0A33868BAF8AB
:1032E0000030E54AE54CC31A82FB031ED917C1EB37
:1032F0006E0101EB4101A3EB810303EB430354F89F
:10330000233018447F2840F34A847F3882FB003200
:10331000C317C3EB620303EB4303A0EB83007330DB
:10332000DFF86C83DFF86CB398F80010C0B205F0DA
:103330003BF8BBF80030022B7FF6D0AB3968BAF807
:103340000030CD4ACB1A82FB030ED817C0EB6E00BB
:1033500000EB4000A3EB800303EB430304EB830388
:10336000586808447F2840F3AA867F3882FB0032E1
:10337000C317C3EB620202EB4202A0EB8200733080
:10338000C0B298F8001005F00FF8BBF80030032B1E
:103390007FF6A4AB3968BAF80030B74ACB1A82FB83
:1033A000030ED817C0EB6E0000EB4000A3EB8003C8
:1033B00003EB430304EB8304A06808447F2840F335
:1033C00057817F3882FB0032C317C3EB620202EBE6
:1033D0004202A0EB8200733098F80010C0B204F0F3
:1033E000E3FFFFF77BBBDFF8A4A299F80000BAF86F
:1033F0000030A14AA14CC31A82FB031ED917C1EBAE
:103400006E0101EB4101A3EB810303EB430354F88D
:10341000233018447F2840F3C6837F3882FB003274
:10342000C317C3EB620303EB4303A0EB83007330CA
:10343000DFF860B2C0B204F0DFFFBBF80030022B4F
:103440007FF601AA99F80010BAF800308A4ACB1A20
:1034500082FB030ED817C0EB6E0000EB4000A3EB1D
:10346000800303EB430304EB8303586808447F287D
:1034700040F329867F3882FB0032C317C3EB620218
:1034800002EB4202A0EB82007330C0B204F0B4FF42
:10349000BBF80030032B7FF6D6A999F80010BAF8D4
:1034A0000030754ACB1A82FB030ED817C0EB6E00B2
:1034B00000EB4000A3EB800303EB430304EB830426
:1034C000A06808447F2840F3C7807F3882FB003221
:1034D000C317C3EB620202EB4202A0EB820073301F
:1034E000C0B204F089FFFFF7AEB90120FFF75BB966
:1034F000DFF898A16049BAF80020604C9A1A81FB65
:10350000020ED017C0EB6E0000EB4000A2EB800271
:1035100002EB420254F8220018447F2840F3BD8396
:10352000A0F17F0381FB0321DA17C2EB610000EBFE
:103530004000A3EB80007330DFF858B198F800101A
:10354000C0B204F031FFBBF80030022B50D939680B
:10355000BAF80030484ACB1A82FB030ED817C0EBEA
:103560006E0000EB4000A3EB800303EB430304EB8E
:103570008303586808447F2840F312867F3882FB13
:103580000032C317C3EB620202EB4202A0EB8200DF
:103590007330C0B298F8001004F006FFBBF800309A
:1035A000032B25D93868BAF80030334AC31A82FB96
:1035B000031ED917C1EB6E0101EB4101A3EB81039F
:1035C00003EB430304EB8304A36818447F284CDD1A
:1035D0007F3882FB0032C317C3EB620202EB420268
:1035E000A0EB82007330C0B298F8001004F0DCFE4B
:1035F0003B68FFF79EBB0021402004F0ADFE5EE576
:1036000099F8000004F0F8FE54E504F0F5FEFFF729
:103610003DB8243C002CB8F8003040F3BB85A342F1
:103620003EF46BADA4B2164BA8F8004001221A700C
:10363000FEF763BD0120FEF7B4BF124B01931B8858
:10364000002B7FF40FACFFF7DBB80F4A8342A8BF13
:1036500003461360FEF708BFFCF7FEFF40E7144681
:10366000FFF7B7BBFCF7F8FF9FE4FCF7F5FFBAE7FD
:10367000FCF7F2FFB0E600BFABAAAA2A700F010068
:10368000529BFF1F889BFF1F289BFF1F249DFF1F2E
:10369000C69BFF1F629BFF1FDFF818A399F800006D
:1036A000BAF80030C14AC24CC31A82FB031ED917B4
:1036B000C1EB6E0101EB4101A3EB810303EB43037B
:1036C00054F8233018447F2840F3E8837F3882FB86
:1036D0000032C317C3EB620303EB4303A0EB830089
:1036E0007330DFF8D4B2C0B204F086FEBBF800300D
:1036F000022B7FF6A8A899F80010BAF80030AB4A60
:10370000CB1A82FB030ED817C0EB6E0000EB400013
:10371000A3EB800303EB430304EB830358680844E3
:103720007F2840F3F2857F3882FB0032C317C3EB5A
:10373000620303EB4303A0EB83007330C0B204F0D9
:103740005BFEBBF80030032B7FF67DA899F80010D4
:10375000BAF80030954ACB1A82FB030ED817C0EB9B
:103760006E0000EB4000A3EB800303EB430304EB8C
:103770008304A06808447F287FF76EAF7F3882FB00
:103780000032C317C3EB620303EB4303A0EB8300D8
:103790007330A5E6DFF81CA23868BAF80030834A17
:1037A000834CC31A82FB031ED917C1EB6E0101EBD8
:1037B0004101A3EB810303EB430354F82330184486
:1037C0007F2840F36E837F3882FB0032C317C3EB40
:1037D000620303EB4303A0EB83007330DFF8DC816B
:1037E000DFF8D4B198F80010C0B204F0DDFDBBF8EA
:1037F0000030022B7FF672A93968BAF800306B4AA4
:10380000CB1A82FB030ED817C0EB6E0000EB400012
:10381000A3EB800303EB430304EB830358680844E2
:103820007F2840F36A857F3882FB0032C317C3EBE1
:10383000620303EB4303A0EB83007330C0B298F83C
:10384000001004F0B1FDBBF80030032B7FF646A951
:103850003868BAF80030554AC31A82FB031ED917DC
:10386000C1EB6E0101EB4101A3EB810303EB4303C9
:1038700004EB8304A36818447F287FF7F9AE7F38F0
:1038800082FB0032C317C3EB620303EB4303A0EBDD
:1038900083007330A0E5DFF81CA14449BAF800208A
:1038A000434C9A1A81FB020ED017C0EB6E0000EB5E
:1038B0004000A2EB800202EB420254F822001844BE
:1038C0007F2840F3F182A0F17F0381FB0321DA1707
:1038D000C2EB610000EB4000A3EB80007330DFF827
:1038E000D8B098F80010C0B204F05EFDBBF800300C
:1038F000022B7FF67DAE3968BAF800302B4ACB1A1E
:1039000082FB030ED817C0EB6E0000EB4000A3EB68
:10391000800303EB430304EB8303586808447F28C8
:1039200040F3EF847F3882FB0032C317C3EB62039E
:1039300003EB4303A0EB83007330C0B298F8001090
:1039400004F032FDBBF80030032B7FF651AE38682F
:10395000BAF80030154AC31A82FB031ED917C1EB0F
:103960006E0101EB4101A3EB810303EB430304EB85
:103970008304A36818447F287FF777AE7F3882FBE3
:103980000032C317C3EB620303EB4303A0EB8300D6
:10399000733028E601283EF488AB0123FFF7C3BB50
:1039A00099F8000004F028FDFFF7A8B8ABAAAA2AEE
:1039B0006C100100249DFF1F629BFF1FC69BFF1F11
:1039C000DFF8E4A299F80000BAF80030B44AB54C28
:1039D000C31A82FB031ED917C1EB6E0101EB410133
:1039E000A3EB810303EB430354F8233018447F28EF
:1039F00040F3DB817F3882FB0032C317C3EB6202E6
:103A000002EB4202A0EB82007330DFF8A0B2C0B23A
:103A100004F0F2FCBBF80030022B7EF614AF99F8EC
:103A20000000BAF800309E4AC31A82FB0321DA175D
:103A3000C2EB610202EB4202A3EB820303EB4303FE
:103A400004EB83035B6818447F2840F328847F38A5
:103A50000C2290FBF2F302FB13007330C0B204F0AF
:103A6000CBFCBBF80030032B7EF6EDAE99F80000DE
:103A7000BAF800308A4AC31A82FB0321DA17C2EB74
:103A8000610202EB4202A3EB820303EB430304EB6C
:103A90008304A36818447F287FF7DEAD7F380C22AB
:103AA00090FBF2F302FB1300733019E5DFF8F8A185
:103AB0003868BAF800307A4A7A4CC31A82FB031E7F
:103AC000D917C1EB6E0101EB4101A3EB810303EBBD
:103AD000430354F8233018447F2840F363817F3830
:103AE00082FB0032C317C3EB620202EB4202A0EB7F
:103AF00082007330DFF8B881DFF8B0B198F80010B9
:103B0000C0B204F051FCBBF80030022B7EF6E6AFE9
:103B10003868BAF80030624AC31A82FB0321DA1708
:103B2000C2EB610202EB4202A3EB820303EB43030D
:103B300004EB83035B6818447F2840F3A7837F3836
:103B40000C2290FBF2F302FB13007330C0B298F822
:103B5000001004F029FCBBF80030032B7EF6BEAF4A
:103B60003868BAF800304E4AC31A82FB0321DA17CC
:103B7000C2EB610202EB4202A3EB820303EB4303BD
:103B800004EB8304A36818447F287FF771AD7F3866
:103B90000C2290FBF2F302FB130073301CE4FCF7E1
:103BA0005BFDFFF7BDBBFCF757FD41E4DFF8F8A074
:103BB0003B49BAF800203B4C9A1A81FB020ED01701
:103BC000C0EB6E0000EB4000A2EB800202EB420271
:103BD00054F8220018447F2840F3EA80A0F17F03C4
:103BE00081FB0321DA17C2EB610101EB4101A3EB79
:103BF00081007330DFF8B4B098F80010C0B204F060
:103C0000D3FBBBF80030022B7FF6F2AC3868BAF871
:103C10000030234AC31A82FB0321DA17C2EB610288
:103C200002EB4202A3EB820303EB430304EB8303A7
:103C30005B6818447F2840F336837F380C2290FB62
:103C4000F2F302FB13007330C0B298F8001004F0D6
:103C5000ABFBBBF80030032B7FF6CAAC3868BAF870
:103C600000300F4AC31A82FB0321DA17C2EB61024C
:103C700002EB4202A3EB820303EB430304EB830456
:103C8000A36818447F287FF7F0AC7F380C2290FBA4
:103C9000F2F302FB13007330A5E4FCF7DDFC4BE408
:103CA000ABAAAA2AFC100100249DFF1F629BFF1FE4
:103CB000C69BFF1FDFF834A399F80000BAF8003064
:103CC000C24AC34CC31A82FB0317D917C1EB670161
:103CD00001EB4101A3EB810303EB430354F82330D1
:103CE00018447F286ADD7F3882FB0032C317C3EB9C
:103CF000620202EB4202A0EB82007330DFF8F0B206
:103D0000C0B204F079FBBBF80030022B7FF6CDA9DE
:103D100099F80000BAF80030AC4AC31A82FB0321BC
:103D2000DA17C2EB610202EB4202A3EB820303EB60
:103D3000430304EB83035B6818447F2840F3B68297
:103D40007F380C2290FBF2F302FB13007330C0B2F9
:103D500004F052FBBBF80030032B7FF6A6A999F8BC
:103D60000000BAF80030994AC31A82FB0321DA171F
:103D7000C2EB610202EB4202A3EB820303EB4303BB
:103D800004EB8304A36818447F2814DD7F380C22D9
:103D900090FBF2F302FB13007330C0B204F02CFB73
:103DA000FFF783B9FCF758FCA4E6FCF755FC2CE6BA
:103DB000FCF752FC1EE7FCF74FFCEEE7FCF74CFC6F
:103DC0009CE7DFF828A23868BAF800307F4A814CB7
:103DD000C31A82FB031ED917C1EB6E0101EB41012F
:103DE000A3EB810303EB430354F8233018447F28EB
:103DF000D8DD7F3882FB0032C317C3EB620303EBCD
:103E00004303A0EB8300733074E6DFF8E0A199F878
:103E10000000BAF800306D4A6E4CC31A82FB031ED4
:103E2000D917C1EB6E0101EB4101A3EB810303EB59
:103E3000430354F8233018447F28B6DD7F3882FBD3
:103E40000032C317C3EB620303EB4303A0EB830011
:103E50007330DAE5DFF894A15C49BAF800205D4CD4
:103E60009A1A81FB020ED017C0EB6E0000EB4000E7
:103E7000A2EB800202EB420254F8220018447F2891
:103E800096DDA0F17F0381FB0321DA17C2EB61000D
:103E900000EB4000A3EB80007330ABE6FCF7DCFBEB
:103EA0001FE4FCF7D9FB99E4FCF7D6FB17E5DFF834
:103EB0003CA199F80000BAF80030444A464CC31AB5
:103EC00082FB0317D917C1EB670101EB4101A3EB9B
:103ED000810303EB430354F8233018447F287FF712
:103EE0006DAF7F3882FB0032C317C3EB620303EB75
:103EF0004303A0EB8300733000E738480090384854
:103F000038490390FEF750B9DFF8E0A099F80000B7
:103F1000BAF800302D4A344CC31A82FB0321DA1759
:103F2000C2EB610202EB4202A3EB820303EB430309
:103F300054F8233018447F2840F3AE817F380C2298
:103F400090FBF2F302FB13007330DFF8A4B0C0B2B1
:103F500004F052FABBF80030022B19D999F800008E
:103F6000BAF800300C22C11A91FBF2F302FB1313D2
:103F700002FB03435B6818447F2840F367847F3863
:103F800090FBF2F302FB13007330C0B204F034FA7A
:103F9000BBF80030032B7EF656ACBAF8003099F827
:103FA00000000C22C11A91FBF2F302FB131302FB77
:103FB0000344A36818447F287FF74EAB7F3890FBFB
:103FC000F2F302FB13007330FFF78ABAABAAAA2AF6
:103FD000700F0100DC1201006C100100749DFF1FC6
:103FE000259BFF1F289DFF1F34140100249DFF1FE8
:103FF000629BFF1FDFF898A33868BAF80030DA4AEE
:10400000DA4CC31A82FB0321DA17C2EB610202EB1E
:104010004202A3EB820303EB430354F8233018441A
:104020007F2840F336817F380C2290FBF2F302FBAD
:1040300013007330DFF85C83DFF85CB398F800108E
:10404000C0B204F0B1F9BBF80030022B1AD93868BD
:10405000BAF800300C22C11A91FBF2F302FB1313E1
:1040600002FB03435B6818447F2840F3EC837F38EE
:1040700090FBF2F302FB13007330C0B298F800100B
:1040800004F092F9BBF80030032B7EF627ADBAF8A6
:10409000003038680C22C11A91FBF2F302FB1313B3
:1040A00002FB0344A36818447F287FF7E1AA7F3806
:1040B00090FBF2F302FB13007330FFF78DB9FCF7AE
:1040C000CBFAFFF75DB9FCF7C7FAFFF7DEB9DFF807
:1040D000C0A2A549BAF80020A44C9A1A81FB02108C
:1040E000D117C1EB600101EB4101A2EB810202EBB0
:1040F000420254F8220018447F2840F3B880A0F10F
:104100007F030C2093FBF0F200FB12307330DFF8DA
:1041100088B298F80010C0B204F046F9BBF800303D
:10412000022B1AD93868BAF800300C22C11A91FB58
:10413000F2F302FB131302FB03435B6818447F286E
:1041400040F3B9837F3890FBF2F302FB1300733026
:10415000C0B298F8001004F027F9BBF80030032B28
:104160007FF646AABAF8003038680C22C11A91FBD3
:10417000F2F302FB131302FB0344A36818447F28E5
:104180007FF773AA7F3890FBF2F302FB13007330C2
:10419000FFF729BA012B3DF4B0AF0124FFF743BA72
:1041A000FCF75AFAFFF7F5B9DFF8E4A199F8000037
:1041B000BAF800306C4A6E4CC31A82FB0321DA173E
:1041C000C2EB610202EB4202A3EB820303EB430367
:1041D00054F8233018447F2846DD7F380C2290FBAA
:1041E000F2F302FB13007330DFF8ACB1C0B204F09D
:1041F00003F9BBF80030022B19D999F80000BAF87E
:1042000000300C22C11A91FBF2F302FB131302FBE4
:1042100003435B6818447F2840F3A3807F3890FBFA
:10422000F2F302FB13007330C0B204F0E5F8BBF800
:104230000030032B7EF639AFBAF8003099F8000051
:104240000C22C11A91FBF2F302FB131302FB03448D
:10425000A36818447F287FF7AEAD7F3890FBF2F358
:1042600002FB1300733098E5FCF7F6F9BCE7FCF7A6
:10427000F3F94CE701339BB22380D9B205203D4CC2
:1042800004F06AF83B782370FDF720BEFCF7E4F9F0
:104290005CE4FCF7E1F9CDE6FCF7DEF955E6FCF766
:1042A000DBF9FFF7DBBBFCF7D7F9CDE4FCF7D4F97A
:1042B0004DE5DFF8DCA099F80000BAF800302A4A92
:1042C0002D4C29E6013B9BB2D9B20520294C138025
:1042D00004F042F83B782370FDF7F8BDDFF8B0A09A
:1042E0003868BAF80030204A234C8AE6029B1B78D3
:1042F000002B7EF488AAFEF7ABBAFCF7ADF9FFF706
:104300009DBAFCF7A9F9FFF718BBFCF7A5F9FFF771
:1043100015BADFF87CA01449BAF80020164CDCE688
:10432000DFF86CA099F80000BAF800300E4A134C80
:1043300042E7134B1B78002B00F0CB82114B1B780C
:10434000002B7DF4DAAE104B1B78002B3DF4D5AE7C
:10435000B8F800300D490A33A8F800300A70FDF7AC
:10436000CCBEFCF779F95FE7ABAAAA2A34140100A6
:10437000FC1001004E9BFF1F4C120100DC120100DB
:10438000B19DFF1FB29DFF1FB39DFF1F529BFF1FDB
:10439000249DFF1FC69BFF1F629BFF1FA14C22880D
:1043A000002A00F02283A049DFF88CB20988BBF80C
:1043B00000000331884227DD9C489D490088B1F800
:1043C00000E0DFF870C2181A0C2190FBF1F901FB34
:1043D00019004FF0900909FB0EFE01FB00E06FF0A1
:1043E0000B0E5CF8000003440EFB02307F2840F304
:1043F00038857F3890FBF1F301FB13007330C0B2B6
:1044000098F8001003F0D0FFBBF800202388134475
:10441000022B23DD854B864A38681B88B2F800C022
:10442000DFF810E2C31A0C2193FBF1F201FB123208
:10443000902303FB0CF301FB023373445B681844C5
:104440007F2840F3A2857F3890FBF1F301FB130036
:104450007330C0B298F8001003F0A6FFBBF800203C
:1044600023881344032B23DD704B714A38681B8863
:10447000B2F800C0DFF8BCE1C31A0C2193FBF1F2E3
:1044800001FB1232902303FB0CF301FB0233734454
:104490009B6818447F2840F37C857F3890FBF1F3BC
:1044A00001FB13007330C0B298F8001003F07CFFDA
:1044B000BBF8002023881344042B7FF799A85A4B9C
:1044C0001B88012B7FF494A83A68A2F10C007F2886
:1044D0007FF7CBA88B3A0C2092FBF0F300FB132064
:1044E0007330FFF780B84F4C2388002B40F01783C0
:1044F000DFF844B14D494E4A098899F80000B2F8F6
:1045000000E0DFF83081C1EB000C0C229CFBF2F1E3
:1045100002FB11C14FF0900C0CFB0EFE02FB01E1FF
:104520006FF00B0E58F8011008440EFB03007F28B3
:1045300040F3F583A0F17F0393FBF2F002FB103010
:104540007330C0B203F058FFBBF800202388134437
:10455000022B22DD354A364B118899F80000B3F85A
:1045600000C0DFF8D0E0411A0C2291FBF2F302FB0D
:104570001311902303FB0CF302FB013373445B68BC
:1045800018447F2840F392847F3890FBF2F302FBBB
:1045900013007330C0B203F02FFFBBF80020238854
:1045A0001344032B22DD214A214B118899F8000086
:1045B000B3F800C0DFF87CE0411A0C2291FBF2F363
:1045C00002FB1311902303FB0CF302FB0133734432
:1045D0009B6818447F2840F3C1847F3890FBF2F336
:1045E00002FB13007330C0B203F006FFBBF80020DB
:1045F00023881344042B7EF726A90B4B1B88012B21
:104600007EF421A999F80020A2F10C007F287FF701
:1046100023A88B3A0C2092FBF0F300FB132073309D
:10462000FEF75EBFC89BFF1FA29BFF1F249DFF1FBD
:10463000D29CFF1FE00B0100629BFF1FB84C238838
:10464000002B40F06182DFF810B3B649B64A098802
:10465000D7F80080B2F800E0B448C1EB080C0C2297
:104660009CFBF2F102FB11C14FF0900C0CFB0EFE13
:1046700002FB01E16FF00B0E405880440EFB0380FB
:104680007F2840F3B483A0F17F0393FBF2F002FB99
:1046900010307330A64BC0B2197803F085FEBBF81A
:1046A000002023881344022B23DD9E4A9E4B118851
:1046B0003868B3F800C0DFF874E2411A0C2291FBAD
:1046C000F2F302FB1311902303FB0CF302FB013303
:1046D00073445B6818447F2840F3FA837F3890FB6B
:1046E000F2F302FB13007330914BC0B2197803F060
:1046F0005BFEBBF8002023881344032B23DD894A8B
:10470000894B11883868B3F800C0DFF820E2411AFD
:104710000C2291FBF2F302FB1311902303FB0CF329
:1047200002FB013373449B6818447F2840F32084C4
:104730007F3890FBF2F302FB130073307C4BC0B266
:10474000197803F031FEBBF8002023881344042BB2
:104750007EF7C4A9774B1B88012B7EF4BFA93A686A
:10476000A2F10C007F2840F3B1808B3A0C2092FB21
:10477000F0F300FB132073306D4BC0B2197803F0D7
:1047800013FEFEF7ABB9DFF89CA199F80000BAF868
:104790000030694CC11A0C2291FBF2F302FB131397
:1047A00002FB03F3E35818447F287FF75DAD7F38A1
:1047B00090FBF2F302FB1300733015E55F4B1A8890
:1047C000182A13D03B681344A3F118007F2840F344
:1047D000C9830C20973B93FBF0F200FB123303F1EB
:1047E0007300534BC0B2197803F0DEFD544B5549AA
:1047F0001A78022A94BF013200221A701A7831F80E
:104800001200182810D10424022A02F10100C2B2B9
:1048100088BF002231F81200182804D1013CF3D1DE
:104820001A70FEF75BB91A703B680344A3F11800D5
:104830007F284BDD0C20973B93FBF0F200FB1233FB
:1048400003F1730098E7FBF707FF16E4FBF704FF9B
:10485000FFF79BBB394B1B88182B12D099F800200F
:104860001344A3F118007F2840F335830C20973BB5
:1048700093FBF0F200FB123303F17300C0B203F0BC
:10488000BBFD2F4A2F4B127833F81230182B3DF412
:10489000DAAF99F800201344A3F118007F287EF7BF
:1048A000DBAE0C20973B93FBF0F200FB123303F1DD
:1048B0007300FEF715BEFBF7CFFE49E4DFF864A0F6
:1048C00099F80000BAF800301F4C63E7FBF7C4FE0C
:1048D00052E71E4B1B78002B7EF460A81C4B1B7804
:1048E000002B3DF40AACB8F800301A490133A8F89F
:1048F00000300A70FDF701BC144B1B78002B7DF4CF
:10490000FCAB134B1B78002B3DF4F7ABB8F8003031
:104910001049013BA8F800300A70FDF7EEBB00BF5C
:10492000C89BFF1F249DFF1FD29CFF1FE00B0100AF
:10493000C69BFF1FA29BFF1F341401006E9BFF1F2D
:10494000C79BFF1F389DFF1F4C120100B29DFF1F28
:10495000B39DFF1F529BFF1F629BFF1FC94A128816
:10496000182A12D01344A3F118007F2840F30A83B9
:104970000C20973B93FBF0F200FB123303F1730022
:10498000C0B298F8001003F00FFDBF4BBF491A7872
:10499000022A94BF013200221A701A7831F81200EC
:1049A000182811D10424022A02F10100C2B288BFE2
:1049B000002231F81200182805D1013CF3D11A70F9
:1049C0003B68FEF7B6B91A703B680344A3F11800C0
:1049D0007F287EF74AAE0C20973B93FBF0F200FB5A
:1049E000123303F17300FEF7FEBDDFF8C8B2E3E453
:1049F000A74B1B88182B12D099F800201344A3F161
:104A000018007F2840F3B8820C20973B93FBF0F20C
:104A100000FB123303F17300C0B203F0EDFC9A4ABD
:104A20009C4B127833F81230182B7FF432AFFDF71D
:104A30000ABF974B1A88182A13D03B681344A3F176
:104A400018007F2840F39B820C20973B93FBF0F2E9
:104A500000FB123303F173008F4BC0B2197803F0DF
:104A6000A3FC894B8B491A78022A94BF0132002299
:104A70001A701A7831F8120018287FF4D5AE042481
:104A8000022A02F1010294BFD2B2002231F81200D0
:104A900018287FF4C8AE013CF2D11A70FEF71EB898
:104AA0007B4A1288182A12D01344A3F118007F28D9
:104AB00040F30B820C20973B93FBF0F200FB123388
:104AC00003F17300C0B298F8001003F06DFC6E4B58
:104AD00070491A78022A94BF013200221A701A789B
:104AE00031F8120018287FF46FAF0424022A02F173
:104AF000010294BFD2B2002231F8120018287FF4CC
:104B000062AF013CF2D15AE7644ADFF8A8B11288DB
:104B1000BBF80010033291427FF7C1AD95E55F4AC3
:104B2000DFF890B11288BBF80010033291427FF792
:104B30000BADDFE45A4C2388002B40F0BB81DFF83B
:104B400074B1584999F80000574A09881788DFF866
:104B50005CE1411A0C2291FBF2FC02FB1C114FF0AC
:104B6000900C0CFB07F702FB01716FF00B075EF86E
:104B70000110014407FB03107F2840F3F6817F38C2
:104B800090FBF2F302FB13007330C0B203F034FC6D
:104B9000BBF8002023881344022B21DD414B424AFD
:104BA00099F800001B88B2F800E0404FC31A0C21AE
:104BB00093FBF1F201FB1232902303FB0EF301FB96
:104BC00002333B445B6818447F2840F3E9817F3817
:104BD00090FBF1F301FB13007330C0B203F00CFC47
:104BE000BBF8002023881344032B21DD2D4B2E4AD4
:104BF00099F800001B88B2F800E02C4FC31A0C2172
:104C000093FBF1F201FB1232902303FB0EF301FB45
:104C100002333B449B6818447F2840F3D0817F389F
:104C200090FBF1F301FB13007330C0B203F0E4FB1F
:104C3000BBF8002023881344042B7EF736AA174BB9
:104C40001B88012B7EF431AA99F80020A2F10C00F8
:104C50007F287FF7B0A88B3A0C2092FBF0F300FB83
:104C600013207330FFF799B8114B01227F210720E1
:104C70001A8003F071FB7F210B2003F06DFBFDF721
:104C8000B8BE00BF6E9BFF1FC79BFF1F389DFF1F55
:104C9000749BFF1FB89CFF1FC69BFF1FA29BFF1F9B
:104CA000C89BFF1F249DFF1FD29CFF1FE00B01002C
:104CB000D69BFF1F629BFF1FC74B04227F2107204B
:104CC0001A8003F049FB00210B2003F045FBFDF7A0
:104CD00089BEC14B02227F2107201A8003F03CFBD2
:104CE0007F210B2003F038FBFDF777BEBA4B002184
:104CF00007201C8003F030FB7F210B2003F02CFBEE
:104D0000FDF766BEB54B00227F2107201A8003F015
:104D100023FB7F210B2003F01FFBFDF772BEFBF787
:104D20009BFC0EE4AE4B1B88182B12D099F8002088
:104D30001344A3F118007F2840F344810C20973BD3
:104D400093FBF0F200FB123303F17300C0B203F0E7
:104D500053FBA44AA44B127833F81230182B3EF4BC
:104D6000A4A999F800201344A3F118007F287FF725
:104D700022A80C20973B93FBF0F200FB123303F1C7
:104D80007300FFF70AB8994A1288182A12D0134400
:104D9000A3F118007F2840F300810C20973B93FB80
:104DA000F0F200FB123303F17300C0B298F8001068
:104DB00003F0FAFA8B4B8E491A78022A94BF01321B
:104DC00000221A701A7831F8120018287FF4FCAD0E
:104DD0000424022A02F1010294BFD2B2002231F867
:104DE000120018287FF4EFAD013CF2D1E7E5FBF7A4
:104DF00033FC4FE47D4B1A88182A13D03B681344C8
:104E0000A3F118007F2840F3D4800C20973B93FB3C
:104E1000F0F200FB123303F17300764BC0B2197845
:104E200003F0C2FA6F4B72491A78022A94BF01321A
:104E300000221A701A7831F8120018287FF4F4ACA6
:104E40000424022A02F1010294BFD2B2002231F8F6
:104E5000120018287FF4E7AC013CF2D11A70FDF77C
:104E60003DBEFBF7F9FBFFF7CABA604B1B88182B56
:104E700012D099F800201344A3F118007F2840F3C2
:104E80009B800C20973B93FBF0F200FB123303F165
:104E90007300C0B203F0B0FA524A554B127833F89F
:104EA0001230182B7FF4F5ACFDF7CDBCFBF7D4FB2B
:104EB000FFF770BB504ADFF854B11288BBF80010FE
:104EC000033291427FF764AE3BE6FBF7C5FBF9E5A1
:104ED000FBF7C2FB08E4FBF7BFFBCFE4434B1B88A7
:104EE000182B11D099F800201344A3F118007F2843
:104EF00059DD0C20973B93FBF0F200FB123303F1DA
:104F00007300C0B203F078FA364A394B127833F89E
:104F10001230182B7FF425AFFEF7C7B8374B1B882C
:104F2000182B11D099F800201344A3F118007F2802
:104F30003CDD0C20973B93FBF0F200FB123303F1B6
:104F40007300C0B203F058FA264A2D4B127833F89A
:104F50001230182B7FF405AFFEF7A7B8FBF77CFBE8
:104F6000FFF741BBFBF778FB3BE4FBF775FB0CE677
:104F7000FBF772FBFFF7E2BBFBF76EFB4CE5FBF7C1
:104F80006BFB69E5FBF768FBFAE4FBF765FBFFF7F2
:104F900060BAFBF761FBFFF786BAFBF75DFB04E73E
:104FA000FBF75AFB19E6FBF757FBAAE7FBF754FBA5
:104FB000C7E7FBF751FB30E7FBF74EFB69E7FBF771
:104FC0004BFB32E6FBF748FBC0E60E4B03930E4B60
:104FD0000293FDF747BF00BF1A9DFF1F509BFF1FA5
:104FE0006E9BFF1FC79BFF1F389DFF1F769BFF1FF8
:104FF000C09CFF1FC69BFF1FA29BFF1F749BFF1F30
:10500000B89CFF1F259BFF1FE29BFF1F629BFF1F9A
:1050100038B507F09FF80B4804F0D6FF00234FF097
:105020007E5201210848FBF721FA084B084A09493A
:10503000802400251C7118461D60BDE838400AF028
:105040004DBD00BFD49BFF1FF89CFF1F789DFF1F25
:105050001C89FF1FFD05000043682A20198803F002
:10506000FFBA00BF10B5044622206368198803F018
:10507000F7FAE36824201988BDE8104003F0F0BA7D
:1050800010B504460A206368198803F0E9FAE3685A
:105090000C201988BDE8104003F0E2BA10B50446B0
:1050A00006206368198803F0DBFAE3680820198892
:1050B000BDE8104003F0D4BA10B50446022063687E
:1050C000198803F0CDFAE36804201988BDE8104080
:1050D00003F0C6BA70B50E4C84B012250422012329
:1050E00006460390029320468DE8240014231021E5
:1050F00006F06EF9062209230293039601952046D5
:1051000000921423102106F063F904B070BD00BFB3
:10511000E09DFF1F2DE9F041224D82B0012602B231
:1051200084B20092284601967823192106F096F859
:1051300004F10C0212B28DE844002846A719782326
:10514000192104F1020806F089F83FB20FFA88F835
:1051500019233A46284619460196CDF8008006F0F4
:105160007DF878233A4628461946CDF80080019606
:1051700004F10A070B3406F071F83FB224B2782329
:105180003A46284619468DE8500006F067F819237C
:1051900000943A4601962846194606F05FF802B098
:1051A000BDE8F081E09DFF1F2DE9F0411E4682B071
:1051B0001446002A6AD0099B4D4A00EBC305012C16
:1051C0006F8929896868A7EB010382FB03E21A440F
:1051D0004FEAE373C3EBA21302887BD0042C38D1CF
:1051E00012FA83F3994203DC9F423946A8BF19465D
:1051F000089A0180B6F90030BDF920803D48971D1E
:105200004FF0000E3FB2194642460097CDF804E039
:1052100006F024F829896A896B68521A1B885C2A6F
:10522000A3EB010359DD03EB43030132C3EB43134B
:1052300093FBF2F303F11B0213B2012032801946F3
:105240004246019000972B4806F008F82A4B0022AE
:105250001A702A4B022CB3F9001045D0082C31D11A
:1052600000221A8091422DD0089AB6F900302148C8
:105270000632012412B2009219460194BDF9202091
:1052800005F0ECFF204602B0BDE8F0811C4D1D4A40
:105290002B681268CB1A93420F4617D9164A3388E7
:1052A00011781448012918BF01241470089A063295
:1052B0001BB212B28DE814001946BDF9202005F08A
:1052C000CDFF2F60012002B0BDE8F081204602B082
:1052D000BDE8F0819BB2D31A84E75C2101FB03F3A4
:1052E00093FBF2F21B32A7E74A1C12B21A80B9E70D
:1052F000C94216B2E09DFF1F5D9EFF1FC29DFF1FAA
:10530000449EFF1F7023010030B583B000230C467C
:1053100005B2009326225B231C210C4805F0EEFC0D
:10532000294601232622094804F0F8FF002C24B264
:1053300005DB214601232622044804F0EFFF044A3E
:10534000044B15801C8003B030BD00BFE09DFF1FE3
:10535000A889FF1FAA89FF1F70B5944C237882B0DB
:105360001BB1934B4FF6FF721A80924BB3F900308A
:10537000C3B9914A8E4B1068B3F9002080F30C003A
:105380005B2303FB00F000131C3082425AD04FF025
:10539000FF31FFF7B9FF894805F014FD00232370A2
:1053A00002B070BD012B32D0022B6AD0032B4FD03C
:1053B000042BF3D1272200258DE8240076231C211D
:1053C0007E487F4E05F04AFF17E0B0F5AF7FA8BFDB
:1053D0004FF4AF70323803FB00F386FB0321DB1779
:1053E000C3EB61111C3109B201231D44272273480C
:1053F00004F094FF0C2D00F08180E9B2714804F0B4
:105400004BFE31284FF05B03DFDC1C21ECE76E4BD9
:105410001A68B2F52F7F32DB41F25C239342A8BFBA
:105420001346A3F52F735B22684802FB03F380FB4E
:105430000320DB17C3EBA0201C305D4BB3F9003019
:105440008342A4D1624BB3F9003001339FD1A5E769
:10545000604B1B68B3F5FA7F11DBB3F57A6FA8BF19
:105460004FF47A63A3F5FA725B485B2303FB02F304
:1054700080FB0320DB17C3EB20201C30DDE71C2062
:10548000DBE7564B1B68B3F5FA7F33DBB3F57A6F76
:10549000A8BF4FF47A63A3F5FA724F485B2303FB6E
:1054A00002F380FB0320DB17C3EB20201C304C4BA6
:1054B0001B68B3F5FA7F1FDBB3F57A6FA8BF4FF413
:1054C0007A63A3F5FA7244495B2303FB02F381FB81
:1054D0000321DB17C3EB21211C31354BB3F900301D
:1054E00083427FF456AF3A4BB3F900308B427FF4DE
:1054F00050AF53E71C20DAE71C21EEE7012007F04C
:10550000D1FC6FF495733238364A03FB00F082FB0E
:105510000023C017C0EB632303F5AF73312B3ADDD3
:10552000B3F5AF7FA8BF4FF4AF735B22323B244D7E
:1055300002FB03F385FB0325DB17C3EB65151C3565
:10554000002007F0AFFC6FF495733238254A03FB57
:1055500000F082FB0023C017C0EB632303F5AF7399
:10556000312B1ADDB3F5AF7FA8BF4FF4AF735B22C9
:10557000323B134902FB03F381FB0321DB17C3EB2F
:1055800061111C310A4BB3F90030AB4207D02846F9
:10559000FFF7BAFEFFE61C25D2E71C21F2E70C4B11
:1055A000B3F900308B42F2D1F5E600BFB89DFF1F82
:1055B000A889FF1FBE9DFF1F2C9DFF1FE09DFF1FA1
:1055C0004B48371BD49BFF1F349BFF1FD3058541DE
:1055D000AA89FF1F849BFF1F011FB8128C9BFF1F0E
:1055E000A89DFF1F67BBCF462DE9F04FDFF8EC8287
:1055F000B74CB8F900604D7854F8264087B0824621
:10560000039305B10D78DFF8FCB2002A34D19BF882
:1056100000308BBBAF4EB6F90000002800F0CE8002
:10562000012800F02481012032232A4601900093B2
:105630005146A94B2046FFF7B7FD00250746B6F9AE
:105640000030022B40F3F48000233380B8F900309F
:10565000A24A002BC0F2F880042BC4BF00231380A1
:10566000039B002B40F0F680002D0CBF38464FF016
:10567000FF3007B0BDE8F08F964EE3682268984887
:1056800004930027059237808BF8007005F08EFA9E
:105690001120FFF73FFD4FF0010919232821CDF814
:1056A00004900091242219468D4805F0D7FD7823F7
:1056B00028212422CDF8049000918948194605F04C
:1056C000CDFD4946864806F05FF90222192184483B
:1056D00006F056F9DDF8149048460AF0D1FF494625
:1056E00002467F4806F0E6FA7D4806F0F9FA3946A8
:1056F00014227B4806F044F903227A49784806F0E0
:10570000D9FA774806F0ECFA39462322744806F0B5
:1057100037F903227449724806F0CCFA704806F053
:10572000DFFA049B002B72D10123704A18461370D4
:10573000FFF7D0FC208963896768191A5C293A88C9
:105740005BDC131A5C2202FB03F292FBF1F31B33C6
:10575000674A6348138001271BB21A2219468DE855
:105760008400142205F07AFD049BDBB1218A638A50
:10577000E768581A5C283A886FDD521A02EB420239
:10578000C2EB4212431C92FBF3F31B33524A5448C0
:105790001380012738221BB28DE88400194632227B
:1057A00005F05CFD534A544BB6F90000012111701D
:1057B0004FF6FF721A8000287FF432AFDFF848916D
:1057C0004E4AD9F800301268C3EB0A0393424CD911
:1057D000464B1A78012A18BF012018700127FFF7DD
:1057E00079FCC9F800A0012D4ED0042D59D0022D0E
:1057F00060D0082D64D0002521E7121A02EB420286
:10580000C2EB42124B1C92FBF3F31B33A0E72F2099
:10581000FFF780FC39463222314806F0B1F8032206
:1058200037492F4806F046FA2D4806F059FA7BE72B
:105830007FF40CAFE368002B3FF406AFB8F90030FB
:10584000264A002BBFF608AF04231380039B002BCE
:105850003FF40AAFFFF780FD06E7511A5C2202FB16
:1058600001F292FBF0F31B3390E70746BBE70027FA
:1058700014238DE888002A4651461D4B2046FFF729
:1058800093FC3D460746DAE6B8F800308BF8005046
:105890000133A8F80030636983B10025204698479A
:1058A000CDE6B8F800300122013BA8F800308BF8B3
:1058B0000020F0E7012333800025C7E61D46BEE641
:1058C0006369002232804FF0FF35002BE6D1BDE640
:1058D000AC89FF1FC29DFF1FBC9DFF1FBE9DFF1F08
:1058E000E09DFF1FF4140100F81401005D9EFF1FEE
:1058F000BA9DFF1FB89DFF1FA889FF1F70230100DD
:10590000FC140100C09DFF1F449EFF1F01210D20BC
:1059100007F09AB800210D2007F096B801460D2037
:1059200007F092B808B50D2007F094F8B0FA80F1AE
:1059300049090D20BDE8084007F086B810B50021E0
:1059400044080D2007F080F8204607F0B9F80D2034
:10595000012107F079F82046BDE8104007F0B0B803
:10596000214A224B10881B68984210B535DA204A2C
:105970001288141A9A42A8BF1A46B4F5157F22DA83
:10598000121A40F2532303FB02F393FBF4F10531A7
:105990000A2006F0C9FE174B197801B3164B1749B8
:1059A0001B6840F2271283F3070302FB03F381FB1A
:1059B00003211944DB17C3EBA11105310920BDE810
:1059C000104006F0B1BE131A4FF41572611C02FBB1
:1059D00003F393FBF1F10531DAE70021D8E7092061
:1059E000BDE8104006F0A0BEE09BFF1F289BFF1FF4
:1059F0008C9DFF1FA49BFF1F2C9BFF1F090402818E
:105A00007F2838B5A8BF7F200F4C4FF4167202FBD9
:105A100000F284FB02311144D2170546C2EBA111FA
:105A20000A2006F081FE7F3D4FF4967303FB05F3D9
:105A300084FB03211944DB17A3EBA1110920BDE866
:105A4000384006F071BE00BF09040281C368B3F993
:105A5000003030B583EAE374A4EBE374002BA0B20A
:105A600018DB012300E0134603EB8302520094424B
:105A7000F9DA0A4D90FBF3F285FB03E403FB120015
:105A8000DB173032D3EBA40380B201F8012BF1D144
:105A90000B7030BD2D230B700131E2E7676666663F
:105AA00038B5094D8224204602F0F4FD35F8021B7A
:105AB00000B28842204601D002F0D2FD0234A4B2E6
:105AC0008A2CF0D138BD00BFC09CFF1F024B802044
:105AD000198802F0C5BD00BF769BFF1F38B5094D80
:105AE0007824204602F0D6FD35F8021B00B2884229
:105AF000204601D002F0B4FD0234A4B2802CF0D1D3
:105B000038BD00BFB89CFF1F024B7620198802F0F9
:105B1000A7BD00BF749BFF1F38B5094D4624204622
:105B200002F0B8FD35F8021B00B28842204601D0D1
:105B300002F096FD0234A4B24E2CF0D138BD00BF65
:105B4000389DFF1F024B4420198802F089BD00BF19
:105B50006E9BFF1F024B4E20198802F081BD00BFD3
:105B6000889BFF1F024B9A20198802F079BD00BF65
:105B7000C89BFF1F024B9820198802F071BD00BF1F
:105B8000A29BFF1F024B8C20198802F069BD00BF49
:105B9000D29CFF1F024B9C20198802F061BD00BF00
:105BA000629BFF1F024B9620198802F059BD00BF6F
:105BB000249DFF1F024B8A20198802F051BD00BFAF
:105BC000E69CFF1F024B1020198802F049BD00BF60
:105BD000E49CFF1F024B2C20198802F041BD00BF3E
:105BE000609BFF1F024B1E20198802F039BD00BFC9
:105BF0005C9BFF1FC3680E20198802F031BD00BFF7
:105C0000024B2820198802F02BBD00BF349DFF1FD6
:105C1000024B6220198802F023BD00BF929BFF1F38
:105C2000024B6420198802F01BBD00BF309DFF1F8E
:105C3000024B5A20198802F013BD00BF709BFF1F52
:105C4000024B1620198802F00BBD00BF509BFF1FAE
:105C5000024B2E20198802F003BD00BFD09BFF1F0E
:105C6000024B3020198802F0FBBC00BF9E9DFF1F35
:105C7000024B1820198802F0F3BC00BFE49BFF1F01
:105C8000024B1A20198802F0EBBC00BF909BFF1F4B
:105C9000024B1C20198802F0E3BC00BF8A9BFF1F47
:105CA000024B6620198802F0DBBC00BF729DFF1F0B
:105CB000024B7220198802F0D3BC00BF949DFF1FD5
:105CC000024B2020198802F0CBBC00BF709DFF1F43
:105CD000024B3220198802F0C3BC00BF629DFF1F37
:105CE000024B6820198802F0BBBC00BFBC9BFF1FA1
:105CF000024B6C20198802F0B3BC00BF309BFF1F21
:105D0000024B5220198802F0ABBC00BF2E89FF1F46
:105D1000024B5020198802F0A3BC00BFA089FF1FCE
:105D2000024B5420198802F09BBC00BFA289FF1FC0
:105D3000024B5C20198802F093BC00BFA689FF1FAC
:105D4000024B5E20198802F08BBC00BF2C89FF1F1C
:105D5000024B6020198802F083BC00BFD49CFF1F57
:105D6000024B5620198802F07BBC00BFC49BFF1F6A
:105D7000244B1B880B2B43D8DFE803F00B10151ABC
:105D80001F24292E33383D06084604221E490AF0F6
:105D900035BD084604221D490AF030BD08460422DC
:105DA0001B490AF02BBD084604221A490AF026BDF9
:105DB0000846042218490AF021BD08460422174962
:105DC0000AF01CBD0846042215490AF017BD084612
:105DD000042214490AF012BD0846042212490AF0AE
:105DE0000DBD0846042211490AF008BD08460422E8
:105DF0000F490AF003BD084604220E490AF0FEBC12
:105E0000704700BF249DFF1F202001001C1E0100C1
:105E1000D01C0100D4200100D41C0100BC200100D2
:105E2000D81C0100DC1C0100401F0100E01C010027
:105E30002C200100E41C0100064B074A10B41C880A
:105E4000064B0846002C14BF11461946042210BC0C
:105E50000AF0D4BCA09BFF1FE81C0100EC1C010051
:105E6000064B074A10B41C88064B0846002C14BF8A
:105E700011461946042210BC0AF0C0BCD29BFF1F79
:105E8000E81C0100EC1C0100064B074A10B41C88FA
:105E9000064B0846002C14BF11461946042210BCBC
:105EA0000AF0ACBCD69CFF1FE81C0100EC1C0100F2
:105EB000064B074A10B41C88064B0846002C14BF3A
:105EC00011461946042210BC0AF098BCEC9CFF1F36
:105ED000E81C0100EC1C0100064B074A10B41C88AA
:105EE000064B0846002C14BF11461946042210BC6C
:105EF0000AF084BC269DFF1FE81C0100EC1C010079
:105F0000064B074A10B41C88064B0846002C14BFE9
:105F100011461946042210BC0AF070BCD69BFF1F24
:105F2000E81C0100EC1C01001B4B1B880A2B0AD843
:105F3000DFE803F00A0E12161A1E22262A2E060089
:105F4000164B186808607047154B18680860704752
:105F5000144B186808607047134B18680860704746
:105F6000124B186808607047114B1868086070473A
:105F7000104B1868086070470F4B1868086070472E
:105F80000E4B1868086070470D4B18680860704722
:105F90000C4B186808607047E69CFF1F141D010039
:105FA000EC1C0100F01C0100F41C0100F81C0100B5
:105FB000FC1C0100001D0100041D0100081D010062
:105FC0000C1D0100101D0100F0B52B4E2B4FDFF80A
:105FD000C4E005460FCE87B06C460FC496E80300B8
:105FE0003B68274A274F44F8040B40F6CC308342E5
:105FF000C8BF3A46BEF800602180012E1188927811
:10600000ADF80D108DF80F202AD032D340F6CA0219
:10601000022E18BF00229A4226DCA3F698031A49E2
:106020001A4AC3EB031381FB03011944DB17C3EBCB
:106030006123243382FB0321DA17C2EBA10202EBB6
:106040008201A3EB4103303330328DF813308DF8E9
:1060500011206946284616220AF0D0FB07B0F0BD91
:1060600040F698029A42D8DD094B1868CDF8110025
:10607000EFE740F6FC02CEE7281D01004C9DFF1F14
:106080001C1D0100181D01003B773B986766666682
:10609000201D0100C89CFF1FF8B5174C174E227831
:1060A000174D33782F888E46003218BF01220146E3
:1060B0007046FFF799FA002398423370237015DB7E
:1060C00014BF012000202B889F420ED040F23A726C
:1060D000A3F5AF730B490C4C02FB03F381FB0312D6
:1060E000DB17A3EB621332332360F8BD07490122AB
:1060F00018460A702270E6E7748AFF1FD19DFF1FC1
:10610000849DFF1FB5814E1B9089FF1F5C9EFF1F62
:10611000014B187802F03CBA409EFF1F014B1878E3
:1061200002F050BAF08FFF1F134BB3F9003030B5B7
:1061300083EAE374A4EBE374002BA0B218DB012321
:1061400000E0134603EB830252009442F9DA0B4D50
:1061500090FBF3F285FB03E403FB1200DB17303204
:10616000D3EBA40380B201F8012BF1D10B7030BD49
:106170002D230B700131E2E7F08FFF1F6766666623
:10618000144BB3F9003070B583EAE375A5EBE37502
:10619000002BACB21ADB012300E0034603EB8300C3
:1061A00040008542F9DA0C4E94FBF3F086FB03E5E0
:1061B00003FB1044DB173030D3EBA503A4B201F886
:1061C000010BF1D105480B70106070BD2D230B70D1
:1061D0000131E0E7709BFF1F67666666401D0100A6
:1061E000134BB3F9003030B583EAE374A4EBE374E6
:1061F000002BA0B218DB012300E0134603EB83025F
:1062000052009442F9DA0B4D90FBF3F285FB03E464
:1062100003FB1200DB173032D3EBA40380B201F88A
:10622000012BF1D10B7030BD2D230B700131E2E752
:106230002E89FF1F67666666134BB3F9003030B5D1
:1062400083EAE374A4EBE374002BA0B218DB012310
:1062500000E0134603EB830252009442F9DA0B4D3F
:1062600090FBF3F285FB03E403FB1200DB173032F3
:10627000D3EBA40380B201F8012BF1D10B7030BD38
:106280002D230B700131E2E7A089FF1F6766666668
:10629000134BB3F9003030B583EAE374A4EBE37435
:1062A000002BA0B218DB012300E0134603EB8302AE
:1062B00052009442F9DA0B4D90FBF3F285FB03E4B4
:1062C00003FB1200DB173032D3EBA40380B201F8DA
:1062D000012BF1D10B7030BD2D230B700131E2E7A2
:1062E000A289FF1F67666666134BB3F9003030B5AD
:1062F00083EAE374A4EBE374002BA0B218DB012360
:1063000000E0134603EB830252009442F9DA0B4D8E
:1063100090FBF3F285FB03E403FB1200DB17303242
:10632000D3EBA40380B201F8012BF1D10B7030BD87
:106330002D230B700131E2E7A689FF1F67666666B1
:10634000134BB3F9003030B583EAE374A4EBE37484
:10635000002BA0B218DB012300E0134603EB8302FD
:1063600052009442F9DA0B4D90FBF3F285FB03E403
:1063700003FB1200DB173032D3EBA40380B201F829
:10638000012BF1D10B7030BD2D230B700131E2E7F1
:106390002C89FF1F6766666608B5702002F07AF9DF
:1063A000044B1988884204D07020BDE8084002F0F0
:1063B00057B908BDC89CFF1F08B5742002F06AF9E0
:1063C000044B1988884204D07420BDE8084002F0CC
:1063D00047B908BD589DFF1F054B1B88084604227E
:1063E00013B904490AF00ABA03490AF007BA00BF10
:1063F000889BFF1F481D0100441D01000E4B1B8898
:10640000032B17D8DFE803F0110C0702084604221B
:106410000A490AF0F3B90846042209490AF0EEB91C
:106420000846042207490AF0E9B908460422064949
:106430000AF0E4B9704700BFD29CFF1F581D01004D
:10644000541D0100501D01004C1D010010B40A4BE9
:106450000A4C0A4693E8030083B0238802AC04E99F
:10646000030004EB8303104653F8081C052203B015
:1064700010BC0AF0C3B900BF84150100309DFF1F96
:1064800030B40A4B0A4D0C4693E8070084B02B88C1
:1064900004AD05E9070005EB8303204653F80C1C07
:1064A000042204B030BC0AF0A9B900BF8C15010069
:1064B000C89CFF1FF0B40C4D0C4F0E460FCD8CB096
:1064C00001AC0FC40FCD0FC495E807003B8884E8EA
:1064D00007000CAA02EB8303304653F82C1C04225D
:1064E0000CB0F0BC0AF08AB9981501001A9DFF1F84
:1064F000F0B40A4D0A4F0E460FCD86B001AC0FC462
:106500002A683B88226006AA02EB8303304653F8D0
:10651000141C042206B0F0BC0AF070B9C4150100C6
:10652000E49BFF1FF0B40A4D0A4F0E460FCD86B014
:1065300001AC0FC42A683B88226006AA02EB8303E1
:10654000304653F8141C0C2206B0F0BC0AF056B9C1
:10655000D81501008A9BFF1FF0B40A4D0A4F0E4662
:106560000FCD86B001AC0FC42A683B88226006AA12
:1065700002EB8303304653F8141C042206B0F0BC2F
:106580000AF03CB9EC150100589DFF1F164B1B8803
:106590000BB31BB283EAE370A0EBE370002B30B5C2
:1065A00084B21DDB012300E0134603EB830252009B
:1065B0009042F9DA0D4894FBF3F280FB03E503FB0C
:1065C0001244DB173032D3EBA503A4B201F8012B40
:1065D000F1D10B7030BD0846042205490AF00EB90E
:1065E0002D230B700131DDE7BC9BFF1F67666666DC
:1065F0005C1D010030B40A4B0A4D0C4693E80700BD
:1066000084B02B8804AD05E9070005EB8303204621
:1066100053F80C1C042204B030BC0AF0EFB800BFE1
:1066200000160100309BFF1F054B1B881BB9054B53
:106630001868086070470846042203490AF0DEB86B
:10664000C89BFF1FEC1C0100E81C0100164B1B88B7
:106650000BB31BB230B583EAE374A4EBE374002BF5
:10666000A0B21CDB012300E0134603EB83025200BF
:106670009442F9DA0D4D90FBF3F285FB03E403FB42
:106680001200DB173032D3EBA40380B201F8012BE8
:10669000F1D10B7030BD064B1868086070472D2390
:1066A0000B700131DEE700BF5C9BFF1F676666660B
:1066B000EC1C0100164B1B880BB31BB230B583EAF0
:1066C000E374A4EBE374002BA0B21CDB012300E015
:1066D000134603EB830252009442F9DA0D4D90FB0E
:1066E000F3F285FB03E403FB1200DB173032D3EB3C
:1066F000A40380B201F8012BF1D10B7030BD064B21
:106700001868086070472D230B700131DEE700BF69
:10671000669DFF1F67666666EC1C0100164B1B88B2
:106720000BB31BB230B583EAE374A4EBE374002B24
:10673000A0B21CDB012300E0134603EB83025200EE
:106740009442F9DA0D4D90FBF3F285FB03E403FB71
:106750001200DB173032D3EBA40380B201F8012B17
:10676000F1D10B7030BD064B1868086070472D23BF
:106770000B700131DEE700BF509BFF1F6766666646
:10678000601D0100174B1B881BB31BB270B583EA59
:10679000E375A5EBE375002BACB21EDB012300E033
:1067A000034603EB830040008542F9DA0E4E94FB6A
:1067B000F3F086FB03E503FB1044DB173030D3EB2B
:1067C000A503A4B201F8010BF1D108480B701060C9
:1067D00070BD074B1868086070472D230B7001319E
:1067E000DCE700BFD09BFF1F67666666241D0100C3
:1067F000EC1C0100164B1B880BB31BB230B583EAAF
:10680000E374A4EBE374002BA0B21CDB012300E0D3
:10681000134603EB830252009442F9DA0D4D90FBCC
:10682000F3F285FB03E403FB1200DB173032D3EBFA
:10683000A40380B201F8012BF1D10B7030BD064BDF
:106840001868086070472D230B700131DEE700BF28
:106850009E9DFF1F67666666EC1C0100164B1B8839
:106860000BB31BB230B583EAE374A4EBE374002BE3
:10687000A0B21CDB012300E0134603EB83025200AD
:106880009442F9DA0D4D90FBF3F285FB03E403FB30
:106890001200DB173032D3EBA40380B201F8012BD6
:1068A000F1D10B7030BD064B1868086070472D237E
:1068B0000B700131DEE700BF729DFF1F67666666E1
:1068C000EC1C0100164B1B880BB31BB230B583EADE
:1068D000E374A4EBE374002BA0B21CDB012300E003
:1068E000134603EB830252009442F9DA0D4D90FBFC
:1068F000F3F285FB03E403FB1200DB173032D3EB2A
:10690000A40380B201F8012BF1D10B7030BD064B0E
:106910001868086070472D230B700131DEE700BF57
:10692000949DFF1F67666666EC1C0100174B1B8871
:106930001BB31BB270B583EAE375A5EBE375002BBF
:10694000ACB21EDB012300E0034603EB83004000F2
:106950008542F9DA0E4E94FBF3F086FB03E503FB68
:106960001044DB173030D3EBA503A4B201F8010BC0
:10697000F1D108480B70106070BD074B18680860B3
:1069800070472D230B700131DCE700BF709DFF1FA6
:1069900067666666641D0100EC1C0100074B1B88DE
:1069A000022B06D0012B0CBF054B064B1868086064
:1069B0007047054B18680860704700BFD49CFF1FE4
:1069C0006C1D0100701D0100681D0100054B1B8836
:1069D0001BB1054B186808607047044B18680860C5
:1069E000704700BFC49BFF1F781D0100741D01008C
:1069F00038B5FBF731F80D4B1B7833B90C4B102031
:106A0000198801F02DFE012038BD0A4D0A4C2B7863
:106A10002288B3FA83F382F008025B091146422010
:106A20002B70228001F01CFE002038BD189DFF1F36
:106A3000E49CFF1FCB9CFF1F6C9BFF1F184B1A8809
:106A400052B3184A128830B50A80B3F90030002BCF
:106A500083EAE374A4EBE374BCBF2D238B70A0B274
:106A6000ACBF02310331012300E0134603EB830284
:106A700052009442F9DA0C4D90FBF3F285FB03E4EB
:106A800003FB1200DB173032D3EBA40380B201F812
:106A9000012BF1D10B7030BD044B186808607047B2
:106AA000909BFF1F7C1D010067666666EC1C010061
:106AB00070B53C4D2B780646002B35D11C467378BB
:106AC0000BB9204670BDFAF7C7FF374A374B384835
:106AD000127831781B78007802EB43034A1E03EBEF
:106AE00080030E2AEDD801A050F822F0556B00006B
:106AF000776B0000C36A0000556B0000C36A00009A
:106B0000C36A0000C36A0000436B0000C36A000050
:106B1000C36A0000C36A0000C36A0000C36A0000C1
:106B2000C36A00003F6B0000AE21224803F0EEFD77
:106B3000204804F03BF800232B700124BFE706F047
:106B4000D1FAAF211B4803F0E1FD1B4A012313706A
:106B50002B70B6E783B91948038804294FF6FF71F3
:106B600003F1FF320CBF01230B46134403F07F03F4
:106B7000013303800FE073B1013B114A32F8133047
:106B80004BB10E4E0F481049104A338001230026A6
:106B900006700B701370084A0221012311702B70CC
:106BA000204670BD748AFF1FB49DFF1FB59DFF1F57
:106BB000689DFF1FE09DFF1F5C9EFF1F649DFF1FE0
:106BC0003C9BFF1FB49BFF1F529BFF1F5F9EFF1F3D
:106BD00010B5064B064C1A882046012101F02EFD07
:106BE00021884220BDE8104001F03ABDA09BFF1F64
:106BF0006C9BFF1F10B5064B064C1A8820460221DD
:106C000001F01CFD21884220BDE8104001F028BDA4
:106C1000D29BFF1F6C9BFF1F10B5064B064C1A88BA
:106C20002046042101F00AFD21884220BDE81040E1
:106C300001F016BDD69CFF1F6C9BFF1F10B5064BC5
:106C4000064C1A882046062101F0F8FC21884220D3
:106C5000BDE8104001F004BDEC9CFF1F6C9BFF1FC2
:106C600010B5064B064C1A882046002101F0E6FCC0
:106C700021884220BDE8104001F0F2BC269DFF1F94
:106C80006C9BFF1F08B5122001F004FD054B19880D
:106C9000884206D0122001F0E3FCBDE8084001F074
:106CA000F7BB08BD1A9DFF1F08B5582001F0F2FC84
:106CB000054B1988884206D0582001F0D1FCBDE868
:106CC000084001F0E5BB08BD669DFF1F08B5142014
:106CD00001F0E0FC054B1988884206D0142001F031
:106CE000BFFCBDE8084001F0D3BB08BDD69BFF1F29
:106CF000F0B480EAE075A5EBE0750028ACB21FDBCC
:106D00001DBF2B230B704E1C0E46012300E01346C3
:106D100003EB830252009542F9DA0B4F94FBF3F236
:106D200087FB030503FB1244DB173032D3EBA503CB
:106D3000A4B206F8012BF1D133700846F0BC7047BD
:106D40002D230B704E1CE0E767666666174B1888AC
:106D50000C2813D0192815D01A2817D01B2819D0A1
:106D60001C281BD01D281DD01E2803D00C3800B2B3
:106D7000FFF7BEBF0E4A1068086070470D4A1068E2
:106D8000086070470C4A1068086070470B4A10682A
:106D9000086070470A4A106808607047094A10681E
:106DA00008607047084A106808607047629DFF1FBE
:106DB0009C1D0100841D0100881D01008C1D010027
:106DC000901D0100941D0100981D0100034B1888BF
:106DD000A0EB8000400000B2FFF78ABF409EFF1F7B
:106DE000024BB3F90000FFF783BF00BF929BFF1F68
:106DF000024B1888033800B2FFF77ABF349DFF1F9B
:106E0000024B18880C3800B2FFF772BF4C9BFF1F73
:106E1000024B1888183800B2FFF76ABF769BFF1F35
:106E2000024B1888183800B2FFF762BF749BFF1F2F
:106E3000024B1888183800B2FFF75ABF6E9BFF1F2D
:106E4000C3681888183800B2FFF752BF054B1B887B
:106E50001BB9054B186808607047084604220349AF
:106E600009F0CCBCA29BFF1FEC1C0100E81C010038
:106E700030B5134C85B001252B463C22022120461B
:106E8000009503F0B9FC204603F090FE002240215B
:106E9000802320460191009311460A4B029504F08D
:106EA00033FB204603F08EFF07480849084A0023B9
:106EB000036083800B608B801360938005B030BDCE
:106EC000E09DFF1F4C160100C49DFF1FD89DFF1FB2
:106ED0004C9EFF1F10B500EBC00000F10F02D2B2B4
:106EE00093B284B09C1E981C3D2303918DE8190039
:106EF0003921024804F06CFA04B010BDE09DFF1F78
:106F0000014B01221A707047D19DFF1FF0B585B06B
:106F1000664C674B0293674A019204230093204614
:106F2000654B664F664E674D4022802103F06CFA38
:106F30002046654A6549664C08F0D0FD654B6648B9
:106F40009F61664FDF61664FB761664FF761664FBD
:106F5000AF61664FEF61664FA761664FE761664FAD
:106F600087616649664FC761664F8F61664A674FA2
:106F7000CF61674F9761674B674FD761674F9F61DD
:106F8000674E684FDF61684FB761684D684FF761C2
:106F9000684F694CAF61694FEF61694F6948A761FC
:106FA000694FE761694F6A4987616A4FC7616A4FF4
:106FB0006A4A8F616A4FCF616A4F6B4B97616B4F23
:106FC000D7616B4F6B4E9F616B4FDF616B4F6C4DA9
:106FD000B7616C4FF7616C4FAF616C4C6C4FEF61F8
:106FE0006C4FA7616C486D4FE7616D4F87616D49CC
:106FF0006D4FC7616D4F8F616D4A6E4FCF616E4FA0
:1070000097616E4B6E4FD7616E4F9F616E4E6F4FA3
:10701000DF616F4FB7616F4D6F4FF7616F4FAF61BA
:107020006F4C704FEF61704FA7617048704FE76110
:10703000704F87617049714FC761714F714A8F619D
:10704000714FCF61714F724B9761724FD761724F21
:10705000724E9F61724FDF61724F734DB761734F14
:10706000F761734F734CAF61734F74487449EF61AC
:10707000744F754DA761E561744F754D754CDFF820
:10708000F8E1754A754B8761754EC561754F8C6126
:10709000754D764CC1F81CE0754876499761D5610D
:1070A0009C61D861B16005B0F0BD00BFE09DFF1FDD
:1070B000A0860100801A06000C90FF1F016E0000E0
:1070C000548EFF1FC48DFF1F1C89FF1F61A4000089
:1070D000B88BFF1FE489FF1F788EFF1FF55B000050
:1070E000F16D0000015C0000395E0000D16B000012
:1070F000615E0000F56B0000895E0000088AFF1FDA
:10710000196C0000E16D0000488CFF1F115C00004D
:10711000B15E0000D88CFF1F3D6C00004D64000084
:10712000248CFF1F215C0000D95E0000B48CFF1F7F
:10713000616C0000CD6D0000908CFF1F116100009C
:1071400029610000308EFF1F1D6100008164000076
:10715000708BFF1F99630000B5640000E08EFF1F75
:10716000856C0000B5660000008CFF1FA96C000054
:10717000816100002C8BFF1F315C0000015F00006B
:107180004C8FFF1FCD6C00001D670000DC8BFF1FC4
:10719000415C000085670000FC8CFF1F515C000013
:1071A000F56700009C8AFF1F615C0000F16400002D
:1071B0006C8CFF1F715C00003D6A00000C8EFF1F8D
:1071C000815C000025650000CC8FFF1F915C0000F2
:1071D0005D680000A08DFF1FA15C0000C568000075
:1071E000C08AFF1FB15C000059650000048FFF1FBB
:1071F000B96300002D690000E88DFF1FC15C00002D
:107200004D6D0000E48AFF1FD15C00008D65000019
:10721000788AFF1FE15C0000F56500009C8FFF1F6E
:10722000F15C0000E1610000948BFF1F015D000034
:1072300039620000508AFF1F115D0000088BFF1F9C
:107240009C8EFF1F91620000215D0000E96200003A
:10725000315D0000416300002C8AFF1FC089FF1FC1
:10726000C08FFF1F9D690000515D0000CD690000C7
:10727000615D000031780000415D0000F0B5461C02
:1072800083B00D460127032336B22AB204463146A5
:107290008DE888002448ADB204F030F80C23AA1C15
:1072A00012B200930197052321B21F4804F026F87B
:1072B0001E4A1F4B12881B68BA422AD023D3022AC7
:1072C00010D11C4CA3F6CA0384FB03241C44DB1717
:1072D000C3EB24140A2CA8BF0A2424EAE474A2B243
:1072E00023B202E000231A461C460D35AA1A0120DB
:1072F0000093019012B2314603230B4803F07CFF48
:10730000204603B0F0BD0C4CA3F6FC0384FB032421
:10731000DDE7084CA3F6980384FB03241C44DB1729
:10732000C3EBE404D6E700BFE09DFF1FC89CFF1F2E
:107330004C9DFF1F898888881F85EB512DE9F043FC
:107340008FB283B0DFF84C80BD1D461D2DB204B254
:1073500036B24FF001090AB2234631464046009545
:10736000CDF8049003F07AFF2A4633462146404682
:107370008DE8200203F072FF07F10C0200953346FE
:1073800012B22146CDF80490404603F067FF03B0E7
:10739000BDE8F083E09DFF1F2DE9F043804685B0F6
:1073A000002956D10121304804F0EEFA2F4998F80F
:1073B000062098F8083011F80290994522DA4FEA31
:1073C00089064D460C24D8F80C3027489B595F6835
:1073D00022B2002104F0D4FA384609F051F93946B6
:1073E0000246214804F066FC1F4804F079FC98F836
:1073F000083001350934AB42A4B206F1040601DDC0
:10740000422CE0D1B9F1000F13D109F106099945D9
:107410000CDA3C2301213B22039102930093019259
:1074200039233F223A21104803F0D2FF05B0BDE8CE
:10743000F0830F2301213B220391029300930192D9
:1074400039230C223A21084803F0C2FF98F808308B
:10745000DBE700213423009301913F230C220248F3
:1074600003F0CAFE9EE700BFE09DFF1FD89DFF1FEF
:1074700010B5104C0121204604F08CFA2046012161
:1074800004F082FA20463422552104F079FA20468D
:107490000222094904F00EFC20460522074904F0A7
:1074A00009FC204604F01CFC2046BDE8104003F017
:1074B00089BC00BFE09DFF1FA01D0100A41D0100AD
:1074C00070B50D46064609F0DBF800EB400084007D
:1074D000002D36D0284609F0D3F800EB40004000DC
:1074E00023185B1003F16001091A282209B217481A
:1074F000C3F1600404F044FA0121144804F044FA92
:10750000284609F0BDF829460246104804F0D2FB8F
:107510000E4804F0E5FB02210C4804F035FA21B2D4
:1075200021220A4804F02CFA304609F0A9F8314625
:107530000246064804F0BEFB0448BDE8704004F073
:10754000CFBB6410C4F16004E5E700BFE09DFF1FFE
:1075500010B50D4B1B5C51F82340237884B013B158
:10756000012004B010BD04AA01A942F8103D204634
:10757000A3699847A38A9B07F2D401A80099FFF753
:107580009FFF012004B010BDC49DFF1F2DE9F04FE7
:107590002F4DDFF8CCB0DFF8C4A0DFF8C8900FCDD6
:1075A00091B003AC0FC40FCD0FC40FCD0FC42B6827
:1075B00023600025A8462F462E4600E09846BAF8DC
:1075C000003024495BF8232028461123F9F7DCF921
:1075D00000EBC00400EB840089FB00340444C017B6
:1075E000C0EB6434C4F13C00C6F13C0207F1410138
:1075F000012600B208F1410300901BB2019612B2BD
:1076000009B2154803F02AFE08EB060305F211152E
:107610003C2B2646ADB24746D0D134226B210E48D2
:1076200004F0AEF900210C4804F0AEF90B4B1B88B6
:1076300010AA02EB830353F8344C204609F020F8DB
:1076400002460548214611B0BDE8F04F04F032BBB8
:107650000C16010024100100E09DFF1F609BFF1F1E
:10766000200E010009000280214B70B5B3F90030F3
:1076700083EAE374A4EBE374002B82B0A1B22FDBA6
:1076800068466D46012300E0134603EB8302520077
:107690009442F9DA174E91FBF3F286FB03E403FB05
:1076A0001211DB173032D3EBA40389B205F8012B9A
:1076B000F1D119462B70FFF703FF0F4B1B786BB10D
:1076C00001210E4804F060F9332274210B4804F0C4
:1076D00057F901220A49094804F0ECFA02B070BDDA
:1076E0002D238DF800300DF101056846CAE700BF73
:1076F000E49CFF1F67666666CB9CFF1FE09DFF1F33
:10770000BC21010010B5424C424882B003F04EFA51
:107710002378C3B906213F4804F036F92378012BBA
:1077200037D90A22022B11463A486BD004F028F9C7
:1077300039490322374804F0BDFA364802B0BDE8A3
:10774000104004F0CDBA354B1A7801210523002AE8
:1077500035D10191009311462E4803F0CFFD304BF7
:107760001A78002A36D005230122019200930022C4
:107770000A21284803F040FD2A4B1A78002A35D107
:1077800001210523019100931421224803F0B6FD45
:10779000C0E7254C2388092B32D9632B8CBF0A21E3
:1077A0001F210A221B4804F0EBF82188194804F035
:1077B000E7FA184802B0BDE8104004F091BA002280
:1077C000019100931146134803F016FD144B1A78EB
:1077D000002AC8D105230121019100930A210D48F7
:1077E00003F08CFD0F4B1A78002AC9D00122052323
:1077F0000192009300221421064803F0FDFC89E762
:107800003021CEE704F0BCF80322084992E700BF1C
:107810005F9EFF1FE09DFF1FB01D0100B49DFF1F75
:10782000B59DFF1F689DFF1F649DFF1FAC1D0100DC
:10783000F8B56D4D287840B96C4B1B6899425CD304
:107840006B4A012313702B70F8BD0C460026694863
:10785000664F03F0ABF904F6AC53324665483B6023
:1078600031212E7004F08CF801216248624D04F041
:1078700091F831465F4804F087F805225F495D487A
:1078800004F018FA5B4804F02BFA0C221021594836
:1078900004F076F80B225A49564804F00BFA0522F8
:1078A0005849544804F006FA524804F019FA564B65
:1078B00050481C68A4F69803C3EB031385FB03250B
:1078C0001D441021DB172022C3EB652504F058F876
:1078D00040F6CC339C4205F124054FF022014FF0D5
:1078E00004000BDCFFF7CAFC484B1C88064674B347
:1078F000012C46D0022C41D00120F8BDFFF71EFD1F
:10790000092243493B4804F0D5F92A22102139487D
:1079100004F036F83F4C374884FB0534EB17C3EBD3
:10792000A404214604F02CFA01223B49314804F01A
:10793000C1F904EB8401A5EB41012E4804F020FAC3
:10794000012236492B4804F0B5F90120F8BD34492D
:107950001022284804F0AEF9264804F0C1F92A2282
:107960001021244804F00CF83146224804F008FAAB
:1079700007222C491F4804F09DF9CBE70C222A4925
:10798000E7E70C2229491B4804F094F9194804F050
:10799000A7F92A221021174803F0F2FF31461548B3
:1079A0001C4E04F0EDF907221E49124804F082F93A
:1079B00086FB0536EB17C3EBA60631460D4804F0EF
:1079C000DFF9224614490B4804F074F906EB8601EE
:1079D000A5EB4101074804F0D3F922460F490548B9
:1079E00004F068F92046F8BD748AFF1F489EFF1F07
:1079F0005C9EFF1FE09DFF1F3B773B98B41D01007D
:107A0000BC1D0100A41D01004C9DFF1FC89CFF1F51
:107A1000C81D010067666666002501007824010024
:107A2000D41D0100E81D0100001E0100F01D010031
:107A30002DE9F041754C2278002A05460F4614BF07
:107A40004FF001084FF000084ED1714E3368CB1A49
:107A5000B3F5FA6F04D86B78A3B94046BDE8F0815E
:107A60006C4B6D486D49DFF8D0E11A70012303704B
:107A70000988237026208EF8002000F0F1FD6B7835
:107A8000002BEAD03760F9F7E7FF654A654B664996
:107A9000127828781B78097802EB4303421E03EB27
:107AA00081030E2AD9D801A151F822F09D7B000054
:107AB000697B00005B7A00009D7B00005B7A000020
:107AC0005B7A00005B7A0000517B00005B7A00006B
:107AD000037B00005B7A00005B7A00005B7A0000A9
:107AE0005B7A0000FF7A0000AF215048484E02F058
:107AF0000DFEFFF707FE002337602370ABE705F0AC
:107B0000F1FA4A4803F052F80221484803F03CFFDA
:107B10000F222321454803F033FF052244494348FF
:107B200004F0C8F8414804F0DBF81E2223213F4846
:107B300003F026FF05223F493C4804F0BBF83B48D0
:107B400004F0CEF8394803F03DF900F0ADFC84E7CD
:107B5000394D2B78012B50D9304B2620198800F055
:107B60007FFD00232B7078E7002B3FF476AF013BBD
:107B7000324A32F81330002B3FF46FAF274C3048B5
:107B800025492D4A23804FF001080023037081F816
:107B9000008082F80080FFF7B5FD5EE793B1013BFE
:107BA000264A32F8131019B31C4B254D1A4C224AA1
:107BB00019800026012326202E702370137000F0F8
:107BC0004FFD15E0154C1E4922880B7004284FF616
:107BD000FF7002F1FF310CBF012202460A440E4E33
:107BE000154D02F07F0201320121228031702B708D
:107BF000FFF788FD4FF001082FE70649064A0123E9
:107C00000020087013702370A6E700BF748AFF1F5E
:107C1000589EFF1F5C9EFF1F529BFF1F649DFF1F0E
:107C2000B49DFF1FB59DFF1F689DFF1FE09DFF1FB7
:107C3000101E0100181E01005F9EFF1F3C9BFF1FCE
:107C4000B49BFF1F2DE9F04F05468BB00F46AD48A2
:107C50000121164603F09EFEAA8812F0010440F0AE
:107C6000B080DFF8CC8298F80030002B7DD1AB7962
:107C7000A54AD15CA1B9DFF8BCA279781AF80390C3
:107C800041B339780139072900F2B780DFE811F0F4
:107C9000F1005401B5006C01B500B500B500E90074
:107CA0007C78002C00F0CA800139EC68387854F8F0
:107CB0002170FC68411EB4F80080072900F2A780FB
:107CC000DFE811F074015901A5006C01A500A500C1
:107CD000A5009F00DFF854A2DAF80020B21AB2F52E
:107CE000967F75D9894A107801281ABF0120107033
:107CF0001170874A18BF0146D05CC0EB0900C0B2C2
:107D0000FFF7E8F80124CAF80060AB889B0770D53C
:107D10007B78002B6DD0F9F79FFE7E4B7E4A7F4823
:107D20001B78127839780078022515FB02330A296E
:107D300003EB800300F04E810C295AD1002B58D060
:107D400003F11900764E774A013B0021400080B2D2
:107D500026F813100123157088F8003000F080FC1D
:107D6000714B032220461A702FE0664802F01EFF76
:107D70000121644803F008FE62482246214603F0D0
:107D8000FFFDAB88580725D42C68204608F078FC06
:107D9000214602465B4803F08DFF5A4803F0A0FFDE
:107DA000092201238DE80C0000217F23554803F0B0
:107DB00055FA00212846FFF7EFFA002388F8003033
:107DC00055E7AB683146384698470BB0BDE8F08FB1
:107DD0000846FAE72B6804A8984704A808F050FC66
:107DE00004A90246474803F065FF464803F078FFC0
:107DF000D6E720460BB0BDE8F08F00240AF80390C8
:107E000083E70021D1543846FB699847FC68A4F801
:107E10000080002725223C238DE884004121182280
:107E2000384803F0E9F9E968A879FFF791FB374A88
:107E30003E4B17701E600BB0BDE8F08F3B490A68DF
:107E4000B21AB2F5967FD4D9304F0E603E78012E2B
:107E500000F0B480E968184601233B70FFF778FB17
:107E6000B3E7304AE9791170012288F80020002434
:107E7000C4E72A7A013A4A45BFDD09F10104E4B2B8
:107E8000A145BAD0224E16F803B0CBEB0900C0B220
:107E90000021FFF71FF82B7A052BD9461BD9CBEB16
:107EA0000402042A40F3AE80A4F1040BBBF1000FDE
:107EB000C0F2B080063B5B45A8BF5B465FFA83F922
:107EC000AA791348B15C994205D000F802900121CB
:107ED0002846FFF761FAC9EB0400C0B201210B4E3E
:107EE000FEF7F8FF0021342301910093054831701B
:107EF00040230B223F21A14603F07EF90124AB79F8
:107F00007CE700BFE09DFF1F4C9EFF1F5D9EFF1F93
:107F1000D89DFF1FB49DFF1FB59DFF1F689DFF1FCC
:107F20003C9BFF1F5C9EFF1F5F9EFF1F449EFF1F29
:107F3000748AFF1FC49DFF1F0FFA89F1E868604C27
:107F400050F821602168049134785E4904980860F3
:107F5000002C71D0012C7FF450AF5B4A317A88F845
:107F600000401170002449E7B9F1000F50D009F129
:107F7000FF34E4B284E7B98A01F0040189B2002930
:107F80003FF440AF3B6A03929847039A00283FF4BE
:107F90003DAFAB79FC680021D15438E77B8A43457B
:107FA0003CD908F101081FFA88F830E73B8A4345BD
:107FB0003BD208F1FF381FFA88F828E725238DE81F
:107FC000180042483C703C231822412103F014F968
:107FD0003046FAE6002B3FF40CAF3D4A3D4E118887
:107FE000394A03F11900013B400080B226F8131012
:107FF000012388F80030157000F032FB364B204624
:108000001D70E2E6002A3FF755AF04F1FF3B4DE754
:108010004C46F3E64FF000094B4651E7BB8ADA07BE
:108020007FF5F5AEB7F81080F1E6BB8AD9077FF58A
:10803000EEAEB7F81280EAE62849C85CC0EB09004A
:1080400009F1010EC0B201214FF0340B02F803E038
:10805000FEF740FFB6681D48019440230B223F21E4
:108060000124CDF800B003F0C7F840230B223F21D4
:108070001648CDF800B0019403F040F921461348AA
:1080800003F082FC304608F0FBFAA0EB800000F120
:108090005F0109B20F220D4803F072FC304608F070
:1080A000EFFA31460246094803F004FE074803F0A0
:1080B00017FEE968A879FFF74BFAAB799EE600BF97
:1080C0009C9EFF1F449EFF1F5C9EFF1FE09DFF1FA5
:1080D000649DFF1F3C9BFF1F5F9EFF1FD89DFF1FDE
:1080E0002DE9F047DFF808926D4B99F800601B68A6
:1080F000DFF800A282B0003601934FF0030018BFF2
:108100000126019F9AF8008004F0A4FC0546042093
:1081100004F0A0FC0446052004F09CFC800040EA2A
:108120004404062004F096FC2C4364B25D4944EA02
:10813000C0000A7880F00F03DBB29A425A4A3CD062
:108140001760002259480B7003788DF800808DF875
:10815000012053B3564A12684EF66021BA1A8A4279
:1081600019D8022B59D0012B5FD0062B48D0032BF6
:1081700063D0042B69D0052B77D0072B7DD0082B3B
:1081800000F08380092B68D016B14A4802F01AFE2D
:1081900002B0BDE8F087484A484C00230121237013
:1081A00003701360938089F800103A46694644488A
:1081B000FFF748FD3043C6B2E6E71268BA1A1E2A36
:1081C0006BD99AF80020934222D0394C3D488AF866
:1081D0000030012B276082EA030207609846B1D085
:1081E000042BAFD137480068381AB0F5C87FA9D939
:1081F000354C2068381A3228A4D927601A46A1E7DE
:108200003A4669463148FFF71DFD3043C6B2BBE729
:10821000012B4FF00002E3D1E4E73A4669462C48CF
:10822000FFF710FD3043C6B2AEE73A46694629482B
:10823000FFF708FD3043C6B2A6E73A46694626482E
:10824000FFF700FD3043C6B29EE73A466946234831
:10825000FFF7F8FC3043C6B296E73A466946204835
:10826000FFF7F0FC3043C6B28EE73A4669461D4838
:10827000FFF7E8FC3043C6B286E73A4669461A483B
:10828000FFF7E0FC3043C6B27EE73A46694617483E
:10829000FFF7D8FC3043C6B276E7002252E700BFB2
:1082A0009C9EFF1F609EFF1FCC9DFF1F5C9EFF1FBB
:1082B000549EFF1FE09DFF1F4C9EFF1F5E9EFF1FF1
:1082C000241C0100649EFF1FD49DFF1F541C01004D
:1082D0007C1B0100A41A0100CC230100BC23010077
:1082E000941A0100FC1A0100601B0100C08FFF1FDF
:1082F000748AFF1FD09DFF1F28B11028044BA8BF10
:10830000102018607047024B01201860704700BFB2
:10831000689EFF1F38B50F4D2B78013B01381B02BB
:10832000C4B203F47063200443F4404343F00C03ED
:1083300000F4FE00184305F0F5FC2868013860F0F1
:108340003F00C0B204F01CFD2046BDE8384004F0F8
:1083500017BD00BF689EFF1F70B5124D2B78013B03
:108360001B0203F47063064643F4304308063204EC
:1083700000F0FE4043F00B03034302F4FE001843F9
:108380000C4605F0CFFC2868013860F04F00C0B201
:1083900004F0F6FC304604F0F3FC2046BDE87040E3
:1083A00004F0EEBC689EFF1F70B5124D2B78013BA8
:1083B0001B0203F47063064643F4104308063204BC
:1083C00000F0FE4043F00903034302F4FE001843AB
:1083D0000C4605F0A7FC2868013860F06F00C0B2B9
:1083E00004F0CEFC304604F0CBFC2046BDE87040E3
:1083F00004F0C6BC689EFF1F38B5104D2B78013BBA
:108400001B0203F47063044643F41043000443F07A
:10841000090300F4FE00184305F084FC28680138C5
:1084200060F06F00C0B204F0ABFC204604F0A8FC82
:108430000020BDE8384004F0A3BC00BF689EFF1FC9
:1084400038B50E4D2B78013B1B0203F470630446D4
:1084500043F45043000443F00D0300F4FE001843BE
:1084600005F060FC2868013860F02F00C0B204F00D
:1084700087FC2046BDE8384004F082BC689EFF1FA0
:1084800008B5002005F018FD0028FAD108BD00BF8E
:1084900008B564210720FFF75FFF7F210B20BDE8AF
:1084A0000840FFF759BF00BF10B500217B20FFF740
:1084B00053FF0024E0B2FFF79FFF0134022004F0D5
:1084C000FFFA802CF6D110BD10B504464FF4406081
:1084D00004F006FC04F05EFC2CB1102C044BA8BF89
:1084E00010241C6010BD024B01241C6010BD00BF95
:1084F000689EFF1F10B5044641F0E00004F040FC08
:1085000004F07F0004F03CFCC4F3C610BDE810404A
:1085100004F036BC38B5134D2B78044641F6FF7293
:10852000A0F50050824203F1FF33A8BF02461B02B0
:1085300002F5005203F47063100443F4604343F007
:108540000E0300F4FE005204184302F0FE421043F2
:1085500005F0E8FB296801392046C9B2BDE838407A
:10856000FFF7C8BF689EFF1F38B504460D46F020D0
:1085700004F006FC35B1254414F8010B04F000FCAE
:10858000AC42F9D1F720BDE8384004F0F9BB00BF98
:1085900000B50B4B83B00246998818680090032AF7
:1085A000ADF8041002D903B05DF804FB684606215B
:1085B0008DF80520FFF7D8FF03B05DF804FB00BF7E
:1085C0003824010000B50B4B024683B01868998827
:1085D0000090131F4C2BADF8041002D903B05DF8C6
:1085E00004FB684606218DF80520FFF7BDFF03B0A8
:1085F0005DF804FB40240100030203F4FE43C0F3D2
:10860000C6101843704700BF03784078DB0103F4BD
:108610007E5300F07F001843704700BF82B002AA6B
:10862000114642F8040D002012F8013B03F07F03CD
:10863000914243EA0020F7D102B07047003210B4F3
:1086400003884FF0010404FA01F418BF012202FA72
:1086500001F123EA04020A43028010BC704700BF04
:1086600070B5CEB20C46054603F0BCFD864203D081
:108670003146284603F0D0FD0135284603F0B2FD0F
:10868000240A844205D021462846BDE8704003F004
:10869000C3BD70BD38B5054603F0A4FD4FF000041E
:1086A00060F30704681C03F09DFD60F30F24A0B283
:1086B00038BD00BFF8B504460020FFF7EBFF002CE3
:1086C00000F049814FF4AF610220FFF7C9FF042099
:1086D0004FF47A61FFF7C4FF0B2004F0BBF90028C8
:1086E00040F038864FF496610620FFF7B9FF4FF44B
:1086F000FA610820FFF7B4FF4FF4AF610A20FFF7DB
:10870000AFFF40F6FC010C20FFF7AAFF4FF4966183
:108710002220FFF7A5FF4FF416612420FFF7A0FFEA
:108720007D212A20FFF79CFF0C210E20FFF798FFE8
:1087300001211020FFF794FF02211220FFF790FF84
:1087400000211420FFF78CFF00211620FFF788FF7F
:1087500002211820FFF784FF01211A20FFF780FF74
:1087600002211C20FFF77CFF04211E20FFF778FF69
:1087700014212020FFF774FF01212620FFF770FF4E
:1087800003212820FFF76CFF04212C20FFF768FF4E
:108790000F212E20FFF764FF00213020FFF760FF3C
:1087A0000C213220FFF75CFF00213420FFF758FF37
:1087B00000213620FFF754FF00213820FFF750FF3B
:1087C00000213A20FFF74CFF00213C20FFF748FF33
:1087D00000213E20FFF744FF00214020FFF740FF2B
:1087E00000214220FFF73CFF1F214420FFF738FF04
:1087F00013214620FFF734FF0E214820FFF730FFFA
:1088000011214A20FFF72CFF0A214C20FFF728FFF7
:1088100000214E20FFF724FF06215020FFF720FF04
:1088200002215220FFF71CFF0C215420FFF718FFF4
:1088300000215620FFF714FF00215820FFF710FFFA
:1088400001215A20FFF70CFF03215C20FFF708FFEE
:108850000A215E20FFF704FF00216020FFF700FFE0
:1088600004216220FFF7FCFE01216420FFF7F8FEDF
:1088700000216620FFF7F4FE0B216820FFF7F0FED1
:108880007F216A20FFF7ECFE00216C20FFF7E8FE55
:1088900000216E20FFF7E4FE00217020FFF7E0FECC
:1088A00000217220FFF7DCFE00217420FFF7D8FEC4
:1088B0001F217620FFF7D4FE13217820FFF7D0FE8A
:1088C0000E217A20FFF7CCFE11217C20FFF7C8FE95
:1088D0000A217E20FFF7C4FE1F218020FFF7C0FE83
:1088E00013218220FFF7BCFE0E218420FFF7B8FE83
:1088F00011218620FFF7B4FE0A218820FFF7B0FE81
:1089000000218A20FFF7ACFE01218C20FFF7A8FE92
:1089100000219620FFF7A4FE00219820FFF7A0FE7B
:1089200000219A20FFF79CFE05219C20FFF798FE6E
:1089300026210020FFF794FE0220FFF7ABFEB0F5E2
:10894000805F034616D34FF4AF610220FFF788FE25
:108950004FF4AF630EE04FF6FF7398423FF4B2AEB0
:10896000262840F003850220FFF794FEB0F5805FD3
:108970000346E8D2D24A04201380FFF78BFEB0F5FD
:10898000805F034680F0A184CE4A06201380FFF763
:1089900081FEA0F52F739BB2B3F57A6F024606D91C
:1089A00040F628210620FFF75BFE40F62822C64B42
:1089B00008201A80FFF76EFEA0F52F739BB2B3F567
:1089C0007A6F024606D940F6E4410820FFF748FED8
:1089D00040F6E442BD4B0A201A80FFF75BFEA0F58B
:1089E000FA739BB240F6AC518B42024606D94FF463
:1089F000AF610A20FFF734FE4FF4AF62B44B0C2096
:108A00001A80FFF747FEA0F5FA739BB240F6AC510F
:108A10008B42024606D940F6FC010C20FFF720FEEF
:108A200040F6FC02AB4B0E201A80FFF733FE1828ED
:108A3000034600F24384A84A10201380FFF72AFE61
:108A4000431E9BB20F2B024604D901211020FFF7D1
:108A500007FE0122A14B12201A80FFF71BFE0A28F5
:108A6000034600F224849E4A14201380FFF712FE6E
:108A70000128034604D900211420FFF7F1FD00234B
:108A8000984A16201380FFF705FE7F28034600F260
:108A90000784954A18201380FFF7FCFD042803463D
:108AA00000F2F883914A1A201380FFF7F3FD0C2897
:108AB000034600F289838E4A1C201380FFF7EAFDEB
:108AC0000428034600F27A838A4A1E201380FFF7A7
:108AD000E1FD0928034600F26B83874A20201380BA
:108AE000FFF7D8FD4628034600F25C83834A222024
:108AF0001380FFF7CFFDA0F5FA739BB240F6AC519F
:108B00008B42024606D94FF496612220FFF7A8FD5A
:108B10004FF496627A4B24201A80FFF7BBFDA0F534
:108B2000FA739BB240F6AC518B42024606D94FF421
:108B300016612420FFF794FD4FF41662714B262036
:108B40001A80FFF7A7FD7F28034600F225836E4AAF
:108B500028201380FFF79EFD0628034600F21683A7
:108B60006A4A2A201380FFF795FDA0F132039BB2D9
:108B7000B3F5967F024604D97D212A20FFF770FDC8
:108B80007D22634B2C201A80FFF784FD0C280346BE
:108B900000F2F6825F4A2E201380FFF77BFD1E282D
:108BA000034600F2E7825C4A30201380FFF772FD33
:108BB0000928034600F26883584A32201380FFF7E1
:108BC00069FD1E28034600F25983554A342013805C
:108BD000FFF760FD7F28034600F24A83514C3620A0
:108BE0002380FFF757FD7F28034600F23B833820A0
:108BF0006380FFF74FFD7F28034600F22D833A2064
:108C0000A380FFF747FD7F28034600F21F833C2027
:108C1000E380FFF73FFD7F28034600F211833E20EB
:108C20002381FFF737FD7F28034600F203834020AE
:108C30006381FFF72FFD7F28034600F2F582422073
:108C4000A381FFF727FD384D28804420FFF722FD40
:108C50003028034600F2E282344A46201380FFF7B0
:108C600019FD3028034600F2D382314C482023807E
:108C7000FFF710FD3028034600F2C4824A206380CB
:108C8000FFF708FD3028034600F2B6824C20A3808F
:108C9000FFF700FD3028034600F2A8824E20E38053
:108CA000FFF7F8FC0128034604D900214E20FFF706
:108CB000D7FC00231F4A50201380FFF7EBFC3BE05A
:108CC000E09BFF1F8C9DFF1F489DFF1F609DFF1FA6
:108CD0002A9DFF1F729BFF1F4C9BFF1FE49CFF1FE1
:108CE0001A9DFF1FD69BFF1F509BFF1FE49BFF1F7A
:108CF000909BFF1F8A9BFF1F5C9BFF1F709DFF1FA8
:108D0000DC9CFF1FD89CFF1F649DFF1F349DFF1F2D
:108D1000849DFF1F609BFF1FD09BFF1F9E9DFF1F19
:108D2000629DFF1F3C9BFF1F6C9BFF1F6E9BFF1FE5
:108D3000389DFF1F889BFF1F431E9BB20B2B0246D3
:108D400004D906215020FFF78BFC0622CD4B522080
:108D50001A80FFF79FFC0428034600F24182CA4AAA
:108D600054201380FFF796FC431E9BB21D2B024636
:108D700004D90C215420FFF773FC0C22C34B56205E
:108D80001A80FFF787FC0128034604D900215620EA
:108D9000FFF766FC0023BE4A58201380FFF77AFCD9
:108DA0007F28034600F21682BA4A5A201380FFF742
:108DB00071FC431E9BB2092B024604D901215A20A3
:108DC000FFF74EFC0122B44B5C201A80FFF762FCD7
:108DD000431E9BB2102B024604D903215C20FFF7EF
:108DE0003FFC0322AD4B5E201A80FFF753FC431E6D
:108DF0009BB21D2B024604D90A215E20FFF730FCEE
:108E00000A22A74B60201A80FFF744FC0228034681
:108E100000F2AA81A34A64201380FFF73BFC0128DB
:108E2000034604D901216420FFF71AFC01239E4A5E
:108E300062201380FFF72EFCC31E9BB2012B02465B
:108E400004D904216220FFF70BFC0422974B662013
:108E50001A80FFF71FFC7F28034600F27F81944AA7
:108E600068201380FFF716FC7F28034600F270810C
:108E7000904A6A201380FFF70DFC7F28034600F21A
:108E800061818D4A6C201380FFF704FC02280346A1
:108E900000F25281894A6E201380FFF7FBFB1928EC
:108EA000034600F24381864A70201380FFF7F2FBED
:108EB0000228034600F23481824A72201380FFF7B1
:108EC000E9FB0628034600F225817F4A74201380BF
:108ED000FFF7E0FB0428034600F2CD807B4A8A209E
:108EE0001380FFF7D7FB0A28034600F2BE80784ABA
:108EF0008C201380FFF7CEFB0428034600F2AF80DE
:108F0000744A98201380FFF7C5FB0128034604D953
:108F100000219820FFF7A4FB00236F4A9A201380BA
:108F2000FFF7B8FB0128034604D900219A20FFF778
:108F300097FB0023694A96201380FFF7ABFB0B28B1
:108F4000034600F28680664A9C201380FFF7A2FB4E
:108F5000831E9BB2032B024604D905219C20FFF7F8
:108F60007FFB05225F4B76201A80FFF793FB3028AA
:108F7000034600F2E9815C4A78201380FFF78AFB00
:108F80003028034600F2DA81584C7A202380FFF71C
:108F900081FB3028034600F2CB817C206380FFF701
:108FA00079FB3028034600F2BD817E20A380FFF7C5
:108FB00071FB3028034600F2AF818020E380FFF789
:108FC00069FB3028034600F2A181494A82201380C0
:108FD000FFF760FB3028034600F29281454C842065
:108FE0002380FFF757FB3028034600F28381862059
:108FF0006380FFF74FFB3028034600F2758188201D
:10900000A380FFF747FB302800F268812B88DFF848
:10901000FCC0394FE08003F00100DFF8F4E0374E88
:10902000ACF80000C3F340003880354D3549364A6E
:10903000C3F38000C3F3C007C3F30014AEF800000D
:109040003770C3F34010C3F380132C800880138063
:10905000F8BD00219620FFF703FB002373E70121F1
:109060008C20FFF7FDFA01234AE700218A20FFF751
:10907000F7FA00233BE700217420FFF7F1FA002301
:109080002CE700BFA089FF1F2E89FF1FA289FF1FA9
:10909000C49BFF1F669DFF1F709BFF1FA689FF1FBC
:1090A0002C89FF1FD49CFF1F309DFF1F929BFF1F29
:1090B000729DFF1FBC9BFF1F809BFF1F309BFF1FEC
:1090C000B69DFF1FC89CFF1F949DFF1F589DFF1F4B
:1090D000E69CFF1FD29CFF1FA29BFF1FC89BFF1F88
:1090E000249DFF1F629BFF1F749BFF1FB89CFF1FE7
:1090F000769BFF1FC09CFF1FA09BFF1FCB9CFF1FE9
:10910000D69CFF1F329DFF1FEC9CFF1F269DFF1F5B
:10911000D29BFF1F00217220FFF7A2FA0023D4E6A2
:1091200000217020FFF79CFA0023C5E600216E2085
:10913000FFF796FA0023B6E600216C20FFF790FABD
:109140000023A7E67F216A20FFF78AFA7F2398E6AB
:109150000B216820FFF784FA0B2389E600216620A3
:10916000FFF77EFA00237AE600216020FFF778FA05
:1091700000234FE60F212E20FFF772FA0F2312E58E
:1091800004212C20FFF76CFA042303E50321282097
:10919000FFF766FA0323E3E401212620FFF760FAD4
:1091A0000123D4E414212020FFF75AFA14239DE46C
:1091B00004211E20FFF754FA04238EE402211C2010
:1091C000FFF74EFA02237FE401211A20FFF748FA45
:1091D000012370E400215820FFF742FA0023E3E561
:1091E00002215220FFF73CFA0223B8E50A214C2065
:1091F000FFF736FA0A2351E511214A20FFF730FA2A
:10920000112343E50E214820FFF72AFA0E2335E506
:1092100013214620FFF724FA132326E51F214420BB
:10922000FFF71EFA1F2317E500214020FFF718FA69
:10923000002304E500213E20FFF712FA0023F6E4A4
:1092400000213C20FFF70CFA0023E8E400213A203B
:10925000FFF706FA0023DAE400213820FFF700FACE
:109260000023CCE400213620FFF7FAF90023BEE406
:1092700000213420FFF7F4F90023AFE40C21322061
:10928000FFF7EEF90C23A0E400213020FFF7E8F906
:10929000002391E402211820FFF7E2F9022301E400
:1092A00000211620FFF7DCF90023FFF7F2BB0221B3
:1092B0001220FFF7D5F90223FFF7D5BB0C210E20B2
:1092C000FFF7CEF90C23FFF7B6BB4FF47A61042009
:1092D000FFF7C6F94FF47A63FFF756BB88200A21DF
:1092E000FFF7BEF90A2091E611218620FFF7B8F9B1
:1092F000112384E60E218420FFF7B2F90E2376E6CF
:1093000013218220FFF7ACF9132367E61F21802089
:10931000FFF7A6F91F2358E60A217E20FFF7A0F9E0
:109320000A234AE611217C20FFF79AF911233CE633
:109330000E217A20FFF794F90E232EE613217820D0
:10934000FFF78EF913231FE61F217620FFF788F918
:109350001F2310E640F628210620FFF781F940F68A
:10936000E4410820FFF77CF9FFF7C6B917287FF61C
:10937000A9A919287FF618AA1B287FF635AA1C2848
:109380003FF44AAA1E287FF64FAA1F283FF454AA8A
:1093900020283FF46DAA21283FF476AA22283FF422
:1093A0007BAA23283FF484AA24283FF4B5AA2528C1
:1093B0007FF4BEAAFFF7B8BAF8B5AF2006F0C8FB35
:1093C000204B214A054603CB1368C5F803001A0C4D
:1093D0009E20C5F807102B80AA70FFF70DF92E46C6
:1093E000002426F80B0FA0B2FFF754F9FFF704F999
:1093F00002349E2C26F8020FF5D16C1E05F1AA0648
:109400004FF0FF3014F8013F082758400F4B40F34E
:1094100000017A1E0B4012F0FF0783EA5000F5D1DD
:10942000B442EFD1C043FFF7F9F83A46C5F8AB00B4
:10943000AF21284604F0C4FC2846BDE8F84006F0F9
:109440008FBB00BF4C240100482401002083B8EDED
:10945000F0B50E4B0E4C054693E8070085B0246826
:109460002E88AD7801AB83E80700270C1846002250
:109470000B21ADF804408DF80670ADF80C608DF846
:109480000E5004F09DFC05B0F0BD00BF5824010053
:1094900048240100F0B5124B124D1E68124F0FCD3B
:1094A00087B06C460FC495E8030044F8040B386895
:1094B0003B79CDF80D00320C262021808DF802205A
:1094C0008DF81130ADF80060FFF796F80022ADF886
:1094D0000B001221684604F073FC07B0F0BD00BF1A
:1094E0004824010064240100A41D0100002004F0B0
:1094F000E3BC00BF02F02EBE70B5124C82B0002556
:1095000040230646294620460093019580232022C9
:1095100001F072FE20222946204602F031FA204650
:10952000012102F037FA304607F0AAF83146024628
:10953000204602F0BFFB204602B0BDE8704001F0BB
:1095400041BC00BFE09DFF1FF0B5AE2983B075D9C7
:109550000546441E00F1AA064FF0FF3014F8012F13
:1095600008275040404A40F300017B1E0A4013F098
:10957000FF0782EA5000F5D1B442EFD1C043FFF7B4
:109580004DF80146D5F8AB000190019A914202D006
:10959000B2F17F2F0BD105F10B00FFF735F89E28B4
:1095A0000BD03248FFF7A8FF002003B0F0BD3048D1
:1095B000FFF7A2FF384603B0F0BD05F10D00FFF73D
:1095C00023F8262840D1002440F6AC5613E00428A6
:1095D0001AD0062821D008281FD00A2828D00C2805
:1095E00022D1A1F5FA7292B2B24201D8FFF738F84F
:1095F00002349E2C0ED004F10D002844FFF704F82D
:10960000022C0146A0B2E2D1B1F5805FEED3023464
:109610009E2CF0D1012003B0F0BDA1F52F7292B2C3
:10962000B2F57A6FE4D8E1E7222801D0242811D1DD
:10963000A1F5FA7292B2B242DAD8D7E70D48FFF735
:109640005BFF002003B0F0BD0B48FFF755FF002083
:1096500003B0F0BD2A28C9D1A1F1320292B2B2F50D
:10966000967FC5D8C2E700BF2083B8EDA8240100CB
:10967000942401007C240100BC24010003290CD99E
:1096800070B5461C82B005460C46304603222A4976
:1096900007F064F810B102B070BD70470B2C05D90B
:1096A00005222649281D07F059F840B12448FFF744
:1096B00023FF244802B0BDE87040FFF7C9BE05F1A2
:1096C0000901032201A807F099F801A803221E4905
:1096D00007F044F8D8B103221C4901A807F03EF86E
:1096E00008B301A803221A4907F038F8B0B919489D
:1096F000FFF702FFA11E89B23046FFF725FF0028C1
:10970000C9D0154802B0BDE87040FFF7F5BE134858
:10971000FFF7F2FEFFF750FE1148F3E71148FFF79D
:10972000EBFE1148C6E71148FFF7E6FE02B0BDE8C0
:109730007040FFF7AFBE00BF48240100B41D010018
:10974000D4240100E8240100EC24010014250100C8
:109750002C2501003025010044250100F0240100E2
:1097600004250100582501006C2501001825010081
:109770002DE9F043174D2B6883B081460F46904684
:10978000F3B1154E34880A1992B218461146328048
:1097900006F05CFD28603A464946204402F06CFD24
:1097A000B8F1000F09D031882868FFF767FF2868F3
:1097B00006F0D6F900232B60338003B0BDE8F083B8
:1097C000054E01930846318006F0C2F9019B2860DE
:1097D0001C46E0E7709EFF1F6C9EFF1F10B51F4CDC
:1097E0004FF4FA70FCF7AAF8204601F0DFF90022E6
:1097F0001146204602F0C4F82046012102F0CAF8C2
:109800002046002102F0C0F80B221549204602F044
:1098100051FA204602F064FA0F221249204602F063
:1098200049FA204602F05CFA0F490722204602F06E
:1098300041FA204602F054FA204601F0C3FA0B4BDD
:109840000B4A1A604FF4FA70FCF778F8FFF722FE23
:109850000848BDE81040FFF74FBE00BFE09DFF1F66
:10986000702501007C2501008C25010028A0FF1F28
:1098700071970000942501000020704790F839206E
:1098800090F83800101A704790F8383090F8392066
:109890009A4205D95A1C034480F83820187E704734
:1098A0004FF0FF30704700BF90F8383090F8392003
:1098B0009A4286BF1B18187E4FF0FF30704700BFDA
:1098C000704700BF38B50546B0F85E0090B195F816
:1098D0005D301446C3F1210294420CD805F13B00DF
:1098E0001844224602F0C8FC95F85D30234485F800
:1098F0005D30204638BD012014462871EEE700BFD8
:10990000B0F85E306BB190F85D30202B07D8C218EC
:10991000013380F85D30012082F83B10704701234D
:1099200003710020704700BF0023426980F838307F
:1099300080F8393080F85C3080F85D3080F85E3037
:1099400080F85F3006CA30B40D68046943662A4364
:1099500083660A60A370426990F861301649146802
:1099600013441D7A5B7B01EBC5051B026D6803F494
:10997000E06343F064032B6090F8623013449D7CF5
:10998000DB7D01EBC5011B02496803F4E06343F092
:1099900064030B6021685368194205D003692722CC
:1099A0005A70036904229A71036920225A7103696B
:1099B00080229A7030BC7047C830010043690CCBDC
:1099C00012681A420CD0094B99420AD9084B9942A5
:1099D000036994BF1A220D225A70036904229A71F6
:1099E0007047036927225A70F7E700BF7F1A060005
:1099F0003F420F0010B50269D378DBB2D9060446A6
:109A00003DD510215806D17038D503F0040303F07A
:109A1000FF02002B51D03D49626E00230B7084F889
:109A20005D30002A5BD0904794F85D30002B56D013
:109A30002369D0229A70236994F83B201A71236914
:109A4000012284F85C200222DA7010BD304B84F8C9
:109A500060009C424AD02F4B9C4252D094F839105F
:109A600013791F29DBB207D82848007820B1601885
:109A7000013184F8391003760223D37010BD5906E2
:109A8000C3D4917801F0100101F0FF000029DDD06E
:109A900013F001031ED194F85C1094F85D00884225
:109AA00081BF4B1C091984F85C3091F83B3013716D
:109AB0002369D0229A702269DEE7236984F839206D
:109AC000C0229A702369114A19790121117002226A
:109AD000DA7010BDC023937022691379CCE701229C
:109AE000002384F85D2084F83B30A1E7626994F894
:109AF0006130094913440322187A02F043FD2269B8
:109B0000ACE7626994F861300449F3E7749EFF1F83
:109B10000C90FF1F7890FF1F7D9B0000899B000029
:109B20000369DB7803F0200373B190F860300133F0
:109B3000DBB2012B80F860301AD9426990F86130AD
:109B40001344187A02F09ABD70B5426903F0FF051C
:109B500090F8613013440446187A02F08FFDA36E2A
:109B60005BB184F8385094F83900BDE8704018476C
:109B700090F85F30002BE0D0704770BD0148FFF7D0
:109B8000CFBF00BF0C90FF1F0148FFF7C9BF00BF48
:109B90007890FF1F2DE9F047374FDFF8E0903B68E2
:109BA000026982B006460093DDF800800021A025FE
:109BB000D3789B065BD53B680193019BC8EB0303FD
:109BC0000F2BF5D949B1102BF2D0002090703369DA
:109BD00080229A7002B0BDE8F087726996F8613011
:109BE00013440521187A02F043FF726996F8613038
:109BF0001344012193F812A0504602F039FF0924C2
:109C00000021504602F020FF2B46013BFDD10121EF
:109C1000504602F019FF2B46013BFDD1013CEFD12C
:109C2000706996F8611001444FF4A0720C7A4B7B76
:109C300009EBC4011B02496803F4E06343F06403C9
:109C40000B6096F862300344997CDB7D09EBC1011F
:109C50001B02496803F4E06343F064030B60013ABC
:109C6000FDD13269D3789B064FF00101A3D40120C6
:109C700002B0BDE8F08700BF9C9EFF1FC830010006
:109C8000F0B503691222DA700269937803F02003B9
:109C900085B004460D46002B5ED0B42393703C493A
:109CA00022690B680093009E05E00B680193019BFD
:109CB0009B1B042B42D8D37803F0200303F0FF0052
:109CC000002BF2D094F85D30002B31D04FF0000E15
:109CD0004FF0020C04EB0E0393F83B3013710B684A
:109CE0000393039F206907E09B060DD50B68029341
:109CF000029BDB1B052B28D8C378DBB203F00202E2
:109D000002F0FF06002AEFD080F803C02669F3783E
:109D1000DBB2DF0632462DD49F062BD5DB0731D4CC
:109D20000EF1010E94F85D305FFA8EFE7345D1D8C6
:109D300000201DBB002384F85E3004E0907023698E
:109D400080229A70042005B0F0BD867023698022BD
:109D500004209A7005B0F0BD03F0FF06FFF71AFF6C
:109D600010B9042005B0F0BD236984F85F60B0220B
:109D70009A7094E78023B3700420DAE72669802381
:109D8000B370D7E7BEF1000F0CBF02200320F6E747
:109D90009C9EFF1F2DE9F04106690025122780F8DF
:109DA000385080F83950F770D0F810C09CF802E0B5
:109DB0000EF0200E88B00446884615461E46BEF1B9
:109DC000000F49D0B4238CF80230784B21691A680F
:109DD0000092DDF800E006E01A6801920198CEEBEF
:109DE0000000042830D8C87800F0200000F0FF07F9
:109DF0000028F1D04FEA480242F00102D2B20A71C3
:109E00001A680292DDF808E0206906E01A680392F9
:109E10000399CEEB010105292AD8C17801F002018E
:109E200001F0FF070029F1D04FF0020C80F803C0C9
:109E30002269D17811F0110722D12DBB002E0CBF61
:109E4000A0238023937003E08F70236980229A708F
:109E5000384608B0BDE8F0810EF0FF07FFF79AFE24
:109E60000028F5D0236984F85F70B0229A70ACE7BF
:109E700087702369802238469A7008B0BDE8F08167
:109E8000802393700027E3E7012D75D0A021917006
:109E900021690A79BE4667464FF0A80C1A680492F9
:109EA000049805E01A680592059A121A052A4AD8FC
:109EB000CA7802F0020202F0FF08002AF2D0CF7046
:109EC0002169CA78D2B212F0100F08465AD1920610
:109ED00058D5013DEDB2012D49D0BEF11F0F3BD940
:109EE0000A79012DDAD11A680692069D05E01A68F2
:109EF0000792079A521B052A46D8C27802F002023E
:109F000002F0FF01002AF2D00223C3702269D37845
:109F1000DBB2D9063AD49B0634D5B023BEF11F0F6D
:109F200093703FD8226904EB0E0312791A760EF172
:109F3000010E5FFA8EFE16B1236980229A7084F8B2
:109F400039E0774684E781F80280236980229A709D
:109F5000774684F839E07BE704EB0E0291F8048041
:109F600082F818800EF1010E5FFA8EFEB9E781F8D3
:109F700002C021690846B0E7A82191702069BE4659
:109F80000279B0E7774663E78170DEE71021A0230E
:109F9000D170013BFDD12269937803F0F703774636
:109FA000937055E723691B79C5E700BF9C9EFF1F8F
:109FB0000148FFF71FBD00BF0C90FF1F0148FFF7CE
:109FC00019BD00BF7890FF1F704700BF38B5144C13
:109FD000037801225B000546204684F83B3084F874
:109FE0005E2084F85D20FFF78BFC20460021FFF700
:109FF00047FE0B4C2978012320461A46FFF7CAFE7C
:10A000000128F6D194F8383094F839209A4205D9CD
:10A01000E218013384F83830107E38BDFF2038BD97
:10A020000C90FF1F38B51B4C037801225B000546DE
:10A03000204684F83B3084F85E2084F85D20FFF7EA
:10A040005FFC20460021FFF71BFE124C29782046BA
:10A0500001230222FFF79EFE0228F6D194F8382051
:10A0600094F839108A420FD2531CDBB2A0189942DF
:10A0700084F83830007E0AD9234402321B7E84F8EB
:10A08000382040EA032038BD4FF6FF7038BD40F459
:10A090007F4038BD0C90FF1F0C2901D9002070476C
:10A0A0000231490001F0FE01FFF7BCBF70B50C4C56
:10A0B0000378164601255B00204684F83B3084F87F
:10A0C0005E5084F85D50FFF71BFC31462046FFF7D9
:10A0D00017FC29462046BDE87040FFF7D1BD00BF00
:10A0E0000C90FF1FF8B505460F4616464124214641
:10A0F0003A462846FFF7DAFF611C0234C9B23246FD
:10A100002846E4B2FFF7D2FF592CF0D1F8BD00BFCA
:10A1100038B504460D463548FFF706FC632280211A
:10A1200020462570FFF7C2FF012002F0C9FC20463F
:10A1300000225E21FFF7BAFF20465D21FFF746FFB0
:10A14000242801D0002038BD204606220C21FFF72C
:10A15000C9FF204601222B21FFF7A8FF204601223C
:10A160002C21FFF7A3FF20460E222D21FFF79EFF93
:10A17000204600222E21FFF799FF204601222F21A1
:10A18000FFF794FF204605223021FFF78FFF20467E
:10A1900001223121FFF78AFF204600223221FFF7FA
:10A1A00085FF204600223321FFF780FF2046002252
:10A1B0003421FFF77BFF204600223521FFF776FF91
:10A1C000204600225B21FFF771FF204610225C2110
:10A1D000FFF76CFF204620225D21FFF767FF204636
:10A1E0008F225E21FFF762FF012038BD0C90FF1F18
:10A1F00010B4047F4160022CC26002D010BC01F098
:10A20000D7BB836810BC184790E80C00F0B41C68FA
:10A2100059682568164F174E29432160164D174976
:10A220001760D66015611160417A154A5C180A31D1
:10A2300094F8244053F8215002EBC40149680D60A2
:10A24000017A5C1803EB8101247ECD6902EBC40125
:10A2500049680D60817A581803EB810390F830004B
:10A26000596B02EBC002F0BC53681960704700BF25
:10A2700001401F00011000380110007800001F800D
:10A28000C8300100704700BFF0B50C1EBDF8146067
:10A2900034DBB0F906701919B942C4BF3B1B1BB2BD
:10A2A000002BA6461CDD002A1146B8BFD11D02F0C6
:10A2B0000705CC10826A012007FB04E1A840012EAB
:10A2C0000A44C0B21ED00CD3022E09D1013B12FAAF
:10A2D00083F3013A12F8011F41409A421170F9D1FB
:10A2E000F0BDC043013B12FA83F3C0B2013A12F849
:10A2F000011F014093421170F9D1F0BD23441BB2FC
:10A300000024C6E7013B12FA83F3013A12F8011F59
:10A3100001439A421170F9D1F0BD00BFF8B50D1E8E
:10A320000EDB14461F46064601F03AFBA84207DD45
:10A33000002C05DB304601F037FBA04201DCF8BD04
:10A34000F8BD304601F02AFB022853D003284BD039
:10A35000012806D16540F3886C406540013B5D1BD8
:10A360002DB2012F03D02AD3022F14D0F8BD002C18
:10A370002246B6F90630B06AB8BFE21D42F3CF02FA
:10A3800002FB035504F00704435D012101FA04F4C4
:10A390001C434455F8BD002C2246B6F90630B06A7D
:10A3A000B8BFE21D42F3CF0202FB035504F00704DD
:10A3B000435D012101FA04F45C404455F8BD002CD2
:10A3C0002246B6F90630B06AB8BFE21D42F3CF02AA
:10A3D00002FB035504F00704435D012101FA04F474
:10A3E00023EA04044455F8BD3389013B591B254633
:10A3F0000CB2B6E7F18832890139013A4D1B141BC2
:10A400002DB224B2ADE700BF2DE9F041079E9DF9C2
:10A410001880089D04461F4600F0C0FF0D4B0E48F3
:10A420000E4984F83380FF22002F08BF1F4684F8AE
:10A430002F20002384F8302084F8312084F8322043
:10A440002060A665E565676261652362A3622046B8
:10A45000BDE8F0810C90FF1F20260100011001389B
:10A4600010B50446806A034B236008B105F078FB01
:10A47000204610BD20260100F8B5436ADBB190F8F4
:10A480002C200125AA4083F83B2083F85E5083F8F6
:10A490005D500446406A03680E461B6800219847D9
:10A4A000606A036831461B6898472946606ABDE8C0
:10A4B000F840FFF7E5BBC26BC56C1368046A23EA7A
:10A4C000050313604CB122684FF00043D36251631F
:10A4D000D36A002BFCDA936BF8BD836B466B0825BF
:10A4E000802410E03768426C3A4332601F68826C07
:10A4F0003A431A601A68876C013D22EA07024FEA64
:10A5000054041A6007D02142ECD13268476C22EA29
:10A5100007023260EAE7F8BD70B50446406A0D46AE
:10A5200000282BD0A16DFFF749FA002D20460CBF63
:10A53000A621A721FFF7A0FF606A20B1E16DBDE869
:10A540007040FFF73BBA216C226D0868236A024312
:10A550000A6093B1DA7A82B1D00703D5224A9969A9
:10A560001160DA7A910703D5204AD9691160DA7A45
:10A57000520702D51E4A1B6A136070BD236A002B66
:10A580002BD0D97A626DE1B172B6D97ACE0706D5F1
:10A590001848D9680668314099610160D97A8807FE
:10A5A00006D51548196906683140D9610160D97A24
:10A5B0004E0705D511485969066831401962016096
:10A5C00062B61B68D968914207D00D4818600D49E2
:10A5D000DA6042F0804018611960226C216D1368C6
:10A5E00023EA01031360A0E700E100E004E100E0DA
:10A5F00008E100E080E100E084E100E088E100E0C3
:10A6000001403F0000003F80436A2DE9F0410546CC
:10A610000E469046002B3ED090F82C100124A1400D
:10A6200083F83B1083F85E4083F85D40406A03681E
:10A6300000211B6808F1FF379847FFB2B8F1000FFF
:10A6400023D03744A046013E686A16F8011F03680C
:10A650001B6898470134B742E4B216D0202CF3D1DE
:10A660000121686AFFF70CFB95F82C206B6A5200F9
:10A6700083F83B2083F85E8083F85D80686A036816
:10A6800000211B6898470124DEE7686A0121BDE8C4
:10A69000F041FFF7F5BAC26BC16C136823EA0103FE
:10A6A00006EB080413604FF00048A6420ED02B6A58
:10A6B00016F801EB63B11A68C2F82C80C2F834E0D6
:10A6C000D36A002BFCDAA642936BF0D1BDE8F0818F
:10A6D000AB6BD5F834C008208021DCF800206F6C0B
:10A6E0001EEA010F14BF3A43BA43CCF800201A689F
:10A6F000AF6C3A431A601A68AF6C013822EA07025D
:10A700004FEA51011A60E8D1CFE700BF70B50446A7
:10A71000406A0D46002828D0A16DFFF74FF920466A
:10A720002946FFF7A9FE606A20B1E16DBDE87040DF
:10A73000FFF744B9216C226D0868236A02430A605E
:10A7400093B1DA7A82B1D00703D5234A99691160AF
:10A75000DA7A910703D5214AD9691160DA7A52076A
:10A7600002D51F4A1B6A136070BD236A002B2BD0D1
:10A77000D97A626DE1B172B6D97ACE0706D5194899
:10A78000D9680668314099610160D97A880706D591
:10A790001548196906683140D9610160D97A4E07B8
:10A7A00005D512485969066831401962016062B6E0
:10A7B0001B68D968914207D00D4818600D49DA60CE
:10A7C00042F0804018611960226C216D136823EA01
:10A7D00001031360A3E700BF00E100E004E100E033
:10A7E00008E100E080E100E084E100E088E100E0D1
:10A7F00001403F0000003F802DE9F041044686B053
:10A80000806A9DF830801E460F461546B4F9083020
:10A81000002800F04281DA1D48BF03F10E02B4F9AE
:10A820000630D21003FB02F2002105F0BDFCB4F9A2
:10A830000820202A00F39280B4F90610A34B0120CF
:10A84000203A733902EBD27201EBD1714FF0200E36
:10A85000029073208DE8014042F34F0241F34F0113
:10A86000204600F051FE606A84F82D70002800F048
:10A870004D81002D40F08A80B4F90830202B14BFA0
:10A880003D253C2584F82C50B8F1000F40F0858020
:10A8900006B394F93300002818DBC0B2012102F09E
:10A8A000E7F8012194F8330002F0CEF8012002F01D
:10A8B00007F9002194F8330002F0C6F80A2002F0EC
:10A8C000FFF8012194F8330002F0BEF8606A002816
:10A8D00000F08280A16DFFF771F804227C492046C8
:10A8E000FFF792FE217A0139C9B22046FFF7C4FD75
:10A8F000784904222046FFF787FE94F92D30012B7A
:10A9000014BF142110212046FFF7B6FD042272491E
:10A910002046FFF779FEB4F90630802B00F09280D4
:10A92000602B00F0A680D9212046FFF7A5FD94F901
:10A930002D30012B14BFF12122212046FFF79CFD71
:10A94000204606226549FFF75FFE606A50B3E16D5D
:10A95000FFF734F8012006B0BDE8F081B4F9061025
:10A960005F4B0120403A52394FF0400E029002EB0B
:10A97000D272522001EBD1718DE8014042F34F02B7
:10A9800041F34F01204600F0BFFD6CE76DB284F843
:10A990002C50B8F1000F3FF47BAFFEF7C5FF002E3F
:10A9A00094D076E7216C226D0868236A02430A601E
:10A9B00073B1DA7A62B1D00703D54A4A9969116056
:10A9C000DA7A91077CD4520702D5474A1B6A136092
:10A9D000012006B0BDE8F081236A002B2BD0D97A84
:10A9E000626DE1B172B6D97ACF0706D53F48D96812
:10A9F0000568294099610160D97A8E0706D53C48DF
:10AA0000196905682940D9610160D97A4D0705D5D2
:10AA100038485969056829401962016062B61B68A7
:10AA2000D968914207D0344818603449DA6042F05E
:10AA3000804018611960226C216D136823EA0103BC
:10AA400013604AE7B4F90830202B00F08680402BD1
:10AA50007FF469AF2A4920460322FFF7D5FD94F918
:10AA60002D30012B14BFCF219F212046FFF704FD7D
:10AA700059E7B4F90830102B7FF455AF214920462F
:10AA80000322FFF7C1FD94F92D30012B14BFAF2134
:10AA900010212046FFF7F0FC45E7DA1D48BF03F11F
:10AAA0000E02B4F90630D21003FB02F210460592F2
:10AAB00005F04EF8A06200283FF44DAF059AB3E6CA
:10AAC000114AD9691160DA7A7DE700BF7826010062
:10AAD000582801005C28010060280100642801005A
:10AAE0006C28010000E100E008E100E080E100E006
:10AAF00084E100E088E100E001403F0000003F8089
:10AB0000742601002C2B010004E100E0012194F8DF
:10AB10003100244F01F0ACFF94F83200012101F024
:10AB2000A7FF94F9312094F9323057F83220E263CC
:10AB300057F83330206A23640125E56425651A68D7
:10AB40002A431A6078B1B8F1000F3FF428AFFFF73D
:10AB50005BFB002E3FF4BAAE9BE60422124920466E
:10AB6000FFF752FDDFE6294694F82F0001F080FF41
:10AB7000294694F8300001F07BFF94F92F2094F9D6
:10AB8000303057F83220626357F833306564A5647B
:10AB90001A68A36322F001021A60002E3FF496AEF9
:10ABA00077E600BFC830010070260100B0F9082028
:10ABB000D31D48BF02F10E03B0F90620806ADB10F6
:10ABC00002FB03F2002105F0EFBA00BFF0B5002947
:10ABD000BDF814502EDBB0F90660B1422ADA002A23
:10ABE00059DBB0F9087014461C44BC42C4BFBB1A00
:10ABF0001BB2002B1EDDD2B2D408D0F828E016FB21
:10AC0000041112F00702DBB20EEB010421D0C2F1F5
:10AC10000807FAB2374F9342BF5C0CD2C3EB020C69
:10AC2000FF2646FA0CF6012D07EA06073FD005D3AA
:10AC3000022D36D0F0BD012D39D030D21EF8016082
:10AC400026EA07070EF801709342F3D3B0F9061015
:10AC50000C449A1AD2B2072A10D9022D36D0002DF0
:10AC600014BFFF26002613462670083BB0F90610D5
:10AC7000DBB2072B0C44F7D802F00702002AD9D028
:10AC80001D4B012D9B5C1DD017D3022DD2D12278F4
:10AC900053402370F0BD13441BB20022A1E7022DE4
:10ACA00025D11EF8016077400EF80170CCE71EF840
:10ACB000016037430EF80170C6E7227822EA0303E9
:10ACC0002370F0BD227813432370F0BD1146237822
:10ACD000DB4323700839B0F90630C9B207291C4498
:10ACE000F5D812F00702A5D0034B9B5CCFE73444A4
:10ACF000AFE700BF102601000026010070B4C47D3C
:10AD0000BDF80C50022C18D0032C1FD0012C0BD0F6
:10AD1000002A03DBB0F90840944201DC70BC7047A4
:10AD2000039570BCFFF7B0BAC4880395013CA41A20
:10AD30000A4621B270BCFFF749BF0689C488013EAC
:10AD4000641AB21AE41A12B221B2E1E70489039537
:10AD5000E41A641A114622B270BCFFF737BF00BF75
:10AD600070B4C57DBDF80C60022D1AD0032D12D031
:10AD7000012D03D0039670BCFFF728BFC488E41AE6
:10AD8000A41A0A4621B2002A03DBB0F90840944213
:10AD900013DC70BC70470489013C641A114622B26E
:10ADA000F1E7C48805890396013CAD1AED1A621AD1
:10ADB00011B22AB270BCFFF709BF039670BCFFF74F
:10ADC00063BA00BF2DE9F8430446406A002863D007
:10ADD000A16DFEF7F3FD052274492046FFF714FC30
:10ADE000A1790139C9B22046FFF746FBB4F9082022
:10ADF000E588A66AD31D48BF02F10E03DB10626A24
:10AE000015FB03F51FFA85F8002A7BD094F82C3047
:10AE10000125AB4082F83B3082F85E5082F85D50ED
:10AE2000606A036840211B6808F1FF379847BFB28A
:10AE3000B8F1000F23D03744A846013E606A16F8E7
:10AE4000011F03681B6898470135B742EDB216D061
:10AE5000202DF3D10121606AFEF712FF94F82C2017
:10AE6000636A520083F83B2083F85E8083F85D803C
:10AE7000606A036840211B6898470125DEE70121CD
:10AE8000606AFEF7FDFE606A002800F08D80E16DCB
:10AE9000BDE8F843FEF792BD236A002B2BD0D97A88
:10AEA000626DE1B172B6D97ACE0706D54048D9684D
:10AEB0000568294099610160D97A8D0706D53D481A
:10AEC000196905682940D9610160D97A480705D513
:10AED00039485969056829401962016062B61B68E2
:10AEE000D968914207D0354818603549DA6042F098
:10AEF000804018611960226C216D136823EA0103F8
:10AF0000136068E7E26BE36C1168276A0B4306EB9A
:10AF1000080913604FF0004E4E450DD016F801CBD6
:10AF20002FB33A68C2F82CE0C2F834C0D36A002BC1
:10AF3000FCDA4E45936BF1D1226C236D11680B4303
:10AF4000136097B1FB7A83B1D90703D51D4BBA695A
:10AF50001A60FB7A9A0703D51B4BFA691A60FB7AD1
:10AF60005B0702D5194B3A6A1A60BDE8F883A36BF8
:10AF7000D4F8348008208021D8F80020656C1CEAC1
:10AF8000010F14BF2A43AA43C8F800201A68A56C11
:10AF90002A431A601A68A56C013822EA05024FEAB2
:10AFA00051011A60E8D1B7E7276AC5E70826010012
:10AFB00080E100E084E100E088E100E001403F0042
:10AFC00000003F8000E100E004E100E008E100E073
:10AFD0002DE9F04F85B09946BDF93870BDF83CA019
:10AFE000BB1AC1EB090B002BB8BF5B42BBF1000FD2
:10AFF000B8BFCBF1000B5B450D461646009380466B
:10B0000048DC4D453A4633464CDC194613460A4661
:10B01000C5EB09019B1A89B2002B0CB2B8BF5B4289
:10B0200004EBD474BE42ACBF4FF0FF3201224D4559
:10B03000039102924FEA640429DC9BB201930DE074
:10B04000D8F80070BF69B847019BE41AA3B21CB2DC
:10B050000135002C2DB211DBA94518DB009B5B45A7
:10B060002A46534631464046EADCD8F8002053468B
:10B070009769294632464046B847E5E7029A1644A2
:10B08000039AA94502EB030436B224B2E6DA05B00E
:10B09000BDE8F08F4A462B46B94635464D45174622
:10B0A0001E46B2DD304629463E464D460746894695
:10B0B000AEE700BF10B404682469A44610BC604722
:10B0C00030B40468BDF808500295A46BA44630BCA7
:10B0D000604700BF30B40468BDF808500295E46BC7
:10B0E000A44630BC604700BF70B40468BDF90C6072
:10B0F000BDF8105003960495246CA44670BC6047BC
:10B10000704700BF10B582B0B0F90C200191016802
:10B11000009200220C6CB0F90A301146A04702B030
:10B1200010BD00BF704700BF01F003010129C175C8
:10B1300006D0032904D0C2880389428183817047E5
:10B140000289C38842818381704700BF2DE9F041A5
:10B150000568134E6F6986B0B7420446BDF830806B
:10B1600010D1013B13441BB20093CDF804800B4671
:10B17000AD6A2046A8472368DB6AB3420AD106B00D
:10B18000BDE8F081059304920391B84703A92568AF
:10B190000EC9E6E7204606B0BDE8F041184700BFFB
:10B1A00001B100002DE9F0410568124E6F6986B0CB
:10B1B000B7420446BDF830800FD1013BCDF8048082
:10B1C0000B4400921BB2AD6A2046A8472368DB6A95
:10B1D000B3420AD106B0BDE8F08105930492039111
:10B1E000B84703A925680EC9E7E7204606B0BDE8C1
:10B1F000F041184701B100002DE9F04F0568DFF874
:10B2000058B06F6985B05F450646BDF93890BDF806
:10B210003CA00C46904615D11F19BC420CDACDF863
:10B2200000A0214601342D6A4B464246304624B2E6
:10B23000A847BC423568F2DBEB6A5B4507D105B035
:10B24000BDE8F08F0393B8473568039BE4E73046C9
:10B2500005B0BDE8F04F184701B100002DE9F043FB
:10B2600087B099420546BDF93840BDF83C6025D00D
:10B27000A24212D00768DFF88080D7F81490C14549
:10B2800032D18DE850002846BC6AA0472B68DB6AA3
:10B29000434524D107B0BDE8F083994202DD08465A
:10B2A0001946034628680E96C46B01335B1A1BB21D
:10B2B0002846A44607B0BDE8F0436047A24202DD3D
:10B2C000134622461C4628680E96631C846B9B1A04
:10B2D0001BB22846A44607B0BDE8F04360472846A5
:10B2E00007B0BDE8F0431847059304920391C8479F
:10B2F00003A92F680EC9C4E701B100002DE9F04F82
:10B30000D0F800E0DFF89090DEF814B083B0CB45C1
:10B310000446BDF93080BDF834A00D4617461E46E0
:10B3200031D1CDF800A0DEF824B0294633463A46A4
:10B330002046D8472368CDF800A008F1FF323A44F0
:10B34000D3F824B0294612B233462046D8472368A2
:10B35000CDF800A02946D3F820B03A46434620460F
:10B36000D8472068CDF800A0711E29444346056ADD
:10B3700009B23A462046A8472368DB6A4B4506D106
:10B3800003B0BDE8F08FD847D4F800E0C9E7204605
:10B3900003B0BDE8F04F184701B10000F0B400243D
:10B3A00001264FF6FF75094F07600471C475C4810B
:10B3B00004824476C4618675067685824582C180A2
:10B3C000028141818281F0BC704700BF382B0100AF
:10B3D0002DE9F04F85B00668BDF84450BDF93880BE
:10B3E000CDF8008004460195D6F848B00392BDF927
:10B3F0003C60BDF9407089469A46D847236801955C
:10B40000009742465146D3F8488020463346C0470D
:10B410002068039B0E930F95856C4B463A46314648
:10B420002046AC4605B0BDE8F04F60472DE9F04F2F
:10B4300087B01746BDF9404000912546E91D0593A8
:10B4400044BF2B4603F10E010268BDF84860536902
:10B450000294C91003912B49BDF9444001968B42D7
:10B46000824645D1002C3CDD029B3C445E1EB6B2B8
:10B470004FF0000923B2049301364D46029B002B86
:10B4800028DD059B002403EB090806E0EDB22B063E
:10B4900004F1010411D4A6421CD0A1B211F0070F8F
:10B4A00023B24FEA4505F1D1002BB8BF0733DB10BB
:10B4B000013418F803502B06EDD5009BD2F818B0D4
:10B4C00019443A4609B2019B5046D847A642DAF8D9
:10B4D0000020E2D1039B01379944049B3FB2BB4259
:10B4E000CCD1D36A074A934206D107B0BDE8F08FAA
:10B4F0009847DAF80020B5E7504607B0BDE8F04FAE
:10B50000184700BF01B1000070B4BDF90C60BDF96F
:10B510001050BDF8144003960495059470BCFFF7D5
:10B5200085BF00BF2DE9F04F93B090460591C169EA
:10B530001090BDF870000790BDF874909DF878A049
:10B540000493002900F0CD800A7A0AC9894604993B
:10B550008A1AD2B203EBC203BAF1010FDA780B9266
:10B5600093F905201E8893F802B00F9293F90640D4
:10B5700079D913B2099323B20C93109B1A68A94B83
:10B580001193194653698B4240F0A6800B9B002B08
:10B5900055D01FFA88F300210D93C8462344DDF8E7
:10B5A000409006910E930F460C46BBF1000F3FD022
:10B5B000BDF818100C9B03971FFA8AF0CB1813FBE9
:10B5C00000F304900E9801440D98034409B21BB295
:10B5D0000A910893002505E00135EBB264009B4514
:10B5E000E4B222D9039B2B44590703D1731C18F8EA
:10B5F00006409EB22306EFD5099BBDF81000E9185E
:10B6000011FB00F10598BAF1010F0FFA8AF301441A
:10B610001CD0079801900093D26909B2174648469A
:10B62000089AB847D9F80020D6E7039F5F44FFB2D5
:10B63000069B0B9901330693DBB29942B5D8D36AC6
:10B64000119A934243D113B0BDE8F08F0F9B1918A4
:10B6500093690A9A29441F4609B2079B4846B8478E
:10B66000D9F80020B8E700230C93099385E70A9ADC
:10B670000D9B0132013B52B213F0FF030A920D936E
:10B680006FD1DDF81890079BDDF83C80DDF820A035
:10B690004B4517D0BAF1010F00F0C8800B9A109DEE
:10B6A000CDF804900BEB8B014FEACB030A440093D7
:10B6B0001146DEF81C405346424609B22846A047D0
:10B6C000D5F800E0DEF82C30119A9342BBD01098E8
:10B6D00013B0BDE8F04F1847109D284698472A68D8
:10B6E00054E7109A0598B2F90A308342ABDDB2F9FB
:10B6F0000C304345A7DD062313FB0A03002BA2DD14
:10B7000008EBCA03002B9EDD537E2BB9049BAF2BA5
:10B7100002D90133DBB20493109BD3F800E0414B14
:10B7200011931A46DEF81430934240F08E801FFACF
:10B7300088F30E9308339BB2BDF8142005930523BC
:10B740000D9300230A93CDF83C800FFA8AF3DDF8BD
:10B750004080CDF818900B921FFA8AFBCDF820A0FC
:10B7600099460A9ABDF810000B9C0E9D05231946B8
:10B7700011FB00232C481146C75C039702FB0B42C8
:10B7800014FA81F312B21BB209920C932C462E4686
:10B790001CE0089B0999012B2AB24B4640462DD04C
:10B7A000079F0197CDF80090DEF81CA0D047D8F88D
:10B7B00000E0039B5B0801340393059BA4B25D4446
:10B7C0005E44A342ADB2B6B23FF451AF039BD8077B
:10B7D000DFD4079B069A9342EBD0089B012B16D02F
:10B7E000069B0193CDF80090DEF81CA009994B460A
:10B7F00032B24046D047D8F800E0DAE7DEF818A0C9
:10B80000079B0C9922B2D047D8F800E0D1E7DEF8C8
:10B8100018A00C991346404622B2D047D8F800E051
:10B82000C7E700BF01B10000882B01000B99109DF4
:10B83000CDF800900531DEF8204009B242460823D9
:10B840002846A047D5F800E03CE7109C20469847E2
:10B85000D4F800E06BE700BFF0B5C36985B00446DB
:10B860002BB30A2968D00D294AD01A7A914247D3BE
:10B87000587A884244D35D688A1A05EBC205AA78D3
:10B88000002A50D0E87800284DD0207E00283AD0F9
:10B8900095F905E0B4F90E00A67DB4F90A7072447A
:10B8A00006FB0202BA4262DCB4F9102030E00A2939
:10B8B00056D00D2924D0027E002A4BD0B0F90E00BC
:10B8C000A57DB4F90A60062212FB0502B2423EDDF4
:10B8D000228AE38102EBC50212B218462282A78AAD
:10B8E000668A02950B468DE8C00001462046FFF7A8
:10B8F00019FEA37DE28903EB430302EB4303E381DB
:10B90000012005B0F0BDA67DB4F90E00B4F91020F9
:10B91000B4F814E0678A02960B468DE88040014631
:10B920002046FFF7FFFD2979E389A27D012001FB75
:10B930000233E38105B0F0BD0022C2819A7A817D95
:10B94000038A01FB02330382012005B0F0BDB4F984
:10B950001020C4E7857DB4F91020B0F90E00BEE7D1
:10B96000028A817DC38102EBC1030382C8E7002004
:10B97000E0819B7A228A03FB062212B22282C7E769
:10B98000C1810282704700BF002908BF0121817573
:10B99000704700BF81824182704700BFC07D704701
:10B9A000B0F90A00704700BFB0F90C00704700BF43
:10B9B00010B4EFF3108272B6437F33B9017F0129CF
:10B9C00007D003290FD00123437702B962B610BC18
:10B9D0007047124C2168A1B1114943610B68836122
:10B9E00008605861EFE70F4C216881B10E4943614F
:10B9F0000B688361086058610C4B4FF080511960EF
:10BA0000E1E7074B4161816120601860DBE7064B8D
:10BA10004161816120601860EEE700BF889EFF1FD2
:10BA2000849EFF1F789EFF1F7C9EFF1F04ED00E099
:10BA300070B5EFF3108272B60C4C206880B10C4EDA
:10BA400000254369236073B19D6102B962B64577F1
:10BA500083689847EFF3108272B620680028F0D10F
:10BA600002B962B670BD3360EFE700BF789EFF1F7A
:10BA70007C9EFF1FFFF7DCBF184A30B41468002C0F
:10BA800027D0036821688B420ED2CB1A0021846034
:10BA9000C1602360E06010600223037530BC704712
:10BAA00011688B42144608D3A2685B1A0360002A0F
:10BAB000F6D18260C460A060EEE7D268C2608460A4
:10BAC000E060C568CB1A0222A8602360027530BC12
:10BAD00070478460C4601060DEE700BF809EFF1F77
:10BAE000F8B5224E34682CB32368002B3AD1204F8E
:10BAF0001D4604E03468ECB12368002B32D1A36802
:10BB000003B1DD6020693360036825751B68BB42A3
:10BB100021D1037F4560022BC46020D0FFF748FF8E
:10BB20006368002BE6D023602046FFF7A5FF34684A
:10BB3000002CE1D1EFF3108372B60E4A0021106899
:10BB4000116003B962B628B18468FFF795FF2046FB
:10BB50000028F9D1F8BD224600219847E0E7836824
:10BB60009847DDE7013B2360E4E700BF809EFF1FAD
:10BB7000F1A10000909EFF1F024A13680133136079
:10BB8000FFF7AEBF9C9EFF1F704700BF0368F0B475
:10BB9000FBB1002501249D60DC601B4C1A601C4435
:10BBA000241104F144056A11032692009E60174F88
:10BBB0000679174B47F8241002F1604202F5614202
:10BBC00005F01F05012000FA05F5E6541560F0BCEC
:10BBD0007047104C236843F40003236000BF0E4BF2
:10BBE0000E4DA4F58734A4F59E7401261E602346ED
:10BBF00004609C68002CD0D01033AB420360F8D1B5
:10BC0000002303601846E2E7008FFCBFE490FF1FAB
:10BC100044E400E03C800440007003404071034075
:10BC20000168A9B10B4BF0B40B441B110A4E0B4F2A
:10BC30000B4D46F8237003F1440202F01F04012368
:10BC40005211A340002445F822308C600460F0BCFF
:10BC5000704700BF008FFCBFE490FF1F89BB00004E
:10BC600080E100E0024A034B012111601B68184784
:10BC70000C710340E490FF1F024A034B0121116045
:10BC80005B6818471C710340E490FF1F024A034B96
:10BC9000012111609B6818472C710340E490FF1F3D
:10BCA000024A034B01211160DB6818473C710340D5
:10BCB000E490FF1FF8B50E4671B17AB107461446FD
:10BCC00000253B6816F8011B1B6838469847013C65
:10BCD0000544F6D12846F8BD0846F8BD1046F8BD23
:10BCE00000B5064A036812885B6883B001A9ADF805
:10BCF00004200222984703B05DF804FB883001005D
:10BD0000F0B507468BB0002A33D0012A08BF0A22BB
:10BD100051B3212400E0F4B2B1FBF2F502FB15119E
:10BD2000C8B2092900F1300198BFC8B20AA988BF7A
:10BD30003730214488BFC0B201F8240C661E294662
:10BD4000002DE8D133B1013CE4B20AAB23442D22EB
:10BD500003F8242C3B6801AA11195B683846C4F12A
:10BD6000220298470BB0F0BD30228DF82520212407
:10BD7000E8E70368C9B21B6898470BB0F0BD00BF85
:10BD80000029BABF49422D2300230A22FFF7B8BF7A
:10BD9000374A384913681B06FCD40B6813F080033C
:10BDA000F8D172B634490A78002A5FD0334A344851
:10BDB000F0B4344C176806682568D4680C303E44EB
:10BDC000143200681268304F35442C442044024439
:10BDD000C2F34E022D4E2E482E4D2F4C42F40042FF
:10BDE0003A60376806682D682C4A24680C303E4457
:10BDF000006812682A4F35442C4420440244C2F3A0
:10BE00004E02284E2848294D294C42F400423A60FF
:10BE1000376806682D68274A24680C303E4400685D
:10BE20001268254F35442C4420440244C2F34E028C
:10BE3000224E2348234D244C42F400423A60376896
:10BE400006682D68214A24680C303E440068126858
:10BE500035442C4420440244C2F34E021C4842F4B0
:10BE6000004202600B7062B6F0BC704762B6704769
:10BE700024B0034024B00B40959EFF1F38B0034010
:10BE80003CB0034040B003402CB0034058B00340E6
:10BE90005CB0034060B0034064B003406CB003404A
:10BEA00030B0034038B00B403CB00B4040B00B40CA
:10BEB00044B00B404CB00B402CB00B4058B00B4082
:10BEC0005CB00B4060B00B4064B00B406CB00B40FA
:10BED00030B00B4030B42948294A2A4B2A4D6024FF
:10BEE000E121047011701B78284C082B30D00A2BEC
:10BEF0002748284937D00C2B0CBF35223D2212236E
:10BF00002A60236002600B60234B24491B78244A7B
:10BF1000BBB101230B601360224B23491B78234ADA
:10BF2000012B26D9042B0FD9082B1ED9102B94BF17
:10BF3000862387230B6013601D4B01221A7030BCCF
:10BF400070470B601360E7E784230B601360F3E72F
:10BF500000F58E200F490830012213232A60236048
:10BF600002600B60D0E73922F7E785230B6013608E
:10BF7000E2E780230B601360DEE700BF004007406C
:10BF800001400740F490FF1F08B003400CB003408D
:10BF900008B00B400CB00B40989EFF1F20B0034030
:10BFA00020B00B40F590FF1F24B0034024B00B409D
:10BFB000959EFF1F0C2830B417D91023984228BF34
:10BFC00018461C46104A114D1178181A8C422870D8
:10BFD00018D00F4913700B7823B10E490E4A002375
:10BFE0000B60136030BCFFF775BF0A2802D90C2321
:10BFF0001C46E7E7082802D90A231C46E2E7082383
:10C000001C46DFE730BC7047F490FF1F949EFF1F73
:10C01000959EFF1F24B0034024B00B4028282FD842
:10C02000334B2DE9F0411E5CFF2E2BD0314B1B789A
:10C03000002B2AD132062CD472B62F4D2F4C2F460E
:10C04000012326602B7062B672B623681B060CD4DF
:10C050003B781BB9F4E72B78002BF1D062B602F0E5
:10C060009BF972B623681806F5D5254B1B6800228C
:10C070002A7062B6234A107843FA00F0BDE8F081D6
:10C08000002070470020BDE8F081FFF781FE3206F6
:10C09000D2D572B61C4DDFF87C801C4C06F04007F0
:10C0A000FFB206F03F06D8F80030DFB123F01003EE
:10C0B000C8F8003001232660134A2B7062B672B6AE
:10C0C000236819060CD413781BB9ECE72B78002BE6
:10C0D000E9D062B602F060F972B623681B06F5D5A6
:10C0E0000B4BC3E743F01003C8F80030E2E700BF92
:10C0F0008C300100959EFF1F979EFF1F00B00340EC
:10C1000010B00340949EFF1F969EFF1F00B00B408F
:10C1100010B00B400CB00B400A4A0B49136843F4B3
:10C12000805313600B7843B9084BC0221A70084B38
:10C1300080F30C0000B218807047044B80221A7004
:10C14000F5E700BF2C800440989EFF1F21C00C40E3
:10C1500000C00C40F0B51B4B1B4E596818689A681C
:10C16000DB6885B06C460FC4337899071DD5174A34
:10C17000174C1378174913F0700318BF1370164A41
:10C18000164B8027177000263320032226706D4639
:10C1900008701A7072B6043C45F001052046A847A5
:10C1A00062B6237813F0700309D10D4B064901E004
:10C1B000013B02D00A78D207FAD505B0F0BD237052
:10C1C00005B0F0BDB830010001000240000002409F
:10C1D000040002400B000240070002400A00024037
:10C1E000410D0300B0F5006F0AD210B5094B1B7862
:10C1F000DB07044606D504F1A0500078C0B210BD9C
:10C2000000207047FFF7A6FF04F1A0500078C0B2ED
:10C2100010BD00BF01000240B0F5006F17D238B565
:10C220000F4B1B78DA070D46044611D504F1A050D8
:10C230000378AB420AD00B4A137813F0700318BF8F
:10C240001370074A05701378DB07FCD538BD7047BB
:10C25000FFF780FF04F1A0500378AB42EBD1F5E784
:10C26000010002400000024008B5F4F707FAF5F7B4
:10C2700007FE02F091F8FAE7844641EA000313F062
:10C2800003036DD1403A41D351F8043B40F8043BDD
:10C2900051F8043B40F8043B51F8043B40F8043BA0
:10C2A00051F8043B40F8043B51F8043B40F8043B90
:10C2B00051F8043B40F8043B51F8043B40F8043B80
:10C2C00051F8043B40F8043B51F8043B40F8043B70
:10C2D00051F8043B40F8043B51F8043B40F8043B60
:10C2E00051F8043B40F8043B51F8043B40F8043B50
:10C2F00051F8043B40F8043B51F8043B40F8043B40
:10C3000051F8043B40F8043B403ABDD2303211D3DF
:10C3100051F8043B40F8043B51F8043B40F8043B1F
:10C3200051F8043B40F8043B51F8043B40F8043B0F
:10C33000103AEDD20C3205D351F8043B40F8043BDF
:10C34000043AF9D2043208D0D2071CBF11F8013BDD
:10C3500000F8013B01D30B8803806046704700BFA3
:10C36000082A13D38B078DD010F003038AD0C3F1B2
:10C370000403D21ADB071CBF11F8013B00F8013B94
:10C3800080D331F8023B20F8023B7BE7043AD9D353
:10C39000013A11F8013B00F8013BF9D20B78037028
:10C3A0004B7843708B7883706046704708B5104CAB
:10C3B00008E0236859050DD423681A050FD42368B3
:10C3C000DB0411D423685803F3D500F08DFE2368F5
:10C3D0005905F1D502F044F823681A05EFD502F0AB
:10C3E000D5F82368DB04EDD500F0F0FCEAE700BFE8
:10C3F0003480044008B5FFF7D9FF00BF014B10227D
:10C400001A80704700200540704700BF094908B5F1
:10C410000B6830B16A461844A2F58052904202D2AD
:10C420000860184608BD03F065FB0C2303604FF05D
:10C43000FF3008BDF890FF1FFEE700BFEFF3138049
:10C4400070B9EFF310836BB9EFF305825AB94FF46B
:10C450008070EFF311832BB1984228BF18467047C4
:10C460004FF0FF3070470F2A01D81846F1E7014B13
:10C47000D05CEEE7F0E300E0F0B44D1E2E46002461
:10C4800000E00134B0FBF2F302FB1300092800F1D5
:10C4900030078ABF3730F8B2C0B206F8010F18462D
:10C4A000002BEED10A1953704CB1107815F8016FBA
:10C4B00028700133E01A834202F80169F5DB08466F
:10C4C000F0BC7047704700BF10B40F4B53F83020DA
:10C4D00092F880422CB1012369B182F8803010BCFF
:10C4E000704703EBC0035B681A6841B922F002028F
:10C4F0001A6010BC704782F8003110BC704742F0DF
:10C5000003021A6010BC7047C83001001C4A02EBDD
:10C51000C00301295B6811D004291BD052F83000F8
:10C52000002280F8802229B1022920D0032922D0BC
:10C530001A6070474FF480721A60704752F83000EA
:10C540004FF4A27280F880121A601A6822F020025A
:10C550001A60704752F830104FF4A272012081F82F
:10C5600080021A601A6842F020021A60704740F296
:10C5700003121A6070474FF481721A60704700BF4F
:10C58000C8300100212848D8F8B5042A44D8DFE88B
:10C5900002F0484B4E0345004FF410262B4B03EBA3
:10C5A000C0030D465C68216811F4E06148D0284B57
:10C5B000284A2949C3F89C2104F140422748C3F87E
:10C5C000A411A2F59221264FC3F8A0017C29254889
:10C5D000C3F8A871C3F8AC012CD9A2F594237C2B25
:10C5E0002AD9A2F596237C2B28D9A2F598237C2B57
:10C5F00029D9A2F59A227C2A27D81B4872B623682B
:10C6000023F4702343F08072C4F384011643236043
:10C6100040F82150266062B6F8BD70474FF43026CE
:10C62000BCE74FF40026B9E74FF44026B6E74FF4D5
:10C630002026B3E70D48E1E70D48DFE70D48DDE7C9
:10C64000FFF764FFB3E70C48D8E7F8BDC830010036
:10C650000082FF1FF188FF1F9988FF1FC588FF1FF9
:10C660006D88FF1F4188FF1FD491FF1FFC90FF1FA3
:10C670003491FF1F8491FF1FB491FF1F1A4B03EBEE
:10C68000C00010B4426802F14043A3F592217C2916
:10C6900023D9A3F594217C290DD9A3F596217C29D2
:10C6A0001FD9A3F598217C2919D9A3F59A237C2BAE
:10C6B00011D80E4C00E00E4C72B613680D4823F0F2
:10C6C0008773C2F3840123F4803343F080731360D3
:10C6D00044F8210062B610BC7047074CECE7074CE9
:10C6E000EAE7074CE8E700BFC8300100D491FF1F1C
:10C6F0003491FF1FC5C40000FC90FF1FB491FF1FC1
:10C700008491FF1F30B4054B054D064C00221021CB
:10C710001A602A602060196030BC704714D0034052
:10C7200004D0034000D00340282838B52ED000297B
:10C7300004464FDD5F4B1B78012505FA03F28A4260
:10C7400002D8212837D938BD0338C2B2012A3AD9D4
:10C75000202C4AD0192C48D0574A126802FB0112EB
:10C7600022FA03F31D2800F29B80DFE800F0928B91
:10C77000847D9999766F99999999999999999968D8
:10C78000615A53994C99999999999945494B1B78B4
:10C790000B2B08D90C2B1CBF0C3B19410846BDE8DC
:10C7A0003840FFF7B9BCC3F10C0399400846BDE817
:10C7B0003840FFF7B1BC2946FFF786FE2946BDE8A1
:10C7C0003840FFF7A3BE3D4A126802FB011222FA6D
:10C7D00003F3C7E72128B6D80021FFF775FE2046EE
:10C7E0000121BDE83840FFF791BE354A126802FBCF
:10C7F000011222FA03F3B5E73249334A0B604FF4D2
:10C800005173136038BD3149314A0B604FF4517395
:10C81000136038BD2F49304A0B6040F24443136027
:10C8200038BD2E492E4A0B6040F24443136038BD98
:10C830002C492D4A0B6040F24443136038BD2B490C
:10C840002B4A0B6040F24443136038BD29492A4A01
:10C850000B6040F24443136038BD2849284A0B60FE
:10C8600040F24443136038BD2649274A0B6040F22A
:10C870004443136038BD2549254A0B6040F24443C8
:10C88000136038BD2349244A0B604FF45173136081
:10C8900038BD2249224A0B604FF45173136038BDF2
:10C8A000212C3FF650AF7F29D4BF00210121204623
:10C8B00093E700BFDC91FF1F08800340089003400E
:10C8C00008800B4010800B4048A0044018800B40AB
:10C8D0004CA004401880034008B00440108003407E
:10C8E00004B004404080034018C004403880034036
:10C8F00014C004402880034010B00440208003404E
:10C900000CB004403080034010C004404880034015
:10C910001CC0044018900340349004401090034021
:10C920003090044038B1102828BF1020044AC3B208
:10C93000107813707047024A012310781370704703
:10C94000DC91FF1F2DE9F8430E4680463249334DF6
:10C95000304603F055F847F6122300281ABF1D464B
:10C960004FF002094FF00109002425FA04F002F00B
:10C9700051FE4FF05E51074602F0A4FE01463046DC
:10C9800003F052F830B90134072CEED1E80902F077
:10C9900041FE07463146384602F048FF4FF07C51D1
:10C9A00002F086FD03F07AF84FF6FF729042A8F18C
:10C9B000030328BF1046012B29D9B8F1170F17D848
:10C9C000174B23FA08F303F0010383F0010223B9A4
:10C9D000B8F1190F0FD0BDE8F883124B124D13496F
:10C9E0001A6044EAC9042A6008601C60BDE8F88344
:10C9F000B8F1200FECD10E4B0E4D0F49002244EA46
:10CA0000C9041A602A6008601C60BDE8F8830B4BFB
:10CA10000B4D0C49F2E700BF001BB740006CDC0275
:10CA20006006F0000080034004800340088003405B
:10CA300000800B4004800B4008800B4000900340B6
:10CA40000490034008900340212801D8FFF73CBD23
:10CA5000704700BF212806D8044B53F8303093F8B4
:10CA60000002C0B270470020704700BFC83001000C
:10CA7000212801D8FFF74ABD704700BF72B60C49A4
:10CA80000C4B0D4A1B680868126862B6520102D549
:10CA9000322B88BF01300949C3F5BB334FF47A729A
:10CAA000FF33A1FB031302FB00F000EB9310704770
:10CAB0009C9EFF1F18E000E004ED00E0ABAAAAAACC
:10CAC0002DE9F843054672B6204F214B214A1B68D9
:10CAD0003C68126862B6520102D5322B88BF01341D
:10CAE00095B3C3F5BB331C4EDFF86490DFF8648068
:10CAF000FF334FF47A72A6FB031302FB04F404EB3A
:10CB0000931472B6D9F800103A68D8F800E062B60B
:10CB1000C1F5BB33FF33A6FB03031EF0806FC4EBEC
:10CB200093134FF47A7002D0322988BF013200FB90
:10CB30000233B3F57A7F04D3013D05D004F57A744E
:10CB4000DFE701F029FCDCE7BDE8F8839C9EFF1FCE
:10CB500018E000E004ED00E0ABAAAAAAF8B52D4B5E
:10CB60002D49DFF8D0E0DFF8D0C02C4E2C4D2D4CF5
:10CB70002D4A2E4F4FF4000018604FF0807018605F
:10CB80004FF0007018604FF0806018604FF0006048
:10CB900018600020086028234BF6FF71CCF80010C5
:10CBA000CEF80030336013602B6023603B60B362CB
:10CBB0009362092245F8242CC4F8D80F05F57F6547
:10CBC000C7F8D41F07F5FF2707F5FA67C6F8F83F3F
:10CBD0002B6006F5FF26C4F8D42F05F5FD2504F5D6
:10CBE000FF24386006F2F4761148316005F5FF65E0
:10CBF00004F5FD642B6023600260FFF76BF91920D8
:10CC0000FFF75EFF00F0B6FF40F21310BDE8F840FA
:10CC1000FFF756BF08E100E00480034014800340A2
:10CC2000248003402C8003401C8003403480034058
:10CC300000800B400C800340088003402DE9F84F32
:10CC4000214B1B6807460BB101221A70DFF8889050
:10CC50001E4D99F80040DFF884801D4E0134272CCA
:10CC60008ABF4FF0000A5FFA84FA5446AB462B782D
:10CC7000A34216D1FFF7E2FB40281FDC33791B06E5
:10CC8000F5D59BF800300133272B86BF00221346D1
:10CC9000DAB218F80330DBB2F3712A702B78A342B2
:10CCA000E8D00C490A4BFFB208F804700120AC220E
:10CCB000087089F800A0DA70BDE8F88FFF28D6DD8B
:10CCC00001F06AFBD3E700BF149FFF1F119FFF1FF6
:10CCD00000C00640109FFF1F189FFF1FA89EFF1F48
:10CCE0001C4BDFF894C01A681B49F0B542F480521F
:10CCF0001A4D1A60DFF884E0194F1A4E1A4C0023BF
:10CD00008CF800304FF451722B701F2840F213350D
:10CD10008EF800303B70337025600A6012D81946D7
:10CD20000124124A124D11701248547000212C2710
:10CD3000402693724FF4003491701174D7702E70A6
:10CD40000460F0BDC0F34431C0F3471400F01F038A
:10CD5000E7E700BF348004400CC00440A59EFF1FDD
:10CD6000119FFF1F109FFF1F08C0044000C0064016
:10CD700031E400E004E100E0A49EFF1F189FFF1FC4
:10CD8000034B1B68DB0401D5FFF758BF704700BF9A
:10CD90003480044010B5044C237823B101F0FCFA30
:10CDA0002378002BFAD110BD109FFF1F054A064BB8
:10CDB00010781B78C0B2DBB2984238BF4030C01A3E
:10CDC000704700BFA49EFF1FA59EFF1F30B42B4BD2
:10CDD0001A7994061FD52A48DA790378294901334C
:10CDE0003F2B0978C8BF00238B42D2B203D0264C18
:10CDF000D9B2E2540170254A116861B1244A12780F
:10CE0000D2B2934236BFC2F140029B1A9B18272B25
:10CE1000C4BF01230B70194AD378DBB2180611D4B2
:10CE20005A060DD5154B1B795B0609D5194B1A49C6
:10CE30001B6800220A7003B11A70104B2C22DA70A2
:10CE400030BC704711790906EAD5144910480C78AE
:10CE50000178C9B28C420DD04A1C272A84BF002118
:10CE60000A460F4D054C98BFD1B2AA5CD2B2E2710E
:10CE70000170D5E76C21D170D2E700BF00C0064039
:10CE8000A49EFF1FA59EFF1FD09EFF1FA09EFF1FF9
:10CE9000119FFF1F149FFF1F109FFF1F189FFF1F51
:10CEA000A89EFF1F21282FD8184B195CFF292BD0D3
:10CEB000174B184ADFF870C003EBC000F0B54368A9
:10CEC000DFF868E0144F154D154E00241C60DEF8A5
:10CED0000030012043F020038840CEF80030146079
:10CEE0004FF4A07338602E60C2F800C0013BFDD142
:10CEF00013689B05FCD42023013BFDD1094B09B2EB
:10CF000033F8110080B2F0BD00207047D831010025
:10CF1000C830010000500440085004400450044050
:10CF2000000002030051044080014A0038800440A0
:10CF3000431E032B14D872B60A4951F8230068B176
:10CF400070B4094C058834F81320466841F8236012
:10CF5000521B24F8132062B670BC704762B670474B
:10CF600000207047749FFF1FB8A1FF1F01380328DE
:10CF70000BD872B6074B53F8203043B100205B68E2
:10CF80000130002BFBD162B6704700207047184675
:10CF9000F9E700BFC89FFF1F30B472B62B4A137861
:10CFA0001D0706D52A4B196A002936D0996A00292F
:10CFB00041D053781C0706D5254B196C00293ED06B
:10CFC000996C002939D09378190705D5204B196E33
:10CFD000002936D0996E89B1D3781B0707D51C4B31
:10CFE000D3F880207AB3D3F8882011213AB162B601
:10CFF000184B00221A7030BC00F04ABE0D21154CAF
:10D00000154D227843F8315003EBC1030830013A43
:10D010005860227062B630BC704704220D4C0F4D30
:10D02000217843F8325003EBC20308304A1E58609F
:10D03000227062B6EFE70521E1E70921DFE7082268
:10D04000ECE70C22EAE71022E8E700BFFC31010020
:10D050000080FF1FF19FFF1FC800400088004000B4
:10D06000431E032B1DD81B4A400140F0100030B472
:10D07000104472B6184CE25C032A1BD8DFE802F0B9
:10D080000212151703220D88E25410F0080F14BF86
:10D09000C823882343EA054308310360416062B630
:10D0A00030BC704708300222EDE70522EBE708307C
:10D0B0000422E8E7094A52F8230038B1084A52F836
:10D0C0002300416042F8231062B6E9E742F82310DA
:10D0D000034AF7E70080FF1F00A0FF1FC89FFF1F44
:10D0E000D89FFF1F00BE70472DE9F04FDFF818B33F
:10D0F000DFF818A387B044E0AD4F4FEA930807EB81
:10D10000C809013ED9F8042003F00803F6B2A2F1E1
:10D11000080003F0FF04002B40F0018157F838307D
:10D120001B0C99B222F8081C002B00F0EF80A14BD9
:10D1300022F8064C42F8044C53F82620002A00F04E
:10D14000CF819D4D55F8263058609C4C45F82600FF
:10D1500034F81630194424F8161000F079FD002830
:10D1600000F0C281964A974B19F0080F00F10800B1
:10D1700018BF1346C9F8040047F8383008238BF865
:10D1800000309BF80040E4B265071CD58E4B1B783D
:10D19000B3B18E490A7802F0FF0322B1013BDBB242
:10D1A0000B7003B900BE8A490A7802F0FF032AB166
:10D1B000013BDBB20B70002B00F0688100F066FED3
:10D1C00004238BF8003004F0080303F0FF02002B67
:10D1D00000F0C9809AF80030DBB21E098CD19A08A1
:10D1E000DFF8CC9159F8321009EBC200C1F383018A
:10D1F000013940680C2900F28580DFE801F07A7A75
:10D200008383838383834683838307000168714D0F
:10D210004068714F714E6860296088B240F2816148
:10D220000024674B49F832304FF0010E88423C60D1
:10D23000C9F81040C9F8184086F800E05C4A00F2CE
:10D24000E780B0F5D06F80F01B82B0F5817F00F0F1
:10D25000D98100F26981802800F02A82822840F07A
:10D26000D781A98801F07F01042900F2D1815C48AF
:10D270005C4A890008441470547001788C0740F1AE
:10D28000608382F800E0022173E1534F3A682AB3C9
:10D29000554B524E554819883478057840298E46AA
:10D2A00045F0020828BF4FF0400E002C84F0010426
:10D2B0003470CEEB01010CBF8824C82409EBC806EA
:10D2C00089B285F0010544EA0E447260198049F87C
:10D2D000384072440570002965D03A603D4B1A8889
:10D2E000B2F5A06F0ED100219A785970404B1A7098
:10D2F00008E038493F4C0D68A54200F0988030495D
:10D3000049F832103C4A0123137037E72C4A2D4B61
:10D3100019F0080F18BF134647F838302EE700F011
:10D32000B7FC364A364952F82630002B00F0E3802D
:10D3300058688C5D42F8260003F10802C9F8042001
:10D34000032C05D8DFE804F02C02292602228A5596
:10D350001A8819F0080F0CBF8823C82343EA024338
:10D3600047F838300AE7E00700F19380210600F122
:10D37000D180A20706D5234A234913780220DBB2C5
:10D3800013700870E30602D51F4B10221A7007B005
:10D39000BDE8F08F04228A55DAE705228A55D7E7DF
:10D3A00003228A55D4E7BEF1400F18BF002294E74C
:10D3B0000080FF1F749FFF1F209FFF1FB8A1FF1F4A
:10D3C000C800400088004000FC9FFF1F859FFF1F92
:10D3D00070A0FF1FE89FFF1F1C9FFF1F849FFF1F60
:10D3E000C0200740F49FFF1F309FFF1FF09FFF1FCB
:10D3F000982007402109000394200740C89FFF1F81
:10D4000000A0FF1F88200740802007409020074091
:10D41000B0F5106F00F07C8140F2A38040F621123D
:10D42000904240F07B82A54A012313706AE74C6862
:10D43000A3498C427FF463AF0178A9297FF45FAFE1
:10D44000417845297FF45BAF8178C2297FF457AFDB
:10D45000C1786B297FF453AF9A489B4E017834789A
:10D4600081F00105002C41F0020105700CBF8820FD
:10D47000C82084F0010449F8310009EBC101934848
:10D480003470002505244D60047038E700F064FF17
:10D4900094E68F4B89488B491A614FF0020E80F851
:10D4A00000E08C4F0A708C49196099608B4E8C4D4E
:10D4B0008C4C9A610D213970FF213170DFF84CE2FC
:10D4C00029702270884D894A8EF800109F27012408
:10D4D00006F8047C5D600470DA6007B0BDE8F08F88
:10D4E00043F82600824D30E6824A47F83800137828
:10D4F0000133137042E68B5D032B00F2BA8001A268
:10D5000052F823F07DD100007DD100005DD50000F0
:10D5100057D500006F49724B80220D2008701A7099
:10D52000A2077FF52FAF26E740F20232904240F08B
:10D53000ED81AA8802F07F02042A69D86D88002D47
:10D5400066D16449CDF804E0920011440A7842F0B3
:10D5500002020A70C1E101238B550FE600238B55AF
:10D560000CE6B0F5086F53D16349644A097811702D
:10D570007146ED888D4280F0E88252480478402D53
:10D58000AE4644F0020C28BF4FF0400E02EB0E03F3
:10D5900009EBCC01029301234A604FEA0E48CEEB1F
:10D5A000050101930025C82242EA080384F0010224
:10D5B00049F83C3035700270DFF814C1424BDFF897
:10D5C000048149BBBEF1400F7FF42DAF42F0020C45
:10D5D00009EBCC03029ADFF8F8E05A608DBB0D042A
:10D5E00045F088059DF804304EF83C500A443370ED
:10D5F0000470134640297FF416AF0021404A3B6077
:10D60000118010E7AA8802F07F02042A40F28B8181
:10D61000304A0F23137006E74029D7D942F002029F
:10D620000CEBC200029E4660BDB19DF80450354827
:10D630001D703346403988F8004040334CF83200C2
:10D64000DCE79DF8043033700D04029B047045F054
:10D65000C8050B444EF83C50CCE79DF804501D70B3
:10D66000029B1D4888F80040403940334CF8320096
:10D67000C4E719F0080F0CBF022303238B557DE587
:10D6800021494A68002AC3D06C88B5F804E003E059
:10D690000C314A68002ABBD00B88A342F8D14B88D2
:10D6A0007345F5D1240A032C0CBF1178098960E772
:10D6B000124A0221147054705BE700BF94200740A7
:10D6C00001000400F09FFF1F849FFF1F859FFF1F25
:10D6D0000080FF1FC02007408800400088200740CE
:10D6E0008020074098200740349FFF1F889FFF1F1E
:10D6F000209FFF1FF19FFF1FFC9FFF1FF49FFF1F35
:10D70000309FFF1FC8004000003201008C200740FE
:10D71000B248116AAC7804700C0600F19881D9F80F
:10D720002820AF49100600F1DB81D9F83020AC4940
:10D73000120600F1D081D9F83820A949130600F16A
:10D74000C581D9F84020A649150600F1BA81D9F85B
:10D750004820A349140600F1AF81D9F85020A04910
:10D76000100600F1A481D9F858209D49120600F155
:10D770009981D9F860209A49130600F18E81D9F871
:10D7800068209749150600F18381D9F870209449E3
:10D79000140600F17881D9F878209149100600F13B
:10D7A0006D81D9F880208E49120600F16181D9F887
:10D7B00088208B49130600F15581D9F890208849BB
:10D7C000150600F14981D9F898208549140600F121
:10D7D000FF808448844A854901908548854D864C60
:10D7E000049700230596029580460F4616461D466F
:10D7F0000394306828B1446800F04AFA2046002CAF
:10D80000F9D100233360029B38681A46002342F89E
:10D81000253028B1446800F03BFA2046002CF9D1AD
:10D8200000223A60019A98F800301146002241F82F
:10D83000042B039A0191023B4FF0000122F81510CE
:10D84000032B07D8DFE803F05D025D024FF0010310
:10D8500088F800300135042D06F1040607F10407AD
:10D8600008F10108C5D1654C654D2278654B049FD0
:10D87000059E0021100729701A7000F192806249FC
:10D8800062780A700021C9F83010C9F83810110701
:10D89000DFF84C816ED4A2785C49DFF844810A70CD
:10D8A00000211207C9F85010C9F858104BD4E2787B
:10D8B00057494B4C0A7013074FF00001C9F870101C
:10D8C000C9F8781000F1AE8033780193002283F01C
:10D8D0000105C9F89020C9F89820002102918846D6
:10D8E0008E460A464B48047844F0020C09EBCC0300
:10D8F0000393019B002B039B5A600CBF8822C82214
:10D9000052E64FF0000388F80030A3E7B0F5A06FAF
:10D910007FF47EAE012300250193DEE740F621224D
:10D920009042F7D074E66D88002D7FF471AE3A49CD
:10D93000CDF804E0920011440A7822F002020A7045
:10D94000CBE7022115E600F083F9002800F0EB8018
:10D950000830324AC8F86400C8F8602000F078F94E
:10D96000002800F0DA8008302D4AC9F86C00C9F8A8
:10D9700068209CE700F06CF9002800F0E080083097
:10D98000264AC8F84400C8F8402000F061F9002891
:10D9900000F0CF800830224AC9F84C00C9F848206E
:10D9A00079E700F055F9002800F0A58008301B4AFF
:10D9B000C9F82400C9F8202000F04AF9002800F036
:10D9C00094800830164AC9F82C00C9F8282056E778
:10D9D000D1F89C00083800F05BF9FAE6FC9FFF1FC5
:10D9E0000080FF1FD89FFF1F749FFF1FC89FFF1F4E
:10D9F00000A0FF1F209FFF1FB8A1FF1FFC310100E7
:10DA0000F19FFF1FC4200740C8200740CC200740DB
:10DA1000D0200740F09FFF1FC02007408800400033
:10DA2000C800400000F014F9002870D008304F4AB8
:10DA3000C4F88400C4F8802000F00AF9002860D0FF
:10DA400008304B4AC9F88C00C9F888203CE7506A76
:10DA5000083800F01DF962E6D1F89400083800F0AB
:10DA600017F9B0E6D1F88C00083800F011F9A4E6F7
:10DA7000D1F88400083800F00BF998E6C86F083830
:10DA800000F006F98DE6486F083800F001F982E6EB
:10DA9000C86E083800F0FCF877E6486E083800F0E9
:10DAA000F7F86CE6C86D083800F0F2F861E6486DEA
:10DAB000083800F0EDF856E6C86C083800F0E8F8D1
:10DAC0004BE6486C083800F0E3F840E6C86B0838CD
:10DAD00000F0DEF835E6486B083800F0D9F82AE6A1
:10DAE000C86A083800F0D4F81FE62A78C9F8280078
:10DAF00001322A70C3E62A78C9F8200001322A7060
:10DB00005AE72A78C9F8880001322A70DCE62A78B8
:10DB1000C4F8800001322A708EE72A78C9F86800BC
:10DB200001322A70C3E62A78C8F8600001322A70F0
:10DB300014E72A78C9F8480001322A70ABE62A783F
:10DB4000C8F8400001322A701FE740298E4628BFDE
:10DB50004FF0400E02EB0E0302930123CEEB0101C6
:10DB60004FEA0E4800250193BCE600BF8800400044
:10DB7000C8004000F8B500F08FFD294B29482A4C19
:10DB80002A4F2B4DDFF8BCC0DFF8BCE0294E002245
:10DB90001A605A609A60DA601A615A619A61DA61B1
:10DBA0001A625A629A62DA621A635A639A63DA6391
:10DBB0001A645A649A64DA641A655A659A65DA6571
:10DBC0001A665A669A66DA661A675A679A67DA6751
:10DBD000C3F880200168C3F8842041F480210160EB
:10DBE000C3F307212170C3F30740134938701B0E9C
:10DBF0002B70FF238CF80030104D8EF80030104849
:10DC00000B700123337084F8642070264FF4007485
:10DC1000102207F82C3C2E70046081F8F820F8BD23
:10DC20000080FF1F348004409C200740B020074044
:10DC3000B4200740942007401020074049E400E04A
:10DC400008E100E08020074088200740704700BFBF
:10DC500072B60D480268B2FA82F30F2B10DC4FF057
:10DC60000041D94022EA0102026062B6074803EB94
:10DC7000C303DB00C2180021C15010465160704739
:10DC800062B60020704700BFE091FF1FBC83FF1FFA
:10DC90000D4B0E4AC31AA2FB03231B090F2B0CD8F2
:10DCA0000B4A127852B972B60A484FF00041026826
:10DCB00021FA03F31A43026062B67047064A1278EB
:10DCC000002AF0D0FFF768B9BC83FF1F398EE33814
:10DCD000F19FFF1FE091FF1FFC9FFF1F38B50E4B08
:10DCE0000E4C1B68218805468BB1B1F5917F05D29A
:10DCF0000B4A4B1C55549BB2238038BD0022084868
:10DD000098470021064A55540123238038BDB1F5B8
:10DD1000917FEDD338BD00BF28A0FF1FC2A1FF1F18
:10DD2000C8A1FF1F2DE9F843214E224F316801237E
:10DD300080463B70B1B1204D4B8801EB830201332B
:10DD400000240F2BC2F808802C7004D84B800023CD
:10DD50003B70BDE8F88340230B800320FFF780F978
:10DD60003460F4E7DFF8549099F80030002BF0D0DD
:10DD7000114D45F6215408E0013C12D02B7883B9AF
:10DD800000F00AFB99F800307BB10320FFF7EEF8B2
:10DD90000528F1D8FFF75CFF014630600028EBD082
:10DDA000CAE701232B70BDE8F883BDE8F88300BF04
:10DDB00044A0FF1F18A0FF1F48A0FF1FFC9FFF1FCC
:10DDC0001201F8B5D5B2A1B3012943D04378044676
:10DDD00000781B0643EA004040F4704045F004061A
:10DDE0008F1E3043FFF79EFF022F04F1020314D968
:10DDF000053414F8023C14F8032C14F8010C1B042D
:10DE000043EA0223334343EA0060033FFFF78AFFFC
:10DE1000022F234604F10304EBD8022F23D0012F55
:10DE20000DD045F4774040F00500BDE8F840FFF71D
:10DE300079BF14482843BDE8F840FFF773BF18784E
:10DE400045F4770545F0060545EA0020BDE8F840B1
:10DE5000FFF768BF03780C4845EA03452843BDE84F
:10DE6000F840FFF75FBF1A78587845F0774545F0DE
:10DE7000070545EA022545EA0040BDE8F840FFF7FE
:10DE800051BF00BF06F0F70007F000F738B5084BA8
:10DE90001C7824B9074D296809B14B8803B938BDEE
:10DEA0009B000B800320FFF7DBF82C6038BD00BF20
:10DEB00018A0FF1F44A0FF1F2DE9F041AD4E3368AD
:10DEC0000746002B00F092801D885A88910803EBCA
:10DED00081010432AA428C6842D25A8004F00F06B3
:10DEE0004FEA1428A449A6F1080208F00F00C4F371
:10DEF0000313062A00F101050B701AD9B31E012B7A
:10DF00005FFA88F04ED9052E48D0042E00F0A48187
:10DF1000731F022B7FD90F2E0ED1F72842D8F0287D
:10DF200002D0964B1B883BB1FFF7D8FE0020BDE81E
:10DF3000F08127B1BD4202D00020BDE8F081082E5B
:10DF4000C4F3033300F08780092E11D00A2E40F06D
:10DF500094800A2BF0D18A4B8A4A1B68A02181E069
:10DF60001846FFF795FE0420FEF7E2FF3060B5E7A4
:10DF7000092BE1D1270E00F07B81834B814A1B687E
:10DF80009021C4F307461170EDB2FCB2002B00F0F3
:10DF90009D80224631462846984797E0F02843D98D
:10DFA000F72841D0F1380E28C6D801A353F820F045
:10DFB00067E100004BE1000039E1000039DF0000BB
:10DFC00039DF00002BE1000039DF00000BE2000028
:10DFD00039DF0000D5E10000EFE1000013E10000AF
:10DFE00039DF0000FBE00000DFE00000674B1B783A
:10DFF000002BA1D00420FEF79BFF034630600028D1
:10E000009AD00588002D7FF460AFFFF741FE3560A0
:10E010002846BDE8F081FFF761FEC4F30740FFF733
:10E020005DFE072E02D1200EFFF758FE534B584AD3
:10E03000198858481468584D524A017000270E0A32
:10E04000F0201F802E7010700CB301225348A0479F
:10E050000120BDE8F081082B7FF46EAF504B494A98
:10E060001B688021C4F307461170EDB2240E6BB318
:10E07000284622463146984728E00B2E11D10B2B1B
:10E080007FF45AAF474B3F4A1B68B021EAE7464B43
:10E090001B68002B00F0FB80404898470120BDE83A
:10E0A000F0810C2E40F000810C2B7FF445AF3F4BEC
:10E0B000344A1B68C0211170EDB2C4F30746002B2F
:10E0C00000F0C88028463146240E98473849314A26
:10E0D000314B0D7016701C700120BDE8F081354B7E
:10E0E0001B68002B00F0D6809847C4F30746254BE9
:10E0F000EDB2240E83F80080E8E72F4B1B68002B5D
:10E10000F2D12E4B1B68A3B1FE209847C4F30746FB
:10E11000EDE72B4B1B68002BE6D1284B1B6843B166
:10E12000FC209847C4F30746E1E7264B1B68002B09
:10E13000DAD1C4F30746DAE7234B1B68C4F307467A
:10E14000002BD4D030469847D1E7204B1A68002ADC
:10E15000EFD0260C630C06F07F0003F47E531843C7
:10E16000F6B29047C3E71A4B1B68C4F30746002B6F
:10E17000E8D1BCE750A0FF1FC6A1FF1FC2A1FF1F2F
:10E180002CA0FF1FC0A1FF1F60A0FF1FFC9FFF1F4F
:10E1900028A0FF1FC4A1FF1FC5A1FF1FC8A1FF1F0B
:10E1A00058A0FF1F5CA0FF1F40A0FF1F1CA0FF1F67
:10E1B000C7A1FF1F08A0FF1F0CA0FF1F10A0FF1F7B
:10E1C0004CA0FF1F3CA0FF1F54A0FF1F24A0FF1F57
:10E1D00038A0FF1F3F4B1B68002B85D13E4B1B68AF
:10E1E000002BA6D0FA209847C4F307467FE73B4BA5
:10E1F0001B68002B7FF478AF374B1B68002B98D03F
:10E20000FB209847C4F3074671E7354B1B68002B8A
:10E210007FF46AAF304B1B68002B8AD0F8209847F8
:10E22000C4F3074663E70E2B7FF486AE2D4A2E4BD0
:10E230001268E0211970002A47D0260C610C06F004
:10E240007F0301F47E511943EDB2A1F50051284638
:10E250009047F6B2240E39E7FFF740FDC4F30740BC
:10E26000FFF73CFD200EFFF739FD0020BDE8F081EF
:10E270001E4B1D4A1B6880211170EDB2C4F3074686
:10E2800083B1314628463A4698473C461EE701206E
:10E29000BDE8F081104B1B68002B3FF44AAFFF2014
:10E2A000984746E71C4611E70D2EBCD10D2B7FF495
:10E2B00043AE0F4B0C4A1B68D0211170EDB2C4F372
:10E2C0000746002B7FF4FEAEC4E7C4F30746EDB269
:10E2D000240EFBE634A0FF1F10A0FF1F14A0FF1F99
:10E2E00004A0FF1F20A0FF1FC0A1FF1F58A0FF1FF9
:10E2F00030A0FF1F38B5164D2868E0B1018844886A
:10E30000A14213DD03191B7A83B104F10803C2187B
:10E310000C1B002302E012F8011F21B10133A342BC
:10E32000F9D1204638BD1C46204638BDFFF7B0FC69
:10E330000020286038BD074B1B780BB9002038BD82
:10E340000220FEF7F5FD28600028D7D1F6E700BFD0
:10E350006CA0FF1FFC9FFF1F0D4B1B78BBB910B5B6
:10E360000C4C216803F0FF024B883F2B07DC07337E
:10E370000B4401F1470003F8012F8342FBD14023F6
:10E380000B800120FEF76CFE0023236010BD704758
:10E3900064A0FF1F68A0FF1F38B5224C237803B18B
:10E3A00038BD01232370FFF7A5FF70BB00F048F8CC
:10E3B00040BB00F0DBF810BBFEF7F8FCE0B900232F
:10E3C0002370EFF30583002BEAD1EFF3108172B6CF
:10E3D000154B1868E0B1154C2278CAB945691D6023
:10E3E00001232370C5B1AA6101B962B60025457742
:10E3F000836898472570D3E700F020F8DFE700F046
:10E400001BF8D9E700F016F8D3E7FFF71FFCCDE7BC
:10E410000029C5D162B638BD054B1D600029E5D184
:10E42000E3E700BF71A0FF1F889EFF1F8C9EFF1FA8
:10E43000849EFF1F704700BF704700BF704700BF3A
:10E44000054A064B10781B78C0B2DBB2984238BF41
:10E450004030C01A704700BF78A0FF1F79A0FF1F8F
:10E46000F0B4384B1A7912F0300F2CD072B6997D77
:10E4700001F0FF0200293DD062B6334F33493878AE
:10E480000D78334E1C46C0B2EDB2431C402BE179EF
:10E4900028BF0023AB4202F1FF32C9B21CBFF154C6
:10E4A000184612F0FF02F0D12A4B1B68C2B23A7034
:10E4B0004BB1A84236BFC5F14005401B4019272883
:10E4C000C4BF01221A701F49CA78D2B2150616D4E9
:10E4D00052060DD51B4B1B795B0609D51E4B1F49F8
:10E4E0001B6800220A7003B11A70164B3C22DA70C6
:10E4F000F0BC70474022D9795A7462B6E3E70B79D1
:10E500001C06E5D5164B174E1C783378E4B2DBB207
:10E510009C420ED0144D01E0A3420AD00133402B9F
:10E5200028BF00230879E85CC0B2C871087D0728BD
:10E53000F2D9DBB2034933700B79180644BF7C2350
:10E54000CB70C5E700A0064078A0FF1F79A0FF1F91
:10E55000BCA0FF1F74A0FF1F00A1FF1FFCA0FF1F96
:10E5600004A1FF1FFDA0FF1F7CA0FF1F054A064B53
:10E5700010781B78C0B2DBB2984238BF4030C01A66
:10E58000704700BF78A1FF1F0DA1FF1FF0B4384BEB
:10E590001A7912F0300F2CD072B6997D01F0FF027B
:10E5A00000293DD062B6334F334938780D78334E69
:10E5B0001C46C0B2EDB2431C402BE17928BF0023BA
:10E5C000AB4202F1FF32C9B21CBFF154184612F03F
:10E5D000FF02F0D12A4B1B68C2B23A704BB1A8427D
:10E5E00036BFC5F14005401B40192728C4BF012292
:10E5F0001A701F49CA78D2B2150616D452060DD524
:10E600001B4B1B795B0609D51E4B1F491B6800225B
:10E610000A7003B11A70164B3C22DA70F0BC7047D6
:10E620004022D9795A7462B6E3E70B791C06E5D526
:10E63000164B174E1C783378E4B2DBB29C420ED0F6
:10E64000144D01E0A3420AD00133282B28BF002338
:10E650000879E85CC0B2C871087D0728F2D9DBB23E
:10E66000034933700B79180644BF7C23CB70C5E790
:10E6700000B0064078A1FF1F0DA1FF1F38A1FF1FAA
:10E6800008A1FF1F7CA1FF1F0CA1FF1F80A1FF1F7E
:10E6900079A1FF1F10A1FF1F70B584B072B6194B8E
:10E6A000194D1A48702241260F2480211A702E70AD
:10E6B0001A460470197013781B06FCD5144B1868A1
:10E6C00062B6144B144C984298BF00EB800001A92D
:10E6D00098BF40000A22FDF7CFFE01A92046002383
:10E6E00011F8012B01333AB10A2B20F8022FF7D190
:10E6F0001623237004B070BD5B00DBB2237004B03E
:10E7000070BD00BF0000024007000240060002404A
:10E71000080002407F969800AC92FF1FFFFFFFFFAA
:10E720002DE9F043DFF8EC808BB006460F4600F091
:10E7300073F898F90030013304460D4637D030465F
:10E74000394600F0DFF9002831D02BA3D3E90023AC
:10E750003046394600F026FE814668BB28A3D3E93F
:10E7600000233046394600F0FFFD00B398F9003031
:10E77000254ACDF82090042400200021022BCDE969
:10E780000467CDE9026700940192CDE906012CD01F
:10E79000684600F0BDF940B3089B1BB101F0AAF92F
:10E7A000089B0360DDE906010BB0BDE8F08320465D
:10E7B00029460BB0BDE8F083134A98F90030019266
:10E7C00003210022CDE90467CDE902670091089298
:10E7D0002BB90E4B4FF06042CDE90623D8E70C4928
:10E7E0000020022BCDE90601D2D101F083F92223CA
:10E7F0000360D1E7AFF30080EF39FAFE422E864086
:10E8000051302DD5104987C06C320100FFFFEF4712
:10E810000000F07FC292FF1F2DE9F04FB04F21F0B2
:10E820000042BA4283B00C464FEAD17605460DD974
:10E83000AC4FBA4225D9C1F31303034340F0EF8034
:10E840000EB10020014603B0BDE8F08FA64B9A42FE
:10E8500000F2CC80A54B9A4200F2DE808AA3D3E975
:10E86000002300F05DF90022A14B00F09BFD002881
:10E8700000F005812846214600229D4B00F050F90A
:10E88000E1E783A3D3E9002300F08CFD002840F0EA
:10E89000CB802846214680A3D3E9002300F064FD05
:10E8A0000028CED1934B284603EBC60821467CA313
:10E8B000D3E9002300F0E6FAD8E9002300F030F9AC
:10E8C00000F07AFD804600F077FA77A3D3E90023C1
:10E8D00006460F4600F0D6FA02460B462846214669
:10E8E00000F01CF972A3D3E90023CDE90001304602
:10E8F000394600F0C7FA82468B4652465B46DDE950
:10E90000000100F00BF905460C462A46234628462E
:10E91000214600F0B7FA68A3D3E9002306460F4664
:10E9200000F0B0FA66A3D3E9002300F0F7F832460E
:10E930003B4600F0A7FA64A3D3E9002300F0F0F807
:10E9400032463B4600F09EFA61A3D3E9002300F073
:10E95000E5F832463B4600F095FA5FA3D3E9002381
:10E9600000F0DEF832463B4600F08CFA02460B46D9
:10E970002846214600F0D2F806460F462846214692
:10E9800032463B46B8F1000F56D000F07BFA3246D3
:10E9900004460D463B4600204FF0804100F0BEF893
:10E9A00002460B462046294600F096FB02460B46DF
:10E9B0005046594600F0B2F8DDE9002300F0AEF809
:10E9C0000B4602464A49002000F0A8F86FF47F7316
:10E9D00098454FDA08F57A7801EB085100224FF09C
:10E9E000B87300F04FFA03B0BDE8F08F424B9A4283
:10E9F0003FF658AF414BF4002344D3E9002300F025
:10EA00008DF83F4BC6F101081C44CDE90001D4E963
:10EA100000ABC6EB080870E74FF0000875E7024648
:10EA20000B4600F07DF80EE717A3D3E9002310464C
:10EA3000194600F027FA06E700F024FA0022804683
:10EA400089464FF080433046394600F067F8024669
:10EA50000B464046494600F03FFB2A46234600F05D
:10EA60005DF802460B460020214900F057F803B03C
:10EA7000BDE8F08F01EB085103B0BDE8F08F804690
:10EA800043E700BFAFF300809C7500883CE4377E0D
:10EA9000EF39FAFE422E864051302DD5104987C0FD
:10EAA000FE822B654715F73F0000E0FE422EE63F51
:10EAB000763C7935EF39EA3DD0A4BE726937663EBF
:10EAC000F16BD2C541BDBB3E2CDE25AF6A56113F6E
:10EAD00093BDBE166CC1663F3E5555555555C53F55
:10EAE000412E8640FFFFEF7F422ED63FFFFF2F3E95
:10EAF0000000F03F70320100B1A2F03F90320100FF
:10EB00008032010041F0004101F58010C00F7047D4
:10EB10000020704781F0004102E000BF83F0004315
:10EB200030B54FEA41044FEA430594EA050F08BFA8
:10EB300090EA020F1FBF54EA000C55EA020C7FEA6C
:10EB4000645C7FEA655C00F0E2804FEA5454D4EBE9
:10EB50005555B8BF6D420CDD2C4480EA020281EAB3
:10EB6000030382EA000083EA010180EA020281EAEB
:10EB70000303362D88BF30BD11F0004F4FEA01313D
:10EB80004FF4801C4CEA113102D0404261EB41014C
:10EB900013F0004F4FEA03334CEA133302D05242D2
:10EBA00063EB430394EA050F00F0A780A4F101048E
:10EBB000D5F1200E0DDB02FA0EFC22FA05F28018C8
:10EBC00041F1000103FA0EF2801843FA05F35941AE
:10EBD0000EE0A5F120050EF1200E012A03FA0EFC2D
:10EBE00028BF4CF0020C43FA05F3C01851EBE37157
:10EBF00001F0004507D54FF0000EDCF1000C7EEB74
:10EC000000006EEB0101B1F5801F1BD3B1F5001FB1
:10EC10000CD349085FEA30004FEA3C0C04F10104D0
:10EC20004FEA445212F5800F80F09A80BCF1004FF9
:10EC300008BF5FEA500C50F1000041EB045141EA7B
:10EC4000050130BD5FEA4C0C404141EB010111F47C
:10EC5000801FA4F10104E9D191F0000F04BF014627
:10EC60000020B1FA81F308BF2033A3F10B03B3F105
:10EC700020020CDA0C3208DD02F1140CC2F10C0295
:10EC800001FA0CF021FA02F10CE002F11402D8BFF3
:10EC9000C2F1200C01FA02F120FA0CFCDCBF41EABF
:10ECA0000C019040E41AA2BF01EB0451294330BD8E
:10ECB0006FEA04041F3C1CDA0C340EDC04F114046B
:10ECC000C4F1200220FA04F001FA02F340EA030042
:10ECD00021FA04F345EA030130BDC4F10C04C4F188
:10ECE000200220FA02F001FA04F340EA0300294668
:10ECF00030BD21FA04F0294630BD94F0000F83F4B2
:10ED0000801306BF81F480110134013D4EE77FEA94
:10ED1000645C18BF7FEA655C29D094EA050F08BFE0
:10ED200090EA020F05D054EA000C04BF19461046C1
:10ED300030BD91EA030F1EBF0021002030BD5FEA05
:10ED4000545C05D14000494128BF41F0004130BD2D
:10ED500014F580043CBF01F5801130BD01F0004581
:10ED600045F0FE4141F470014FF0000030BD7FEAF4
:10ED7000645C1ABF194610467FEA655C1CBF0B46EF
:10ED8000024650EA013406BF52EA033591EA030F06
:10ED900041F4002130BD00BF90F0000F04BF0021FE
:10EDA000704730B54FF4806404F132044FF0000531
:10EDB0004FF0000150E700BF90F0000F04BF0021AA
:10EDC000704730B54FF4806404F1320410F0004510
:10EDD00048BF40424FF000013EE700BF42004FEA0B
:10EDE000E2014FEA31014FEA02701FBF12F07F4388
:10EDF00093F07F4F81F06051704792F0000F14BF85
:10EE000093F07F4F704730B54FF4607401F00045C8
:10EE100021F0004120E700BF50EA010208BF70471F
:10EE200030B54FF000050AE050EA010208BF704714
:10EE300030B511F0004502D5404261EB41014FF47D
:10EE4000806404F132045FEA915C3FF4DCAE4FF081
:10EE500003025FEADC0C18BF03325FEADC0C18BF68
:10EE6000033202EBDC02C2F1200300FA03FC20FAB9
:10EE700002F001FA03FE40EA0E0021FA02F1144406
:10EE8000C1E600BF70B54FF0FF0C4CF4E06C1CEA1B
:10EE900011541DBF1CEA135594EA0C0F95EA0C0F90
:10EEA00000F0DEF82C4481EA030621EA4C5123EA03
:10EEB0004C5350EA013518BF52EA033541F4801132
:10EEC00043F4801338D0A0FB02CE4FF00005E1FBE5
:10EED00002E506F00042E0FB03E54FF00006E1FB2F
:10EEE00003569CF0000F18BF4EF0010EA4F1FF0472
:10EEF000B6F5007F64F5407404D25FEA4E0E6D41B2
:10EF000046EB060642EAC62141EA55514FEAC520C2
:10EF100040EA5E504FEACE2EB4F1FD0C88BFBCF53E
:10EF2000E06F1ED8BEF1004F08BF5FEA500E50F1EF
:10EF3000000041EB045170BD06F0004646EA0101B5
:10EF400040EA020081EA0301B4EB5C04C2BFD4EBE7
:10EF50000C0541EA045170BD41F480114FF0000EE0
:10EF6000013C00F3AB8014F1360FDEBF002001F04E
:10EF7000004170BDC4F10004203C35DA0C341BDCC8
:10EF800004F11404C4F1200500FA05F320FA04F09A
:10EF900001FA05F240EA020001F0004221F00041CE
:10EFA00010EBD37021FA04F642EB06015EEA430E41
:10EFB00008BF20EAD37070BDC4F10C04C4F1200571
:10EFC00000FA04F320FA05F001FA04F240EA020024
:10EFD00001F0004110EBD37041F100015EEA430EF5
:10EFE00008BF20EAD37070BDC4F1200500FA05F215
:10EFF0004EEA020E20FA04F301FA05F243EA020394
:10F0000021FA04F001F0004121FA04F220EA0200A2
:10F0100000EBD3705EEA430E08BF20EAD37070BDE8
:10F0200094F0000F0FD101F00046400041EB0101C8
:10F0300011F4801F08BF013CF7D041EA060195F0AA
:10F04000000F18BF704703F00046520043EB030364
:10F0500013F4801F08BF013DF7D043EA0603704751
:10F0600094EA0C0F0CEA135518BF95EA0C0F0CD05C
:10F0700050EA410618BF52EA4306D1D181EA0301A2
:10F0800001F000414FF0000070BD50EA410606BF9C
:10F090001046194652EA430619D094EA0C0F02D1E1
:10F0A00050EA013613D195EA0C0F05D152EA033626
:10F0B0001CBF104619460AD181EA030101F0004144
:10F0C00041F0FE4141F470014FF0000070BD41F08D
:10F0D000FE4141F4780170BD70B54FF0FF0C4CF467
:10F0E000E06C1CEA11541DBF1CEA135594EA0C0F86
:10F0F00095EA0C0F00F0A7F8A4EB050481EA030ED3
:10F1000052EA03354FEA013100F088804FEA0333B9
:10F110004FF0805545EA131343EA12634FEA022287
:10F1200045EA111545EA10654FEA00260EF0004148
:10F130009D4208BF964244F1FD0404F5407402D29A
:10F140005B084FEA3202B61A65EB03055B084FEA2B
:10F1500032024FF480104FF4002CB6EB020E75EB28
:10F16000030E22BFB61A754640EA0C005B084FEA50
:10F170003202B6EB020E75EB030E22BFB61A7546CD
:10F1800040EA5C005B084FEA3202B6EB020E75EB18
:10F19000030E22BFB61A754640EA9C005B084FEA90
:10F1A0003202B6EB020E75EB030E22BFB61A75469D
:10F1B00040EADC0055EA060E18D04FEA051545EA8C
:10F1C00016754FEA06164FEAC30343EA52734FEA35
:10F1D000C2025FEA1C1CC0D111F4801F0BD141EAAE
:10F1E00000014FF000004FF0004CB6E711F4801F13
:10F1F00004BF01430020B4F1FD0C88BFBCF5E06FF3
:10F200003FF6AFAEB5EB030C04BFB6EB020C5FEA02
:10F21000500C50F1000041EB045170BD0EF0004E57
:10F220004EEA113114EB5C04C2BFD4EB0C0541EA89
:10F23000045170BD41F480114FF0000E013C90E686
:10F2400045EA060E8DE60CEA135594EA0C0F08BF4A
:10F2500095EA0C0F3FF43BAF94EA0C0F0AD150EA49
:10F2600001347FF434AF95EA0C0F7FF425AF1046DC
:10F2700019462CE795EA0C0F06D152EA03353FF404
:10F28000FDAE1046194622E750EA410618BF52EA81
:10F2900043067FF4C5AE50EA41047FF40DAF52EA55
:10F2A00043057FF4EBAE12E74FF0FF3C06E000BFF2
:10F2B0004FF0010C02E000BF4FF0010C4DF804CDFF
:10F2C0004FEA410C7FEA6C5C4FEA430C18BF7FEABF
:10F2D0006C5C1BD001B050EA410C0CBF52EA430CED
:10F2E00091EA030F02BF90EA020F0020704710F16D
:10F2F000000F91EA030F58BF994208BF90422CBFFC
:10F30000D8176FEAE37040F0010070474FEA410CF4
:10F310007FEA6C5C02D150EA013C07D14FEA430C12
:10F320007FEA6C5CD6D152EA033CD3D05DF8040B83
:10F33000704700BF8446104662468C4619466346B5
:10F3400000E000BF01B5FFF7B7FF002848BF10F18C
:10F35000000F01BD4DF808EDFFF7F4FF0CBF0120D1
:10F3600000205DF808FB00BF4DF808EDFFF7EAFF4D
:10F3700034BF012000205DF808FB00BF4DF808ED08
:10F38000FFF7E0FF94BF012000205DF808FB00BFFD
:10F390004DF808EDFFF7CEFF94BF012000205DF887
:10F3A00008FB00BF4DF808EDFFF7C4FF34BF012094
:10F3B00000205DF808FB00BF4FEA410212F5001281
:10F3C00015D211D56FF47873B3EB625212D94FEAAC
:10F3D000C12343F0004343EA505311F0004F23FA96
:10F3E00002F018BF404270474FF00000704750EAEB
:10F3F000013005D111F0004008BF6FF000407047A8
:10F400004FF00000704700BF4FEA4102B2F1E04305
:10F4100024BFB3F5001CDCF1FE5C0DD901F0004CFB
:10F420004FEAC0024CEA5070B2F1004F40EB83004B
:10F4300008BF20F00100704711F0804F21D113F177
:10F440003872BCBF01F00040704741F480114FEAB0
:10F450005252C2F11802C2F1200C10FA0CF320FA39
:10F4600002F018BF40F001004FEAC1234FEAD32356
:10F4700003FA0CFC40EA0C0023FA02F34FEA4303C0
:10F48000CCE77FEA625307D150EA01331EBF4FF049
:10F49000FE4040F44000704701F0004040F0FE4064
:10F4A00040F40000704700BF80F0004002E000BF61
:10F4B00081F0004142001FBF5FEA410392EA030F5F
:10F4C0007FEA226C7FEA236C6AD04FEA1262D2EBA9
:10F4D0001363C1BFD218414048404140B8BF5B42AE
:10F4E000192B88BF704710F0004F40F4000020F047
:10F4F0007F4018BF404211F0004F41F4000121F05D
:10F500007F4118BF494292EA030F3FD0A2F10102A6
:10F5100041FA03FC10EB0C00C3F1200301FA03F1E4
:10F5200000F0004302D5494260EB4000B0F5000F07
:10F5300013D3B0F1807F06D340084FEA310102F1C6
:10F540000102FE2A51D2B1F1004F40EBC25008BF78
:10F5500020F0010040EA03007047490040EB000042
:10F5600010F4000FA2F10102EDD1B0FA80FCACF171
:10F57000080CB2EB0C0200FA0CF0AABF00EBC25070
:10F5800052421843BCBFD0401843704792F0000F5E
:10F5900081F4000106BF80F400000132013BB5E7B1
:10F5A0004FEA41037FEA226C18BF7FEA236C21D027
:10F5B00092EA030F04D092F0000F08BF084670478C
:10F5C00090EA010F1CBF0020704712F07F4F04D15A
:10F5D000400028BF40F00040704712F100723CBF6D
:10F5E00000F50000704700F0004343F0FE4040F497
:10F5F000000070477FEA226216BF08467FEA236355
:10F600000146420206BF5FEA412390EA010F40F43F
:10F61000800070474FF0000304E000BF10F000438B
:10F6200048BF40425FEA000C08BF704743F0964372
:10F6300001464FF000001CE050EA010208BF70478D
:10F640004FF000030AE000BF50EA010208BF704714
:10F6500011F0004302D5404261EB41015FEA010C29
:10F6600002BF84460146002043F0B64308BFA3F121
:10F670008053A3F50003BCFA8CF2083AA3EBC25303
:10F6800010DB01FA02FC634400FA02FCC2F1200222
:10F69000BCF1004F20FA02F243EB020008BF20F059
:10F6A0000100704702F1200201FA02FCC2F12002BF
:10F6B00050EA4C0021FA02F243EB020008BF20EAB4
:10F6C000DC7070474FF0FF0C1CEAD0521EBF1CEAE2
:10F6D000D15392EA0C0F93EA0C0F6FD01A4480EAD0
:10F6E000010C400218BF5FEA41211ED04FF00063B9
:10F6F00043EA501043EA5111A0FB01310CF00040E5
:10F70000B1F5000F3EBF490041EAD3715B0040EA0A
:10F71000010062F17F02FD2A1DD8B3F1004F40EBDA
:10F72000C25008BF20F00100704790F0000F0CF0AD
:10F73000004C08BF49024CEA502040EA51207F3A71
:10F74000C2BFD2F1FF0340EAC250704740F400004C
:10F750004FF00003013A5DDC12F1190FDCBF00F03D
:10F7600000407047C2F10002410021FA02F1C2F1EB
:10F77000200200FA02FC5FEA310040F1000053EA87
:10F780004C0308BF20EADC70704792F0000F00F0D5
:10F79000004C02BF400010F4000F013AF9D040EADB
:10F7A0000C0093F0000F01F0004C02BF490011F46F
:10F7B000000F013BF9D041EA0C018FE70CEAD1536D
:10F7C00092EA0C0F18BF93EA0C0F0AD030F0004CED
:10F7D00018BF31F0004CD8D180EA010000F00040A1
:10F7E000704790F0000F17BF90F0004F084691F05F
:10F7F000000F91F0004F14D092EA0C0F01D1420299
:10F800000FD193EA0C0F03D14B0218BF084608D161
:10F8100080EA010000F0004040F0FE4040F40000AB
:10F82000704740F0FE4040F4400070474FF0FF0C3E
:10F830001CEAD0521EBF1CEAD15392EA0C0F93EA85
:10F840000C0F69D0A2EB030280EA010C49024FEAD7
:10F85000402037D04FF0805343EA111143EA101390
:10F860000CF000408B4238BF5B0042F17D024FF448
:10F87000000C8B4224BF5B1A40EA0C00B3EB510F23
:10F8800024BFA3EB510340EA5C00B3EB910F24BF0C
:10F89000A3EB910340EA9C00B3EBD10F24BFA3EB91
:10F8A000D10340EADC001B0118BF5FEA1C1CE0D159
:10F8B000FD2A3FF650AF8B4240EBC25008BF20F00C
:10F8C000010070470CF0004C4CEA50207F32C2BF60
:10F8D000D2F1FF0340EAC250704740F400004FF0FD
:10F8E0000003013A37E792F0000F00F0004C02BF2E
:10F8F000400010F4000F013AF9D040EA0C0093F0F8
:10F90000000F01F0004C02BF490011F4000F013B51
:10F91000F9D041EA0C0195E70CEAD15392EA0C0FB9
:10F9200008D142027FF47DAF93EA0C0F7FF470AFF1
:10F93000084676E793EA0C0F04D14B023FF44CAF34
:10F9400008466EE730F0004C18BF31F0004CCAD1C9
:10F9500030F000427FF45CAF31F000437FF43CAF05
:10F960005FE700BF4FF0FF3C06E000BF4FF0010C27
:10F9700002E000BF4FF0010C4DF804CD4FEA400209
:10F980004FEA41037FEA226C18BF7FEA236C11D053
:10F9900001B052EA530C18BF90EA010F58BFB2EB06
:10F9A000030088BFC81738BF6FEAE17018BF40F086
:10F9B000010070477FEA226C02D15FEA402C05D13A
:10F9C0007FEA236CE4D15FEA412CE1D05DF8040BBF
:10F9D000704700BF844608466146FFE70FB5FFF752
:10F9E000C9FF002848BF10F1000F0FBD4DF808ED0A
:10F9F000FFF7F4FF0CBF012000205DF808FB00BFFB
:10FA00004DF808EDFFF7EAFF34BF012000205DF854
:10FA100008FB00BF4DF808EDFFF7E0FF94BF0120A1
:10FA200000205DF808FB00BF4DF808EDFFF7D2FF9E
:10FA300094BF012000205DF808FB00BF4DF808EDE1
:10FA4000FFF7C8FF34BF012000205DF808FB00BFAE
:10FA50004FEA4002B2F1FE4F0FD34FF09E03B3EBDB
:10FA600012620DD94FEA002343F0004310F0004F1B
:10FA700023FA02F018BF404270474FF00000704771
:10FA800012F1610F01D1420205D110F0004008BF10
:10FA90006FF0004070474FF00000704742000ED2F8
:10FAA000B2F1FE4F0BD34FF09E03B3EB126209D4B9
:10FAB0004FEA002343F0004323FA02F070474FF06F
:10FAC0000000704712F1610F01D1420202D14FF0E4
:10FAD000FF3070474FF00000704700BF0B460146F3
:10FAE000184600F001B800BF13460A46014602203E
:10FAF00000F0B8BE014B1868704700BFF096FF1FBA
:10FB000070B50F4E0F4D761BB61018BF002405D0F0
:10FB1000013455F8043B9847A642F9D10A4E0B4DE3
:10FB2000761B03F0BFFBB61018BF002406D00134CB
:10FB300055F8043B9847A642F9D170BD70BD00BF8F
:10FB4000B0320100B0320100C4320100B032010015
:10FB5000024B0146186800F00BB800BFF096FF1F7B
:10FB6000024B0146186800F041BF00BFF096FF1F2E
:10FB70002DE9F04F01F10B05162D83B0064640F23A
:10FB80009F8035F0070500F1BF80A94200F2BC80DC
:10FB900000F058FBB5F5FC7FC0F09C826B0A00F0CA
:10FBA000BA80042B00F28381A80900F1390E4FEAD4
:10FBB0004E033830C44F07EB8303A3F108015C68A0
:10FBC000A14207D1ACE0002A80F2AC80E468A142F7
:10FBD00000F0A680636823F003035A1B0F2AF2DDAE
:10FBE000B9493C6901F1080E744500F0B3816368BE
:10FBF00023F003035A1B0F2A00F39981002AC1F84E
:10FC000014E0C1F810E080F29E80B3F5007F80F030
:10FC10006781DB0803F1010C01229B1002FA03F358
:10FC20004A6851F83C80C4F8088001EBCC091A43BB
:10FC3000A9F10803E3604A6041F83C40C8F80C4071
:10FC4000831001249C40944200F28A80144206D121
:10FC500020F003006400144200F10400FAD007EB26
:10FC6000C009CC468046DCF80C108C4507D173E106
:10FC7000002A80F28181C9688C4500F06D814B6853
:10FC800023F003035A1B0F2AF2DD0C46D1F80CC0F7
:10FC900054F8088F4B1945F001054D6042F0010101
:10FCA000C8F80CC03046CCF808807B613B61C3F8D3
:10FCB0000CE0C3F808E059609A5000F0C5FA1FE064
:10FCC000102921D800F0BEFA1025062302207E4F0D
:10FCD00007EB8303A3F108025C68944200F04581BE
:10FCE0006368E168A56823F00303234430465A683B
:10FCF000E96042F001028D605A6000F0A5FA083414
:10FD0000204603B0BDE8F08F00240C23204633606A
:10FD100003B0BDE8F08F80234FF0400E3F2049E74D
:10FD200070465DE72344E1685A68A56842F0010225
:10FD3000E96030468D605A6000F086FA083420464B
:10FD400003B0BDE8F08F234430465A6842F0010208
:10FD50005A6000F079FA0834204603B0BDE8F08F0D
:10FD6000BC68636823F00308A84504D3C5EB080307
:10FD70000F2B00F38C80554BDFF860911A68D9F88F
:10FD8000003001332A4404EB080A00F0608102F5D8
:10FD900080520F3222F47F6222F00F021146304669
:10FDA000019200F04BFCB0F1FF3F8346019A00F056
:10FDB0005881824500F2FC80454B1968DA451144B0
:10FDC000196000F05381D9F80000DFF810E101302C
:10FDD0001BBFCAEB0B0A5144CEF800B019601BF0F0
:10FDE000070100F01781C1F10800C1F5805183447B
:10FDF00008315A44C2F30B02C2EB010949463046AE
:10FE0000019300F01BFC431C019B00F03F81CBEBF6
:10FE100000024A4442F001021968C7F808B0494498
:10FE2000BC42CBF804201960DFF8A49016D0B8F1DA
:10FE30000F0F40F2FD806268A8F10C0323F0070366
:10FE4000E01802F001024FF0050E1A430F2B62601A
:10FE5000C0F804E0C0F808E000F21C811D4BBC684B
:10FE60001A68914288BF19601B4B1A6891426268F8
:10FE700088BF196022F003029542A2EB050301D866
:10FE80000F2B04DC304600F0DFF9002438E762195C
:10FE900043F0010345F0010565603046BA605360E8
:10FEA00000F0D2F90834204603B0BDE8F08F142BDF
:10FEB00071D9542B00F2A480280B00F16F0E4FEA89
:10FEC0004E036E3076E600BFF496FF1F8CA1FF1F35
:10FED00090A1FF1F88A1FF1F84A1FF1F009BFF1F90
:10FEE0005A0A042A5ED9142A00F2B38002F15C0196
:10FEF00049005B3207EB810C57F82110DFF8DC81F9
:10FF0000ACF1080C8C4500F088804A6822F00302AE
:10FF1000934202D289688C45F7D1D1F80CC07A6837
:10FF2000C4F80CC0A160CCF80840CC6088E6631926
:10FF300042F0010745F00105656030464B610B61F9
:10FF4000C3F80CE0C3F808E05F609A50083400F092
:10FF50007BF9D5E64A6873E608F1010818F0030F4B
:10FF60000CF1080C7FF47FAE30E0DC68A34208BFE0
:10FF700002303FF435AEB3E60B440C465A68C9680C
:10FF800054F8085F42F001025A603046E9608D6023
:10FF900000F05AF9B4E603F15C0E03F15B004FEA9E
:10FFA0004E0307E69A0902F1390149003832A1E708
:10FFB000BC424A4B3FF400AF9C68626822F00302E7
:10FFC0005AE759F80839994540F0828010F0030F3C
:10FFD00000F1FF30F5D17B6823EA04037B60640005
:10FFE0009C423FF6BDAE002C3FF4BAAE1C424046E8
:10FFF0007FF435AE64001C4200F10400FAD02EE616
:020000021000EC
:10000000B3F5AA7F18D8E80B00F1780E4FEA4E033B
:100010007730CFE54FF48051EBE60121D8F804307A
:10002000921001FA02F21A43C8F80420614677E7F9
:100030000123CBF8043025E740F25452934220D8F4
:10004000A80C00F17D0E4FEA4E037C30B2E5103271
:10005000A4E6542A26D81A0B02F16F0149006E3229
:1000600048E7BC68626822F0030205E7CAF30B00A8
:1000700000287FF4A8AE4244BB6842F001025A60F7
:10008000ECE6FE234FF07F0E7E2093E501224FF039
:100090000009C1E604F10801304600F0A7FCD9F8D8
:1000A0000010DBE6B2F5AA7F05D8DA0B02F1780181
:1000B000490077321EE740F254518A4205D89A0C23
:1000C00002F17D0149007C3214E7FE217E2211E716
:1000D0007B6884E7E808431C5B00F8E5F496FF1FA3
:1000E0008842F0B50DD98B1898420AD28118002A9F
:1000F00051D09A1A13F8014D01F8014D9342F9D1EC
:10010000F0BD0F2A48D941EA00039B0746D100F110
:10011000100401F11003154653F8106C44F8106CEC
:1001200053F80C6C44F80C6C53F8086C44F8086CE9
:10013000103D53F8046C44F8046C0F2D03F11003C8
:1001400004F11004E8D8A2F1100323F00F0302F029
:100150000F0E1033BEF1030F1944034421D91E1FA3
:100160000D467446043C55F8047B46F8047F032C86
:10017000F8D8AEF1040424F00304043423442144E9
:1001800002F0030262B1013B0A4411F8014B03F88B
:10019000014F8A42F9D1F0BD0346F3E70346F2E787
:1001A000F0BD7246EEE700BF70B4840746D0541E1F
:1001B000002A41D0CDB2034602E0621EE4B31446E9
:1001C00003F8015B9A07F8D1032C2ED9CDB245EA8A
:1001D00005250F2C45EA054519D903F110022646DD
:1001E000103E0F2E42F8105C42F80C5C42F8085C9E
:1001F00042F8045C02F11002F2D8A4F1100222F0DD
:100200000F0204F00F041032032C13440DD91E46C4
:100210002246043A032A46F8045BFAD8221F22F049
:1002200003020432134404F003042CB1C9B21C4489
:1002300003F8011BA342FBD170BC70471446034670
:10024000C2E700BF704700BF704700BF024B0A46BD
:100250000146186800F002B8F096FF1F2DE9F04F34
:10026000174683B0002900F0C1800E46814607F191
:100270000B05FFF7E7FF56F804EC162D2EF00304EC
:10028000A6F1080840D810221546AF4241D8944242
:1002900075DAC94B996808EB04008842416800F0A0
:1002A000D98021F0010303445B68DB077DD51EF094
:1002B000010F35D039464846FFF75AFC0746E0B1F2
:1002C00056F8043C23F001034344A0F108029A428B
:1002D00000F04481221F242A00F23181132A00F207
:1002E000048103463246116819605168596092686A
:1002F0009A603146484600F079FB4846FFF7A4FF74
:10030000384603B0BDE8F08F25F00705002D2A46DA
:10031000BBDA0C230020C9F8003003B0BDE8F08F31
:1003200056F8083CC3EB080ADAF8043023F0030C53
:1003300004EB0C039342BDDB5746DAF80C1057F878
:10034000080F221F242AC160886000F21781132A37
:1003500040F212813168CAF808107168CAF80C10AE
:100360001B2A00F22B8108360AF110023168116055
:1003700071685160B16891603E461C46D046631B6F
:100380000F2B1DD8D8F8043003F001032343444455
:10039000C8F80430636843F0010363604846FFF720
:1003A00053FF304603B0BDE8F08F21F00301214434
:1003B000914221DBC36882680C46D3609A60DEE715
:1003C000D8F8042008EB050102F00102154343F0C0
:1003D00001020B44C8F804504A605A6842F0010216
:1003E00008315A60484600F001FBD7E7114603B0D8
:1003F000BDE8F04FFFF7BCBB1EF0010F7FF45AAF12
:1004000056F8083CC3EB080ADAF8043023F0030C72
:1004100001EB0C0E96458BDBC36882685746D360B0
:100420009A6057F8081FDAF80C30CB60221F242A94
:10043000996000F29980132A62D93368CAF80830AB
:100440007368CAF80C301B2A00F2A08008360AF143
:10045000100356E021F0030BA34405F1100083457F
:1004600059DA1EF0010F7FF425AF56F8081CC1EBD6
:10047000080ADAF8041021F0030CE34458453FF76A
:1004800057AF5746DAF80C1057F8080F221F242AE6
:10049000C160886000F2B480132A40F2A580316800
:1004A000CAF808107168CAF80C101B2A00F2AF8055
:1004B00008360AF110023168116071685160B16844
:1004C00091600AEB0501C5EB0B0242F00102996055
:1004D0004A60DAF8043003F001031D434846CAF8C5
:1004E0000450FFF7B1FE38465CE733680360736879
:1004F00043601B2A27D800F1080306F10802F2E640
:100500003B4632681A6072685A60B2689A603E462A
:100510007446D04633E708EB0501C5EB0B0B4BF0F7
:10052000010299604A6056F8043C03F001031D4340
:10053000484646F8045CFFF787FE304632E731460E
:10054000FFF7CEFDD5E6B3688360F368C360242A65
:1005500028D000F1100306F11002C4E650F8043C64
:1005600023F003031C440AE7314638467446D0465C
:10057000FFF7B6FD3E4602E73A46F7E63146384613
:100580001C46D046FFF7ACFD3E46F8E6B368CAF815
:100590001030F368CAF81430242A1BD010360AF140
:1005A0001803AEE7336903617369436106F118020A
:1005B00000F1180397E600BFF496FF1FB168CAF870
:1005C0001010F168CAF81410242A0FD010360AF15E
:1005D0001802CBE63369CAF818307369CAF81C30C0
:1005E00018360AF120038CE73A4664E73269CAF804
:1005F00018207269CAF81C2018360AF12002B5E6E4
:10060000314638460193FFF76BFD019B59E7B1680E
:10061000CAF81010F168CAF81410242A03D0103652
:100620000AF1180247E73269CAF818207269CAF855
:100630001C2018360AF120023DE700BF38B5074CF0
:100640000023054608462360FBF7E0FE431C00D06C
:1006500038BD2368002BFBD02B6038BDECA2FF1FF8
:10066000FFFFFFFFFFFFFFFFFFFFFFFFFFFFFFFF9A
:10067000FFFFFFFFFFFFFFFFFFFFFFFFFFFFFFFF8A
:1006800090F800F06DE9024520F007016FF0000CD2
:1006900010F0070491F820F040F049804FF000047A
:1006A0006FF00700D1E9002391F840F000F1080055
:1006B00082FA4CF2A4FA8CF283FA4CF3A2FA8CF38D
:1006C0004BBBD1E9022382FA4CF200F10800A4FAF4
:1006D0008CF283FA4CF3A2FA8CF3E3B9D1E9042348
:1006E00082FA4CF200F10800A4FA8CF283FA4CF37F
:1006F000A2FA8CF37BB9D1E9062301F1200182FA39
:100700004CF200F10800A4FA8CF283FA4CF3A2FA3E
:100710008CF3002BC6D0002A04BF04301A4612BA4C
:10072000B2FA82F2FDE8024500EBD2007047D1E94F
:10073000002304F00305C4F100004FEAC50514F0DE
:10074000040F91F840F00CFA05F562EA05021CBFAF
:1007500063EA050362464FF00004A9E7002A41D08E
:1007600040EA010313F00303F0B425D1032A23D98F
:1007700004680D68AC421FD1043A35D0A4F10135AC
:1007800025EA040414F0803F31D1071D0D1D0DE052
:1007900057F8043B0E68A3F10134B34224EA030482
:1007A0000AD1043A20D014F0803F23D1032A2946ED
:1007B000384605F10405EBD803780C789C4202F129
:1007C000FF320CD182B114B916E06AB17BB110F8D6
:1007D000013F11F8014FA34202F1FF32F5D0181B7F
:1007E000F0BC7047104670471046F0BC7047184682
:1007F000F0BC70470020F3E72046F1E740EA010330
:100800009B0770B42BD1032A29D90C4603462146F5
:1008100054F8046BA6F1013525EA060515F0803F72
:1008200006D1043A032A43F8046B2146EFD8A2B15B
:100830000C781C70013A013301313CB16AB111F8F6
:10084000014B03F8014B013A002CF7D12AB11A44AD
:10085000002103F8011B9A42FBD170BC704703468C
:10086000E5E700BF2DE9F047254C2568D5F848415C
:100870000646884692469946C4B360681F2817DC2E
:10088000431C76B104EB80050122C5F888A0D4F89A
:10089000881182401143022EC4F88811C5F80891CE
:1008A0001ED00230636044F820800020BDE8F0874D
:1008B000144B03B34FF4C870FFF74AF90446D0B1A4
:1008C000D5F84831002780E88800C5F84841384607
:1008D0000123C4F88871C4F88C71002EE1D0D1E7EF
:1008E000D4F88C110A43C4F88C21DAE705F5A67414
:1008F000C5F84841C1E74FF0FF30BDE8F08700BFC1
:10090000A032010051FB0000024B13B1024800F07D
:1009100005B87047000000002909010000230146C6
:100920001A461846FFF79EBF38B5074D074C2C1BDB
:10093000A41005D0013C55F8043D9847002CF9D18E
:10094000BDE8384002F0BEBC00000000000000001E
:10095000F8B5234F0C460646FFF774FCBB685D688C
:1009600025F00305291B01F6EF7121F47F6121F0C9
:100970000F01A1F58054B4F5805F07DB00213046FC
:10098000FFF75CFEBB682B44984204D03046FFF76B
:100990005BFC0020F8BD61423046FFF74FFE01309E
:1009A0000DD0104BBA6819682D1B45F00105304673
:1009B000091B55601960FFF747FC0120F8BD0021B5
:1009C0003046FFF73BFEBA68831A0F2BDEDD064C7C
:1009D0000449246843F00103001B53600860D5E715
:1009E000F496FF1F90A1FF1F009BFF1F002945D019
:1009F0002DE9F0410D468046FFF724FC55F8047CB4
:100A00006A4927F00103A5F10804E2188E685068CE
:100A1000B24220F0030062D0FE0750600BD455F8BC
:100A2000087CE41B01F1080EA56875453B446FD0B6
:100A3000E768EF60BD6015186D68ED0742D543F0BB
:100A400001026260E350B3F5007F18D2DB085A1C44
:100A50004D6851F83270A76001209B1000FA03F333
:100A600001EBC2001D430838E0604D6041F83240A0
:100A7000FC604046BDE8F041FFF7E6BB70475A0A0C
:100A8000042A53D89A0902F139077F0002F1380588
:100A900001EB870051F827204449083890424DD097
:100AA000516821F003018B4202D292689042F7D143
:100AB000D068E060A2608460D4604046BDE8F04148
:100AC000FFF7C2BB95683A4FBD4203443FD0D068A0
:100AD000E86043F0010285606260E350B3E7FF071E
:100AE000034407D455F8082CA41A1344A068E268FC
:100AF000C26090602F4A126843F001009342606028
:100B00008C60B6D32C4B40461968FFF721FFB0E745
:100B100011184968C90744D49168D268CA6003446F
:100B200043F0010091606060E350A2E7142A17D8F7
:100B300002F15C077F0002F15B05A9E7AA104B6890
:100B4000012505FA02F213434B600246B1E743F078
:100B500001024C610C61E560A5606260E35088E7CA
:100B6000542A06D81A0B02F16F077F0002F16E05B6
:100B70008EE7B2F5AA7F06D8DA0B02F178077F007C
:100B800002F1770584E740F25450824206D89A0C6D
:100B900002F17D077F0002F17C0579E7FE277E25C3
:100BA00076E743F001026260E35062E7F496FF1FCC
:100BB000FC96FF1FFC9AFF1F8CA1FF1F0000780509
:100BC0003408540B800C3C0F5C12E015FA19141E0B
:100BD0006022AC265C2B0C30BC34023AFF3FFFFF96
:100BE000FDFFFFFFFBFFFFFFF8FFFFFFFDFFFFFF24
:100BF000FBFFFFFFF8FFFFFFFDFFFFFFFAFFFFFF17
:100C0000F7FFFFFFFDFFFFFFFBFFFFFFF7FFFFFF0A
:100C1000FCFFFFFFFBFFFFFFF7FFFFFFFDFFFFFFF5
:100C2000FAFFFFFFF7FFFFFFFDFFFFFFFBFFFFFFE7
:100C3000F8FFFFFFFDFFFFFFFBFFFFFFF8FFFFFFD8
:100C4000FDFFFFFFFAFFFFFFF7FFFFFFFCFFFFFFC6
:100C5000FBFFFFFFF7FFFFFFFDFFFFFFFBFFFFFFB6
:100C6000F7FFFFFFFDFFFFFFFAFFFFFFF7FFFFFFAB
:100C7000FDFFFFFFFBFFFFFFF7FFFFFFFDFFFFFF94
:100C8000FBFFFFFFF7FFFFFFFDFFFFFFFAFFFFFF87
:100C9000F7FFFFFFFDFFFFFFFAFFFFFFF8FFFFFF7A
:100CA000FDFFFFFFFAFFFFFFF7FFFFFFFDFFFFFF65
:100CB000FAFFFFFFF7FFFFFFFDFFFFFFFAFFFFFF58
:100CC000F8FFFFFFFDFFFFFFFAFFFFFFF8FFFFFF49
:100CD000FDFFFFFFFAFFFFFFF7FFFFFFFCFFFFFF36
:100CE000FBFFFFFFF7FFFFFFFDFFFFFFFAFFFFFF27
:100CF000F7FFFFFFFDFFFFFFFAFFFFFFF7FFFFFF1B
:100D0000FEFFFFFFFBFFFFFFF8FFFFFFFEFFFFFF00
:100D1000FBFFFFFFF8FFFFFFFDFFFFFFFAFFFFFFF5
:100D2000F7FFFFFFFCFFFFFFFAFFFFFFF7FFFFFFEB
:100D3000FCFFFFFFFAFFFFFFF7FFFFFFFDFFFFFFD5
:100D4000FAFFFFFFF7FFFFFFFDFFFFFFF9FFFFFFC8
:100D5000F7FFFFFFFDFFFFFFF9FFFFFFF7FFFFFFBB
:100D6000FDFFFFFFFAFFFFFFF7FFFFFFFDFFFFFFA4
:100D7000FAFFFFFFF7FFFFFFFDFFFFFFFAFFFFFF97
:100D8000F6FFFFFFFDFFFFFFFAFFFFFFF7FFFFFF8B
:100D9000FEFFFFFFFBFFFFFFF7FFFFFFFEFFFFFF71
:100DA000FBFFFFFFF7FFFFFFFDFFFFFFFAFFFFFF66
:100DB000F7FFFFFFFDFFFFFFFBFFFFFFF8FFFFFF58
:100DC000FDFFFFFFFBFFFFFFF8FFFFFFFDFFFFFF42
:100DD000FAFFFFFFF7FFFFFFFCFFFFFFF9FFFFFF39
:100DE000F7FFFFFFFCFFFFFFF9FFFFFFF7FFFFFF2C
:100DF000FDFFFFFFFAFFFFFFF7FFFFFFFDFFFFFF14
:100E0000FAFFFFFFF7FFFFFFFDFFFFFFF9FFFFFF07
:100E1000F6FFFFFFFDFFFFFFFAFFFFFFF7FFFFFFFA
:100E2000D8130100B4130100901301006C130100EA
:100E300024100100E00E0100040F0100280F010042
:100E40004C0F01008C110100B0110100BC0B01001E
:100E50004810010000000000070000000C00000026
:100E60001000000013000000180000001C0000002B
:100E700000000000070000000C000000130000004C
:100E8000180000001F000000240000000000000007
:100E90000C000000180000002400000030000000DA
:100EA0003C0000004800000000000000FBFFFFFFC6
:100EB000F4FFFFFFEFFFFFFFE8FFFFFFE3FFFFFF90
:100EC000DCFFFFFF00000000F4FFFFFFE8FFFFFF73
:100ED000DCFFFFFFD0FFFFFFC4FFFFFFB8FFFFFFF6
:100EE0000000580246056608540BD80E5C12E01547
:100EF000FA19141E6022AC265C2B0C30BC34023A6A
:100F0000FF3FFFFF0000900120031405D0075A0A9D
:100F1000AC0DCC10B4146A18E81C342180252A2B9F
:100F200070301437FF3FFFFF0000C800F401840356
:100F3000140508072E091C0CD80EF811AE159619C9
:100F4000401F1C25F22B5834FF3FFFFF00006400B8
:100F5000C8009001BC021A04DC059E07F609800C4B
:100F6000A00F2413A2174C1D5424442FFF3FFFFF52
:100F7000FBFFFFFFF8FFFFFFF4FFFFFFFAFFFFFF9C
:100F8000F7FFFFFFF4FFFFFFFDFFFFFFF9FFFFFF8C
:100F9000F4FFFFFFFAFFFFFFF7FFFFFFF4FFFFFF84
:100FA000FCFFFFFFF7FFFFFFF4FFFFFFFBFFFFFF6B
:100FB000F8FFFFFFF4FFFFFFFDFFFFFFFAFFFFFF5A
:100FC000F4FFFFFFFDFFFFFFF9FFFFFFF4FFFFFF4F
:100FD000FDFFFFFFF8FFFFFFF4FFFFFFFCFFFFFF38
:100FE000F7FFFFFFF4FFFFFFFBFFFFFFF8FFFFFF2F
:100FF000F4FFFFFFFCFFFFFFF7FFFFFFF4FFFFFF22
:1010000040067805B004E80384032003BC025802BC
:10101000F40190012C01FA00C8009600640032002F
:101020001900FFFF0000FF03FF07FF0BFF0FFF1377
:10103000FF17FF1BFF1FFF23FF27FF2BFF2FFF3390
:10104000FF37FF3BFF3FFFFF0000D007800CD80EAB
:101050000010C012EC130C17FA19141E6022AC26F3
:101060005C2B0C30BC34023AFF3FFFFFFBFFFFFF5D
:10107000F8FFFFFFF4FFFFFFFAFFFFFFF7FFFFFF9F
:10108000F4FFFFFFFDFFFFFFF9FFFFFFF4FFFFFF8E
:10109000FAFFFFFFF7FFFFFFF4FFFFFFFCFFFFFF7B
:1010A000F7FFFFFFF4FFFFFFFBFFFFFFF8FFFFFF6E
:1010B000F4FFFFFFFDFFFFFFFAFFFFFFF4FFFFFF5D
:1010C000FBFFFFFFF8FFFFFFF4FFFFFFFDFFFFFF48
:1010D000F8FFFFFFF4FFFFFFFCFFFFFFF7FFFFFF3D
:1010E000F4FFFFFFFBFFFFFFF8FFFFFFF4FFFFFF31
:1010F000FCFFFFFFF7FFFFFFF4FFFFFFFBFFFFFF1A
:10110000F8FFFFFFF6FFFFFFFAFFFFFFF8FFFFFF0B
:10111000F6FFFFFFFDFFFFFFFBFFFFFFF9FFFFFFF4
:10112000FDFFFFFFF9FFFFFFF7FFFFFFFEFFFFFFE0
:10113000FCFFFFFFF7FFFFFFFBFFFFFFF8FFFFFFD5
:10114000F6FFFFFFFCFFFFFFFAFFFFFFF6FFFFFFC9
:10115000FDFFFFFFFBFFFFFFF9FFFFFFFCFFFFFFAE
:10116000FAFFFFFFF6FFFFFFFEFFFFFFFCFFFFFFA1
:10117000F7FFFFFFFBFFFFFFF8FFFFFFF6FFFFFF9B
:10118000FEFFFFFFFCFFFFFFF7FFFFFF000058021D
:1011900046056608540BD80E5C127017FC21F82A1D
:1011A00070305834DC37663A8C3C803EFF3FFFFF9E
:1011B0000000580246056608540BA00FD4172823D8
:1011C000F82A442F643284354038663A8C3C803E9D
:1011D000FF3FFFFF00000000070000000C000000C0
:1011E00010000000130000001A0000001F000000A3
:1011F00000000000070000000C00000010000000CC
:1012000013000000180000001C0000002C01130156
:10121000FA00E100C800AF0096007D0064004B00BA
:101220003200190000000000CDCC4C3DCDCCCC3DAF
:101230009A99193ECDCC4C3E0000803E9A99993E39
:101240003333B33ECDCCCC3E6666E63EFBFFFFFFBC
:10125000F7FFFFFFF6FFFFFFFBFFFFFFF7FFFFFFBB
:10126000F6FFFFFFFBFFFFFFF7FFFFFFF6FFFFFFAC
:10127000FDFFFFFFFCFFFFFFF8FFFFFFFDFFFFFF8C
:10128000FCFFFFFFF8FFFFFFFDFFFFFFFCFFFFFF7D
:10129000F8FFFFFFFBFFFFFFF7FFFFFFF6FFFFFF7A
:1012A000FBFFFFFFF7FFFFFFF6FFFFFFFBFFFFFF67
:1012B000FAFFFFFFF8FFFFFFFCFFFFFFF9FFFFFF53
:1012C000F8FFFFFFFDFFFFFFFCFFFFFFF8FFFFFF41
:1012D000FCFFFFFFFAFFFFFFF7FFFFFFFBFFFFFF32
:1012E000F7FFFFFFF4FFFFFFFBFFFFFFF7FFFFFF2D
:1012F000F4FFFFFFFBFFFFFFF7FFFFFFF4FFFFFF20
:10130000FDFFFFFFF8FFFFFFF4FFFFFFFDFFFFFF03
:10131000F8FFFFFFF4FFFFFFFDFFFFFFF8FFFFFFF8
:10132000F4FFFFFFFBFFFFFFF7FFFFFFF4FFFFFFEF
:10133000FBFFFFFFF7FFFFFFF4FFFFFFFBFFFFFFD8
:10134000F8FFFFFFF4FFFFFFFCFFFFFFF9FFFFFFC8
:10135000F4FFFFFFFDFFFFFFF8FFFFFFF4FFFFFFBC
:10136000FCFFFFFFF7FFFFFFF4FFFFFF0000780522
:10137000220B0410B4143219B01DFC214826FE299A
:10138000822D383126344637663A223DFF3FFFFF33
:101390000000D007100E88133219AA1E28237427C4
:1013A0005C2B442F643284354038663A8C3C803E56
:1013B000FF3FFFFF0000540BEC13FA1908201C2517
:1013C0003629EC2C0C302C33E8357238663AF63B73
:1013D000863D163FFF3FFFFF0000CC10581BFC214D
:1013E000AC26C62A7C2E3831F4334C36A438983AD1
:1013F0005A3C543D803E7A3FFF3FFFFF0000000013
:10140000070000000C0000001000000013000000A6
:10141000180000001A000000070000000C00000087
:101420001000000013000000180000001A00000067
:101430001F000000FBFFFFFFF7FFFFFFF4FFFFFFB0
:10144000FBFFFFFFF7FFFFFFF4FFFFFFFDFFFFFFC5
:10145000F7FFFFFFF4FFFFFFFDFFFFFFF8FFFFFFB8
:10146000F4FFFFFFFAFFFFFFF7FFFFFFF4FFFFFFAF
:10147000FBFFFFFFF7FFFFFFF4FFFFFFFBFFFFFF97
:10148000F7FFFFFFF4FFFFFFFBFFFFFFF7FFFFFF8B
:10149000F4FFFFFFFDFFFFFFF8FFFFFFF4FFFFFF7B
:1014A000FDFFFFFFF8FFFFFFF4FFFFFFFDFFFFFF62
:1014B000F8FFFFFFF4FFFFFFFAFFFFFFF8FFFFFF5A
:1014C000F4FFFFFF34150100E09BFF1F0000FF0F3A
:1014D0008C9DFF1F0000FF0FB95000000015010098
:1014E000849DFF1F32005E0100000000000000002C
:1014F0005950000054485200534E53004D4158007B
:10150000544F5543482053454E5345004558545277
:101510004120434F4E54524F4C4C45520000000066
:1015200050495443482042454E44000042495445E6
:101530000000000042524541544800FF0C150100D4
:10154000DC9CFF1FF401A00FD89CFF1FF401A00F2B
:10155000655000002C150100489DFF1FBC025C1265
:10156000609DFF1FBC025C129D5000002015010011
:101570002A9DFF1FF401A00F729BFF1FF401A00F13
:1015800081500000841E01008C1E0100781E0100A5
:101590007C1E0100801E0100EC1C01003C1E0100AD
:1015A000581E01005C1E0100601E0100641E010047
:1015B000681E01006C1E0100701E0100441E010027
:1015C000741E0100EC1C0100E81C01004C1E01000F
:1015D000501E0100541E0100EC1C01003C1E0100C5
:1015E000401E0100441E0100481E0100281E01008B
:1015F0002C1E0100301E0100341E0100381E0100A7
:1016000088250100201E0100241E0100941E0100F7
:10161000981E01009C1E0100A01E0100A41E0100D6
:10162000A81E0100AC1E0100B01E0100B41E010086
:10163000B81E0100BC1E0100C01E0100C41E010036
:1016400001000000C81E01000700000000000000AB
:10165000000000000000000000000000000000008A
:10166000000000000000000000000000000000007A
:10167000000000000000000000000000000000006A
:10168000000000000000000000000000000000005A
:10169000000000000000000000000000000000004A
:1016A000000000000000000000000000000000003A
:1016B000000000000000000000000000000000002A
:1016C000000000000000000000000000000000001A
:1016D000000000000000000000000000000000000A
:1016E00000000000000000000000000000000000FA
:1016F00000000000000000000000000000000000EA
:1017000000000000000000000000000000000000D9
:1017100000000000000000000000000000000000C9
:1017200000000000000000000000000000000000B9
:1017300000000000000000000000000000000000A9
:101740000000000000000000000000000000000099
:101750000000000000000000000000000000000089
:101760000000000000000000000000000000000079
:101770000001FFFFFFE3600007736000000000004E
:101780000001FFFFFFE360000EE3600000000000C7
:1017900000018000000360001DC360000000000025
:1017A0000001BFFFFFE360003B836000000000001A
:1017B0000001BFFFFFE3600077036000000000004E
:1017C0000001B00000036000EE03600000000000B4
:1017D0000001B00000036001DC03600000000000B5
:1017E0000001B00000036003B803600000000020A7
:1017F0000001B0000003600770036000000000609B
:101800000001BFFFFFE3600EE00360000000006026
:101810000001BFFFFFE3601DC00360000003006024
:10182000000180000003603B80036000000300E0D3
:101830000001BFFFFFE3607700036000000300C00A
:101840000001BFFFFFE360EE00036000000380C003
:101850000001B000000361DC00036000000780C0ED
:101860000001B000000363B8000360000007C0C0BF
:101870000001B00000036770000360000006C0C0F4
:101880000001B00000036EE000036000000660C1CC
:101890000101B00000037DC000036000000630C3FA
:1018A0000301BFFFFFE37B8000036000000C30C337
:1018B0000701BFFFFFE3770000036000000C1CC3BB
:1018C0000601800000030E0000036000000C0CC243
:1018D0000E01FFFFFFE3FC0000036000000C0EC6DA
:1018E0001E01FFFFFFE3F80000036000000C07C6C5
:1018F0001E0000000000000000000000000C03C6F5
:10190000760000000000000000000000000C01C78D
:10191000E60000000000000000000000000C00C70E
:10192000C60000000000000000000000000C0003E2
:10193000060000000000000000000000000C000095
:10194000000000000000000000000000000C00008B
:101950000000000000000000000000000000000087
:101960000000000000000000000000000000000077
:101970000000000000000000000000000000000067
:101980000000000000000000000000000000000057
:101990000000000000000000000000000000000047
:1019A0000000000000000000000000000000000037
:1019B0000000000000000000000000000000000027
:1019C0000000000000000000000000000000000017
:1019D0000000000000000000000000000000000007
:1019E00000000000000000000000000000000000F7
:1019F00000000000000000000000000000000000E7
:101A000000000000000000000000000000000000D6
:101A100000000000000000000000000000000000C6
:101A200000000000000000000000000000000000B6
:101A300000000000000000000000000000000000A6
:101A40000000000000000000000000000000000096
:101A50002821010034210100E69CFF1F00000A003C
:101A600001000000295F0000B55B000000000000DD
:101A70000000000020220100B4210100749BFF1F20
:101A80000000300000000000216E0000095B000033
:101A90000000000038200100000005010A000000DD
:101AA000788DFF1FC95F00000600000009000000DC
:101AB000288FFF1F0000000038220100B421010020
:101AC0003C9DFF1F0000300000000000416E000040
:101AD000195B00000000000000000000FC21010074
:101AE000B4210100BC9CFF1F00003000000000007A
:101AF000416E0000DD5A0000000000002C1F0100B4
:101B0000000002010B000000708FFF1F00000000AA
:101B1000902101009C210100889BFF1F0000010013
:101B200001000000D9630000555B000000000000C8
:101B300000000000F0210100B4210100BE9CFF1F45
:101B40000000300000000000416E0000DD5A00007F
:101B5000000000000100000040200100060000001D
:101B6000C81E01000000040508000000508BFF1F84
:101B70000100000038200100090000000000000002
:101B800001000000317A0000000000005022010036
:101B9000B4210100389DFF1F00003000000000004C
:101BA000416E0000195B0000000000000100000011
:101BB000642001000300000000000000CC210100AF
:101BC000B4210100C29CFF1F000030000000000093
:101BD000416E0000A15A000000000000000000005B
:101BE000E4210100B4210100769BFF1F00003000BA
:101BF00000000000116E0000CD5A0000000000003F
:101C00000000000014220100B4210100B89CFF1F55
